:100000000C943D1C0C946E1C0C946E1C0C946E1C79
:100010000C946E1C0C946E1C0C946E1C0C946E1C38
:100020000C946E1C0C946E1C0C946E1C0C946E1C28
:100030000C946E1C0D9469030C946E1C0C946E1C35
:100040000C946E1C0C94F2D50C946E1C0C946E1CCB
:100050000C946E1C0C9463D70C9495D60C9429FECA
:100060000C946E1C0C94BBD70C94E5D70C946E1CAE
:100070000C946E1C0C946E1C0C946E1C0C946E1CD8
:100080000C946E1C0C946E1C0C946E1C0C946E1CC8
:100090000C946E1C0C946E1C0C946E1C0C9437FC0F
:1000A0000C946E1C0C946E1C0C946E1C0C946E1CA8
:1000B0000C946E1C0C946E1C0C946E1C0C946E1C98
:1000C0000C946E1C0C946E1C0C946E1C0C946E1C88
:1000D0000C946E1C0C946E1C0C946E1C0C946E1C78
:1000E0000C946E1C2C9344934493449344934493F4
:1000F0004493449344934493449344934493449348
:100100004493449344934493449344934493449337
:1001100044934493449344931B93CD92D79251922A
:100120004493FD9207934493449362923F92449385
:10013000F39244931193E992E1924493449344934C
:10014000AF92B992C392449344934493449344939B
:1001500044934493449344931B93CD92D7925192EA
:100160004493FD9207934493449362923F92449345
:10017000F39244931193E992E1924493449344930C
:10018000AF92B992C3922CB0B5B048B179B2B6BFB4
:10019000B6BFB6BFB6BFB6BFB6BFB6BFB6BFB6BFB7
:1001A000D9B10DB243B2B6BFB6BFB6BFB6BFB6BFC8
:1001B000B6BFB6BFB6BFB6BFB6BFB6BF5BB5BDB5FF
:1001C0001DB67DB6DDB63DB79DB7B6BF7DBB08B8E1
:1001D00065B8C2B81FB97CB9D9B936BAA3BA10BBD1
:1001E000B6BFB6BFB6BFB6BFB6BFDEB3ABB401B421
:1001F000C5BBF4BB5CBCC5BCDCBC14BD43BD72BD9F
:10020000C7BD1EBE73BECCBEEBBEF3BCB6BFB6BF91
:10021000B6BFB6BFB6BFB6BFB6BFB6BFB6BFB6BF36
:10022000B6BFB6BFB6BFADB3B6BFB6BFB6BFB6BF3B
:10023000B6BFB6BFB6BFB6BF62BFB6BF7AB4B6BFB1
:10024000B6BFB6BF12BF3BBFB6BFB6BFB6BFB6BF25
:100250001FB0B6BFB6BFBCB252B390B303B589FDF1
:100260008EFD93FD9DFDA7FD20FEB1FDB9FDC1FDF5
:10027000CBFDD5FDDFFDEEFDF8FD20FE02FE0CFE00
:1002800016FE4CFF4FFF3EFF42FF48FF86FF53FF25
:1002900057FF5DFF61FF65FF6BFF6FFF73FF86FF19
:1002A00079FF7DFF81FF07634236B79BD8A71A39D4
:1002B000685618AEBAAB558C1D3CB7CC5763BD6DB4
:1002C000EDFD753EF6177231BF000000803F05A8B6
:1002D0004CCDB2D44EB93836A9020C50B9918688AB
:1002E000083CA6AAAA2ABE000000803F0D941D006B
:1002F000436F6C6420657874727573696F6E2064E7
:100300006973616C6C6F77656400436F6C64206522
:100310007874727573696F6E20616C6C6F77656449
:10032000004175746F726574726163743A0053654D
:100330007474696E67206D6F746F7220637572726A
:10034000656E742E2E2E00536574204D6963726F96
:100350007374657070696E6700547269676765725F
:10036000696E67207761746368646F672E204966E1
:10037000206163746976617465642C2074686520FB
:100380007072696E7465722077696C6C2072657327
:1003900065742E0053657474696E672054687265C5
:1003A00073686F6C6420546F3A00494E5420504972
:1003B0004E3A20004D323531200020746F2000531A
:1003C000657420766F6C756D6574726963206578ED
:1003D00074727573696F6E20666F722065787472BF
:1003E00075646572200044697361626C656420768F
:1003F0006F6C756D6574726963206578747275735E
:10040000696F6E20666F72206578747275646572AC
:1004100020004D313134200048656174696E6720D9
:1004200045787472756465720050696E2063616E00
:10043000206E6F7420626520736574206279204D90
:1004400034322C206D617920696E20696E76616C82
:100450006964206F7220696E207573652E200049D3
:100460006C6C6567616C20532076616C75652066E5
:100470006F72204D3432005A2028432920746F7740
:10048000657220666C6F6F722073657420746F3AAA
:100490002000592028422920746F77657220666CED
:1004A0006F6F722073657420746F3A200058202893
:1004B000412920746F77657220666C6F6F722073AC
:1004C000657420746F3A2000526F64205261646931
:1004D00075732073657420746F3A2000473133348C
:1004E0002000506F7346726F6D53746570733A00DD
:1004F000436F6D7044656C74613A0043616C69626E
:10050000726174696F6E206D6F76656D656E7420B3
:100510006973206C696D6974656420746F20313073
:100520006D6D2E004669727374206D6F7665207450
:100530006F20746F75636820617420782C793D306A
:100540002C3020746F206175746F2D736574207268
:1005500061646975732E0043616C696272617469CC
:100560006F6E206D6F76656D656E74206973206C9B
:10057000696D6974656420746F2031306D6D2E0073
:1005800043616E6E6F742073657420726164697567
:100590007320616E6420666C6F6F722061742073CB
:1005A000616D652074696D652E0043616C696272CE
:1005B0006174696F6E20636F6465206973206C6974
:1005C0006D6974656420746F20626F74746F6D2040
:1005D000313025206F66205A20686569676874008D
:1005E00052656C617469766520706F736974696FA8
:1005F0006E696E67004162736F6C75746520706F11
:10060000736974696F6E696E670047363920005AE6
:100610003A2000593A2000583A20004F46465345A8
:100620005453204F464620425920544F4F204D5599
:100630004348205F20545259494E47204147414981
:100640004E3A200053657474696E672050726F6271
:10065000652053656E736974697669747920546F87
:100660003A005A2070726F6265206661696C656439
:10067000206F6E2073656E73697469766974793A58
:10068000200053657474696E672050726F62652034
:1006900053656E736974697669747920546F3A0092
:1006A0005A2070726F6265206661696C6564206FA4
:1006B0006E2073656E73697469766974793A200087
:1006C00053657474696E672050726F62652053655C
:1006D0006E736974697669747920546F3A005A2090
:1006E00070726F6265206661696C6564206F6E2050
:1006F00073656E73697469766974793A2000686508
:100700006865004E6577205261646975733A200010
:100710004F6C64205261646975733A200043616CC8
:1007200063756C61746564205261646975732069D6
:100730007320626164203A0053657474696E6720A7
:1007400050726F62652053656E736974697669745F
:100750007920546F3A005A2070726F62652066618A
:10076000696C6564206F6E2073656E736974697659
:100770006974793A200053657474696E6720507209
:100780006F62652053656E73697469766974792048
:10079000546F3A005A2070726F6265206661696C0E
:1007A0006564206F6E2073656E7369746976697411
:1007B000793A2000473332200050524F42452D5A9B
:1007C0004F46465345543A004733300053657474DE
:1007D000696E672050726F62652053656E7369742D
:1007E000697669747920546F3A0050726F6265734C
:1007F00020646F206E6F74206D617463682E204FCB
:100800006666206279200047333020004D31313751
:100810002043414C4942524154494F4E20434F4D91
:10082000504C4554450068656865004E6577204822
:100830006F72697A6F6E74616C205261646975734E
:100840003A20004F6C6420486F72697A6F6E746151
:100850006C205261646975733A200043616C637562
:100860006C617465642052616469757320697320DA
:100870006261643A20004D3131372043414C494296
:10088000524154494F4E204641494C454400436132
:100890006C6962726174696F6E204661696C65642F
:1008A0000053657474696E672050726F62652053DF
:1008B000656E736974697669747920546F3A005A69
:1008C0002070726F626520284852202D205A2074B3
:1008D0006F77657229206661696C6564206F6E2090
:1008E00073656E73697469766974793A20004E6530
:1008F00077205A204865696768743A004F6C642015
:100900005A204865696768743A004D313137204391
:10091000414C4942524154494F4E204641494C4571
:10092000440043616C6962726174696F6E20466154
:10093000696C65640053657474696E672050726FEA
:1009400062652053656E73697469766974792054A1
:100950006F3A005A2070726F626520284852202D2D
:100960002043656E74657220506F696E742920662D
:1009700061696C6564206F6E2073656E736974695C
:10098000766974793A200047363920005A3A2000B7
:10099000593A2000583A20004D31313720456E64D5
:1009A00073746F70204F6666736574204572726F42
:1009B00072004F464653455453204F4646204259F5
:1009C00020544F4F204D5543482E2041626F727482
:1009D000696E672E2053656E7369746976697479E0
:1009E0003A20004D3131372043414C494252415465
:1009F000494F4E204641494C45440043616C696271
:100A0000726174696F6E204661696C65640053653C
:100A10007474696E672050726F62652053656E73DF
:100A20006974697669747920546F3A005A2070723B
:100A30006F626520285A20546F776572292066619D
:100A4000696C6564206F6E2073656E736974697676
:100A50006974793A20004D3131372043414C494285
:100A6000524154494F4E204641494C454400436150
:100A70006C6962726174696F6E204661696C65644D
:100A80000053657474696E672050726F62652053FD
:100A9000656E736974697669747920546F3A005A87
:100AA0002070726F626520285920546F7765722913
:100AB000206661696C6564206F6E2073656E736972
:100AC0007469766974793A20004D31313720434199
:100AD0004C4942524154494F4E204641494C4544AD
:100AE0000043616C6962726174696F6E204661696E
:100AF0006C65640053657474696E672050726F6230
:100B0000652053656E736974697669747920546FD2
:100B10003A005A2070726F626520285820546F770F
:100B2000657229206661696C6564206F6E2073654B
:100B30006E73697469766974793A2000456E6473DE
:100B4000746F70287329206E6F7420776F726B69D1
:100B50006E672070726F7065726C79005A20005950
:100B600020005820004572726F723A20004D3131DA
:100B70003720454E4453544F50204552524F520057
:100B80004D3130342053300A4D3134302053300A47
:100B90004D313037004D31313720493243204572D5
:100BA000726F722E2041626F7274696E67004932F3
:100BB00043204572726F72202D2043616C6962720E
:100BC0006174696F6E2041626F7274656400456E76
:100BD0006473746F70287329206E6F7420776F723E
:100BE0006B696E672070726F7065726C79005A2045
:100BF000005920005820004572726F723A20004D53
:100C000031313720454E4453544F50204552524FB6
:100C100052006578656375746547436F6465202F7E
:100C200020717565756544656C74614D6F766520DE
:100C300072657475726E73206572726F7200696985
:100C40007332646820616363656C65726F6D65748F
:100C5000657220696E697469616C697A696E672E64
:100C60002E2E00616363656C65726F6D65746572CD
:100C7000206932632072656376206661696C656401
:100C80002E00616363656C65726F6D6574657220BB
:100C9000777269746520693263206661696C656486
:100CA0002E00616363656C65726F6D65746572209B
:100CB00073656E6420693263206661696C65642EB9
:100CC0000000000100250030001D000C001E002463
:100CD0000031001C000B00180023002F001B000A2D
:100CE0000017000D0047000300040022002B001A2B
:100CF0000041004200000002003500206465672EBC
:100D0000204300206D656173757265642000457233
:100D1000726F723A436F756C64206E6F7420686FE7
:100D20006C642074656D7065726174757265200005
:100D3000206D730020616674657220004572726FC9
:100D4000723A54656D702E20726169736564207407
:100D50006F20736C6F772E2052697365203D2000E1
:100D60004739310A4731452D313830463630303039
:100D70000A473930004D3131372045787472756437
:100D8000657220300A54300A4D38342050340A47F6
:100D900039310A47314531373246363030300A472B
:100DA000314535463530300A473930001C151C14A2
:100DB0000000002243141F1FC0116C11FC10AC1066
:100DC0000000000000002410180FC80E4C0ED00DBB
:100DD0000400081D900058091C01B007A801C806AE
:100DE00034023006C002C0054C036805D80318055C
:100DF0006404D004F00498047C0560040806300400
:100E0000940600042007D003AC07A8033808800329
:100E1000C408580350093003DC090803680AD802E3
:100E2000F40AB002800B88020C0C6002980C3002AD
:100E3000240DF801B00DC0013C0E8001C80E300138
:100E4000540FB800B40F2800E00F00000400401D4C
:100E5000900060091C01B007A801D00634023806D2
:100E6000C002C8054C036805D80318056404D804FB
:100E7000F00498047C05600408063004940600041D
:100E80002007D003AC07A80338088003C408580320
:100E900050093003DC090803680AE002F40AB802CA
:100EA000800B88020C0C6002980C3002240DF801B3
:100EB000B00DC0013C0E8001C80E3001540FB800C7
:100EC000B40F2800E00F000004000016D800C00690
:100ED000AC0178058002C004540348042804E803E8
:100EE000FC049803D0055003A40618037807D80221
:100EF0004C08A80220097002F4093802C80A080246
:100F00009C0BD001700C9001440D5001180EF8009C
:100F1000EC0E8800C00F00000400681D4C00500B50
:100F200094005809DC0050082401A8076C01280728
:100F3000B401C006FC017006440228068C02F005CC
:100F4000D402B8051C03880564035805AC033005BA
:100F5000F40310053C04E8048404C804CC04A80489
:100F6000140590045C057004A4055804EC053804CD
:100F7000340620047C060804C406F0030C07D803DA
:100F80005407C8039C07B003E40798032C088003A8
:100F900074087003BC085803040948034C09300363
:100FA00094091803DC090803240AF0026C0AE00221
:100FB000B40AC802FC0AB002440BA0028C0B8802DF
:100FC000D40B70021C0C5802640C4002AC0C2802BA
:100FD000F40C10023C0DF001840DD801CC0DB801C9
:100FE000140E98015C0E7001A40E4801EC0E18015D
:100FF000340FD8007C0F8800C40F0800FC0F0000DD
:1010000000000000000000000000000000000000E0
:1010100000000000000000000000000000000000D0
:10102000000000000000401F450060094F0010094B
:101030005C00C0086B0070087D0020089200D0079B
:10104000AC008007CC003007DE00E00623019006EC
:101050005E014006A601F005FF01A0056D025005E6
:10106000F30200059603B0045A046004400510041E
:101070004806C0036E077003A8082003EB09D002DE
:10108000230B8002410C3002390DE001040E900167
:10109000A20E4001170FF000690FA000A20F500030
:1010A000C60F0000DD0FB0FFEB0F60FF0400700DF6
:1010B000D8004804AC0158038002D80254038002CF
:1010C00028043802FC040002D005C801A4069801D7
:1010D000780770014C08480120091801F409F00054
:1010E000C80AC8009C0BA000700C7000440D3800AA
:1010F000180E0000EC0EA8FFC00FE8FE0400001B55
:1011000054006009640010097400C008840070086D
:101110009C002008B800D007D800800700013007E5
:101120002C01E00668019006AC0140060002F005C3
:101130006802A005E0025005740300052404B00411
:10114000F0046004DC051004E406C0030408700326
:1011500030092003780B8002600DE001A80E4001E9
:10116000680FA000C00F0000E80F60FF0400801AA5
:10117000D8009808AC012007800250065403C80527
:1011800028045805FC040005D005B004A406680432
:10119000780728044C08E8032009B003F409700319
:1011A000C80A38039C0BF802700CB002440D6802A8
:1011B000180E0802EC0E8801C00F8800F00F000026
:1011C0000000A00F5C006009690010097900C008E8
:1011D0008C007008A2002008BD00D007DE00800748
:1011E000050130073401E0066D019006B2014006AA
:1011F0000702F0056D02A005E80250057B0300051B
:101200002B04B004F8046004EB06C0033509200386
:101210007F0B8002650DE001B00E40011D0FF00054
:10122000480FC8006C0FA000ED0F60FFFE0F48FED6
:101230000000002110422063308440A550C660E7C2
:1012400070088129914AA16BB18CC1ADD1CEE1EF7B
:10125000F13112100273325222B5529442F772D613
:1012600062399318837BB35AA3BDD39CC3FFF3DECB
:10127000E36224433420040114E664C774A4448563
:10128000546AA54BB528850995EEE5CFF5ACC58D1B
:10129000D55336722611163006D776F6669556B4B3
:1012A000465BB77AA719973887DFF7FEE79DD7BC6B
:1012B000C7C448E5588668A7784008611802282303
:1012C00038CCC9EDD98EE9AFF9488969990AA92BBB
:1012D000B9F55AD44AB77A966A711A500A333A1253
:1012E0002AFDDBDCCBBFFB9EEB799B588B3BBB1A0B
:1012F000ABA66C877CE44CC55C222C033C600C41A3
:101300001CAEED8FFDECCDCDDD2AAD0BBD688D495A
:101310009D977EB66ED55EF44E133E322E511E70F2
:101320000E9FFFBEEFDDDFFCCF1BBF3AAF599F78AA
:101330008F8891A981CAB1EBA10CD12DC14EF16F5B
:10134000E18010A100C230E32004502540467067C0
:1013500060B9839893FBA3DAB33DC31CD37FE35EEC
:10136000F3B1029012F322D2323542145277625610
:1013700072EAB5CBA5A89589856EF54FE52CD50DFC
:10138000C5E234C324A01481046674476424540560
:1013900044DBA7FAB79987B8975FE77EF71DC73C8C
:1013A000D7D326F2369106B01657667676154634B0
:1013B000564CD96DC90EF92FE9C899E9898AB9AB9C
:1013C000A94458654806782768C018E1088238A300
:1013D000287DCB5CDB3FEB1EFBF98BD89BBBAB9A2C
:1013E000BB754A545A376A167AF10AD01AB32A9250
:1013F0003A2EFD0FED6CDD4DCDAABD8BADE89DC93C
:101400008D267C076C645C454CA23C832CE01CC19F
:101410000C1FEF3EFF5DCF7CDF9BAFBABFD98FF8CB
:101420009F176E367E554E745E932EB23ED10EF0EF
:101430001E7C3C3E5E2B3D3F2F5B5D3B2C2A225C9D
:10144000004D617854656D703A004469616D657452
:1014500065723A00416363656C65726174696F6EB1
:101460003A004D617853706565643A004A65726B65
:101470003A004D617842656454656D703A0050726F
:10148000696E746572547970653A44656C74610074
:101490005A54726176656C416363656C3A005954C5
:1014A000726176656C416363656C3A005854726191
:1014B00076656C416363656C3A005A5072696E746C
:1014C000416363656C3A00595072696E744163639D
:1014D000656C3A00585072696E74416363656C3A8A
:1014E000005A53697A653A005953697A653A005847
:1014F00053697A653A005A4D61783A00594D6178DE
:101500003A00584D61783A005A4D696E3A00594D8B
:10151000696E3A00584D696E3A004A65726B5859C7
:101520003A005072696E746C696E654361636865F8
:101530003A00454550524F4D3A004175746F6C6505
:1015400076656C3A005A50726F62653A0043617377
:10155000654C69676874733A00537570706F727484
:101560004C6F63616C46696C616D656E7463686134
:101570006E67653A00537570706F7274473130470B
:1015800031313A005A486F6D654469723A005948E2
:101590006F6D654469723A0058486F6D65446972B1
:1015A0003A00536F667477617265506F7765725356
:1015B00077697463683A004C43443A0046616E3A76
:1015C000005344436172643A004865617465644243
:1015D00065643A004D6978696E6745787472756420
:1015E00065723A004E756D45787472756465723A2D
:1015F00000496E7075744275666665723A004261A4
:101600007564726174653A004E6F20636173652082
:101610006C6967687473004D313134200064656C07
:101620006179203130306D732E00686F6D654178BF
:1016300069732000686F6D6541786973202F207190
:101640007565756544656C74614D6F76652072656E
:101650007475726E73206572726F7200486F6D657B
:101660002044656C7461005072696E7465723A3A18
:10167000736574757020006D6F7665546F52656187
:101680006C202F20717565756544656C74614D6FB4
:1016900076652072657475726E73206572726F72F2
:1016A000006D6F7665546F202F20717565756544E8
:1016B000656C74614D6F76652072657475726E73BA
:1016C000206572726F720053746570706572204489
:1016D000697361626C6564004B696C6C6564006978
:1016E00073506F736974696F6E416C6C6F7765646A
:1016F00020005344206572726F72206669786564B9
:10170000005344206572726F7220646964206E6FAA
:1017100074207265636F76657221005344205265B0
:101720006164204572726F720055706C6F616469FC
:101730006E672E2E2E00005344207072696E742046
:1017400073746F7070656420627920757365722E92
:10175000005344206361726420696E73657274651E
:1017600064005344204361726420696E736572742F
:10177000656400534420436172642072656D6F7626
:10178000656400534420636172642072656D6F76F6
:10179000656400457874722E00436F6E6669673A1F
:1017A000004F6E6520686561746572207365656DB4
:1017B00073206465636F75706C65642066726F6D0D
:1017C00020746865726D6973746F72202D2064696E
:1017D0007361626C696E6720616C6C20666F722049
:1017E000736166657479210048656174657220646F
:1017F00065636F75706C6564004372656174696FD1
:101800006E206661696C6564004469726563746F1B
:10181000727920637265617465640044656C6574F7
:10182000696F6E206661696C65640046696C65204D
:1018300064656C6574656400446F6E6520736176E1
:10184000696E672066696C652E0057726974696EEF
:101850006720746F2066696C653A20006F70656E52
:10186000206661696C65642C2046696C653A2000CD
:101870004E6F74205344207072696E74696E6700F5
:101880005344207072696E74696E67206279746562
:10189000200066696C652E6F70656E206661696CEC
:1018A00065640046696C652073656C656374656486
:1018B000002053697A653A0046696C65206F70654F
:1018C0006E65643A00456E642066696C65206C69DB
:1018D000737400426567696E2066696C65206C6987
:1018E0007374006572726F722077726974696E67C3
:1018F00020746F2066696C6500534420696E6974BA
:10190000206661696C00616476616E6365204C20BD
:101910005B303D6F66665D006578747275646572F4
:1019200020636F6F6C6572207370656564205B3037
:101930002D3235355D0064697374616E63652074A2
:101940006F2072657472616374207768656E2068B9
:10195000656174696E67205B6D6D5D0074656D70A7
:101960002E20666F722072657472616374696F6E87
:10197000207768656E2068656174696E67205B43D7
:101980005D0074656D702E2073746162696C697A94
:10199000652074696D65205B735D00592D6F666607
:1019A000736574205B73746570735D00582D6F668A
:1019B00066736574205B73746570735D0050494491
:1019C000206D61782076616C7565205B302D323535
:1019D000355D0050494420442D6761696E005049CF
:1019E0004420492D6761696E0050494420502D679D
:1019F00061696E2F646561642D74696D650050497D
:101A000044206472697665206D696E0050494420F7
:101A10006472697665206D61780068656174206D17
:101A2000616E61676572205B302D335D00616363B9
:101A3000656C65726174696F6E205B6D6D2F735E8E
:101A4000325D0073746172742066656564726174DE
:101A500065205B6D6D2F735D006D61782E2066656E
:101A6000656472617465205B6D6D2F735D007374C6
:101A700065707320706572206D6D00436F72722EF9
:101A800020646961676F6E616C2043205B6D6D5DE2
:101A900000436F72722E20646961676F6E616C2003
:101AA00042205B6D6D5D00436F72722E2064696130
:101AB000676F6E616C2041205B6D6D5D004D6178DC
:101AC000207072696E7461626C6520726164697500
:101AD00073205B6D6D5D00546F776572205A2065D1
:101AE0006E6473746F70206F6666736574205B73C9
:101AF000746570735D00546F776572205920656E50
:101B00006473746F70206F6666736574205B7374A2
:101B10006570735D00546F776572205820656E6440
:101B200073746F70206F6666736574205B73746581
:101B300070735D005365676D656E74732F732066F7
:101B40006F722074726176656C005365676D656EA7
:101B500074732F7320666F72207072696E74696E71
:101B60006700486F72697A6F6E74616C20726F647F
:101B70002072616469757320617420302C30205BA1
:101B80006D6D5D00446961676F6E616C20726F649A
:101B9000206C656E677468205B6D6D5D00486F6DCD
:101BA000696E67206665656472617465205B6D6D42
:101BB0002F735D004D61782E2066656564726174D7
:101BC00065205B6D6D2F735D0053746570732070BD
:101BD0006572206D6D0054726176656C206163637F
:101BE000656C65726174696F6E205B6D6D2F735EDD
:101BF000325D00416363656C65726174696F6E206C
:101C00005B6D6D2F735E325D004D61782E206A65CD
:101C1000726B205B6D6D2F735D005A206D617820B3
:101C20006C656E677468205B6D6D5D0059206D6139
:101C300078206C656E677468205B6D6D5D00582060
:101C40006D6178206C656E677468205B6D6D5D00FA
:101C50005A20686F6D6520706F73205B6D6D5D003D
:101C60005920686F6D6520706F73205B6D6D5D002E
:101C70005820686F6D6520706F73205B6D6D5D001F
:101C800053746F7020737465707065722061667430
:101C9000657220696E6163746976697479205B6D21
:101CA000732C303D6F66665D004D61782E20696E45
:101CB0006163746976652074696D65205B6D732C52
:101CC000303D6F66665D005072696E7465722061AA
:101CD0006374697665205B735D0046696C616D6550
:101CE0006E74207072696E746564205B6D5D004176
:101CF0006476616E63656420557365720042617538
:101D00006472617465004550523A33200045505268
:101D10003A3220004550523A3120004550523A3074
:101D2000200050726F746F636F6C207665727369F8
:101D30006F6E206368616E6765642C2075706772D2
:101D40006164696E6700436F6E666967757261747E
:101D5000696F6E20726573657420746F20646566A8
:101D600061756C74732E00436F6E6669677572617E
:101D700074696F6E206C6F616465642066726F6D4C
:101D800020454550524F4D2E00436F6E6669677572
:101D9000726174696F6E2073746F72656420746F02
:101DA00020454550524F4D2E004175746F6C65763D
:101DB000656C206163746976652028312F302900B5
:101DC0005A2D70726F6265205933005A2D70726FF0
:101DD0006265205833005A2D70726F626520593247
:101DE000005A2D70726F6265205832005A2D707241
:101DF0006F6265205931005A2D70726F62652058EC
:101E000031005A2D70726F626520782D792D7370B4
:101E1000656564205B6D6D2F735D005A2D70726F68
:101E20006265207370656564205B6D6D2F735D0066
:101E30005A2D70726F6265206F66667365742079C3
:101E4000205B6D6D5D005A2D70726F6265206F664C
:101E5000667365742078205B6D6D5D004D61782E32
:101E6000207A2D70726F6265202D20626564206477
:101E70006973742E205B6D6D5D005A2D70726F62F8
:101E80006520686569676874205B6D6D5D007761CA
:101E90006974005072696E7465722068656967685C
:101EA000743A005A2D70726F6265206661696C65C4
:101EB00064005472616E73666F726D6174696F6EE7
:101EC000206D61747269783A004175746F6C657643
:101ED000656C696E672064697361626C656400415A
:101EE00075746F6C6576656C696E6720656E61628E
:101EF0006C6564004175746F6C6576656C206D610E
:101F00007472697820726573657400004732382FE7
:101F10006E47315A32352F6E005A2D70726F6265DE
:101F20002073746174653A005265736574205A2099
:101F3000686569676874005A2D70726F6265206108
:101F4000766572616765206865696768743A002024
:101F50005374657020566172696174696F6E206692
:101F6000726F6D2050726F626520746F20626564BD
:101F70002044697374616E63653A005A2D70726F04
:101F800062653A005072696E7465722073657420E0
:101F9000696E746F206472792072756E206D6F6443
:101FA0006520756E74696C2072657374617274213A
:101FB000003A20776F726B696E67003A2074656D26
:101FC000702073656E736F7220646566656374005C
:101FD000657874727564657220004D54454D503AB1
:101FE00000504944204175746F74756E65206669B0
:101FF0006E6973686564202120506C61636520748C
:102000006865204B702C204B6920616E64204B6406
:1020100020636F6E7374616E747320696E207468D0
:102020006520436F6E66696775726174696F6E2EA5
:1020300068206F7220454550524F4D005049442052
:102040004175746F74756E65206661696C65642195
:102050002074696D656F7574005049442041757432
:102060006F74756E65206661696C656421205465C6
:102070006D706572617475726520746F2068696730
:102080006800204B643A2000204B693A2000204B26
:10209000703A200020436C61737369632050494497
:1020A000002054753A2000204B753A2000206D61C5
:1020B000783A2000206D696E3A200020643A2000B2
:1020C00020626961733A2000504944204175746F61
:1020D00074756E6520737461727400546172676503
:1020E0007445787472004E6F206D6F766520696E4E
:1020F0002064656C7461207365676D656E7420770C
:10210000697468203E2031207365676D656E742E9A
:1021100020546869732073686F756C64206E6576EF
:1021200065722068617070656E20616E64206D61FB
:102130007920636175736520612070726F626C65D0
:102140006D210044656C746120526164697573206F
:10215000432830293A0044656C74612052616469F7
:10216000757320422830293A0044656C746120520E
:10217000616469757320412830293A00416C7068A8
:10218000612043283930293A00416C70686120424F
:1021900028333330293A00416C706861204128327D
:1021A0003130293A00546F77657220333A00546F0A
:1021B00077657220323A00546F77657220313A00A9
:1021C000496E76616C69642064656C746120636F2C
:1021D0006F7264696E617465202D206D6F76652065
:1021E00069676E6F726564006C696E656172204C20
:1021F0003A00454550524F4D2075706461746564D6
:10220000002C2073706565643D00206C696E65610B
:10221000722073746570733A004A65726B3A007A83
:102220005F6D61783A00795F6D61783A00785F6D33
:1022300061783A004C20004820002069732000207B
:10224000746F2000536574206F75747075743A2034
:10225000004D53312C4D53322050696E730045317F
:102260003A0045303A005A3A00593A0020002C0012
:10227000206D696E0020686F7572732000206461A4
:10228000797320006D20005072696E74696E67204A
:1022900074696D653A005072696E74656420666990
:1022A0006C616D656E743A0046616E73706565644D
:1022B0003A00482E205261646975733A00466C6F8B
:1022C000774D756C7469706C793A0053706565640C
:1022D0004D756C7469706C793A00202F002F003AAC
:1022E0000020403A00543A0020453A00205A3A0073
:1022F00020593A0020583A00583A00467265652045
:1023000052414D3A00556E6B6E6F776E20636F6D64
:102310006D616E643A00536F667477617265205226
:1023200065736574005761746368646F67205265F4
:102330007365740042726F776E206F7574205265FA
:102340007365740045787465726E616C20526573B4
:10235000657400506F7765725570007374617274A4
:1023600000424C4B2000736B6970200020676F7433
:1023700020004572726F723A6578706563746564A7
:10238000206C696E6520005344207265616420658D
:1023900072726F7200205200204A002049002050C3
:1023A00000205300204600204500205A00205900FC
:1023B000205800446F6E65207072696E74696E6794
:1023C0002066696C6500466F726D6174206572727B
:1023D0006F720057726F6E6720636865636B737509
:1023E0006D004563686F3A00526573656E643A002C
:1023F0005761726E696E673A00496E666F3A0045C2
:1024000072726F723A00494E46004E414E006F6B39
:10241000004649524D574152455F4E414D453A5253
:10242000657065746965725F302E39322E322046D0
:1024300049524D574152455F444154453A3230313B
:102440003731313133204D414348494E455F54596E
:1024500050453A4861636B657220483220005265EE
:10246000717565737450617573653A004D3131371C
:1024700020494E5345525420534420434152440076
:102480004D3131372053442043415244204552526C
:102490004F520055495F414354494F4E5F53455495
:1024A0005F4D454153555245445F4F524947494E50
:1024B00020004E6F205344204361726400536875BE
:1024C00074204F666620414C4C204865617473004F
:1024D00050726568656174204142530050726568AE
:1024E00065617420504C410055495F414354494F48
:1024F0004E5F484F4D455F5A200055495F41435458
:10250000494F4E5F484F4D455F59200055495F4147
:102510004354494F4E5F484F4D455F582000554941
:102520005F414354494F4E5F484F4D45414C4C200D
:102530000055495F414354494F4E5F5A504F5349EC
:1025400054494F4E5F464153545F4E4F5445535488
:10255000200055495F414354494F4E5F5A504F53F5
:102560004954494F4E5F4E4F5445535420005549EE
:102570005F414354494F4E5F45504F534954494F73
:102580004E200055495F414354494F4E5F5A504FCA
:10259000534954494F4E5F46415354200055495FBB
:1025A000414354494F4E5F59504F534954494F4E40
:1025B0005F46415354200055495F414354494F4EB3
:1025C0005F58504F534954494F4E5F464153542032
:1025D0000055495F414354494F4E5F5A504F53494C
:1025E00054494F4E200055495F414354494F4E5F77
:1025F00059504F534954494F4E200055495F41436C
:1026000054494F4E5F58504F534954494F4E200044
:1026100042616E6742616E6700536C6F7742616E14
:102620006700446561642054696D65005049440049
:10263000003A002064617973200050657263656E12
:1026400074205072696E7465643A00206465662077
:1026500000465720446174652032303137313131C2
:1026600033004861636B6572204832005365654DE5
:1026700065434E43004861636B657220483200FD3C
:1026800032B3324B32EE31416374696F6E3A256C6E
:102690006100040003004E6F00596573004E2F4126
:1026A000004F6666004F6E000000003FCDCC4C3DF1
:1026B0000AD7A33B6F12033A52657065746965725D
:1026C000207620302E39322E3200004014548025DE
:1026D000000040380000004B0000807000000096B1
:1026E0000000C0DA000000E10000002C010008B288
:1026F000010000C2010000F401000084030090D03A
:10270000030000E803000008070020A107000010F4
:102710000E0040420F0060E3160000000000110AA6
:102720000411040A1111001C1F11111F0000040ADA
:102730000A0A0E1F1F0E001F1111111F0000001F9B
:102740001F1F1F1F0000040A040000000000040EE9
:1027500015041C00000002000006005D27752FC351
:1027600027442C9627972C05280200000700702785
:10277000752F7E27442C9627972CCF2BAA278527A9
:1027800002452D00005072696E74657220536574A5
:1027900074696E6773009D2702332E000041646ADE
:1027A0007573742054656D707300B12702DB2700C8
:1027B00000416476616E6365642053657474696E6C
:1027C000677300CA27025E2D00005072696E74653F
:1027D000722053657474696E67730002000009000B
:1027E000E227752FF028DC28CC28BC28F427A52860
:1027F0008D280528FB2702722B000044656275674F
:1028000067696E67000C2802562E000043616C69F0
:1028100062726174696F6E204D656E7500031027DA
:10282000020024282F28282836280000000000470E
:102830002800000000006C6F6164656420662E2033
:10284000454550524F4D00436F6E66696775726122
:1028500074696F6E0003102702005C2867286028E7
:102860006E2800000000007F280000000000737444
:102870006F72656420696E20454550524F4D00438C
:102880006F6E66696775726174696F6E0094280374
:10289000070400004C6F61642066726F6D2045452F
:1028A00050524F4D00AC28030604000053746F7261
:1028B0006520746F20454550524F4D00C32802FFDC
:1028C000280000457874727564657200D32802068A
:1028D0002B0000466565647261746500E32802326E
:1028E0002B0000416363656C65726174696F6E00F3
:1028F000F72802522A000047656E6572616C00027B
:10290000000010000629752F3E2A2A2A182A072AB5
:10291000F229C329DB29AC2999298529742963293E
:102920004E29392926292D29042F04000050494415
:10293000204D61783A2558440040290426040000BF
:102940004472697665204D61783A25584D005529C5
:1029500004250400004472697665204D696E3A25AD
:10296000586D006A29042404000050494420443A68
:10297000255864007B290423040000504944204961
:102980003A255869008C29042204000044542F5031
:10299000494420503A25587000A029042D04000015
:1029A000436F6E74726F6C3A25586800B329044601
:1029B000040000416476616E6365206C696E3A259F
:1029C000586C00CA29044D040000576169742055F1
:1029D0006E6974733A2558556D6D00E229044C04F4
:1029E0000000576169742054656D702E255854029B
:1029F0004300F929042E040000537461622E5469C7
:102A00006D653A255877000E2A042A0400004163B8
:102A100063656C3A255841001F2A042B0400004DC1
:102A200061782046523A25584600312A042C040089
:102A30000053746172742046523A25586600452A44
:102A4000042904000053746570732F4D4D3A2553CB
:102A500065000200000400592A752F8E2A762A612B
:102A60002A682A02A22A00004D61782E20496E6150
:102A70006374697665007D2A02D42A000053746568
:102A80007070657220496E61637469766500952A7D
:102A9000041004000042617564726174653A256F28
:102AA00063000358040200A92AB42AAD2ABB2A00F5
:102AB00000000000C52A00000000005B735D2030AC
:102AC0003D4F6666004469732E2041667465723A14
:102AD000256970000320040200DB2AE62ADF2AEDC4
:102AE0002A0000000000F72A00000000005B735D70
:102AF00020303D4F6666004469732E204166746540
:102B0000723A2569730002000003000D2B752F2314
:102B10002B132B1A2B0413040000486F6D653A2504
:102B2000665A002A2B04160400004D61783A256687
:102B30007A000200000400392B752F612B512B41C4
:102B40002B482B040E0400004A65726B3A25616A1B
:102B500000582B040D0400004D6F76653A25615A2C
:102B600000682B040A0400005072696E743A2561F3
:102B70007A000200000500792B752FBC2BA92B963B
:102B80002B832B8A2B033504000044727920727545
:102B90006E3A256464009D2B033404000045727274
:102BA0006F7273203A25646500B02B033304000074
:102BB000496E666F2020203A25646900C32B0332DA
:102BC0000400004563686F2020203A25646F00D61A
:102BD0002B02E32B000053442043617264204D65B7
:102BE0006E75000200000600EA2B752F442C312C74
:102BF0001B2C092CF62BFD2B03F403010244656CFE
:102C00006574652066696C6500102C02632C0200F7
:102C100053746F70205072696E7400222C03F70396
:102C20000400436F6E74696E7565205072696E742E
:102C300000382C03F603020450617573652050724E
:102C4000696E74004B2C03F503010253656C6563D8
:102C5000742053442046696C650001000001006146
:102C60002C752F02000003006A2C852C7B2C702C05
:102C7000772C035424020059657300822C03E80367
:102C800000004E6F008C2C010000000053746F7028
:102C9000205072696E74009E2C02AF2C00004164BB
:102CA0006A7573742046616E2073706565640002F6
:102CB00000000700B62C752F2D2D192D042DEF2C9B
:102CC000DA2CC42CCB2C031E040000536574204660
:102CD000616E2031303025252500E12C031D0400D4
:102CE000005365742046616E20373525252500F692
:102CF0002C031C0400005365742046616E2035309F
:102D0000252525000B2D031B040000536574204668
:102D1000616E20323525252500202D031A04080078
:102D20005475726E2046616E204F666600342D0425
:102D30005204000046616E2073706565643A254652
:102D400073252525000200000A004C2D752FAA2DA1
:102D5000912D082EF52DDB2D612FC32D1B2E02008A
:102D6000000A00652D752FAA2D912D082EF52DDB5B
:102D70002D612F792DC32D1B2E802D03B20F000046
:102D8000556E6C6F636B2046756C6C204D656E756F
:102D900000982D0448040000466C6F772020526193
:102DA00074653A256F6625252500B12D041F0400A2
:102DB00000537065656420526174653A256F6D2516
:102DC000252500CA2D034204001044697361626C1A
:102DD0006520537465707065727300E22D033804CA
:102DE000000053687574204F666620414C4C2048A3
:102DF0006561747300FC2D03470400005072656820
:102E000065617420414253000F2E033704000050C7
:102E100072656865617420504C4100222E033604AF
:102E2000000041545820706F776572206F6E2F6FCD
:102E300066660002000003003A2E752F3E2E452ED6
:102E4000043D0400004E4F5A2054656D703A202016
:102E500025453002430002000006005D2E752F93C9
:102E60002E692E612F2B2F7F2E702E04210400003F
:102E7000482E20526164697573203A256F68008678
:102E80002E03AC0F0000536574205A204F726967FF
:102E9000696E009A2E02AB2E000046756C6C2043C2
:102EA000616C6962726174696F6E000200000400F7
:102EB000B22E752FE82ED32EBA2EC12E03B10F00DD
:102EC00000426567696E2043616C69627261746972
:102ED0006F6E00DA2E03B50F0000424544204152C8
:102EE0004520434C45414E00EF2E03B40F00004DEA
:102EF000414B452053555245204E4F5A5A4C452080
:102F000026000200000600092F752F612F4F2F3D6C
:102F10002F2B2F152F1C2F028E2F00004578747237
:102F20002E20706F736974696F6E00322F02EF305C
:102F300000005A20506F736974696F6E00442F024D
:102F4000443100005920506F736974696F6E0056E8
:102F50002F02993100005820506F736974696F6EA9
:102F600000682F03FD030000486F6D6520507269F3
:102F70006E746572007C2F03E80300005072657662
:102F8000696F75732053637265656E20010003F0ED
:102F9000030400952FB22FAB2FA42F9D2FB92F0024
:102FA00000000000C72F0000000000D82F00000024
:102FB0000000E72F0000000000255566206D2070FE
:102FC00072696E7465640020453A2565632F254556
:102FD0006302437E256F43003120636C69636B207D
:102FE0003D2031206D6D00453A257833206D6D0010
:102FF00003FC030400F72F14300D300630FF2F1BA5
:103000003000000000001C3000000000002C3000E8
:10301000000000003C300000000000004D617820FE
:10302000656E6473746F703A25735A004D696E2033
:10303000656E6473746F703A25737A005A3A257816
:1030400032206D6D0003FB0304004C3069306230A8
:103050005B30543070300000000000713000000020
:1030600000008130000000000091300000000000EE
:10307000004D617820656E6473746F703A257359E2
:10308000004D696E20656E6473746F703A257379B4
:1030900000593A257831206D6D0003FA030400A130
:1030A00030BE30B730B030A930C53000000000006D
:1030B000C6300000000000D6300000000000E630FE
:1030C0000000000000004D617820656E6473746F2D
:1030D000703A257358004D696E20656E6473746F85
:1030E000703A25737800583A257830206D6D0003CA
:1030F000EF030400F63013310C310531FE301A3184
:1031000000000000001B3100000000002B31000017
:103110000000003B310000000000004D6178206598
:103120006E6473746F703A25735A004D696E206532
:103130006E6473746F703A25737A005A3A25783248
:10314000206D6D0003EE0304004B31683161315A8C
:103150003153316F31000000000070310000000079
:1031600000803100000000009031000000000000ED
:103170004D617820656E6473746F703A25735900E1
:103180004D696E20656E6473746F703A25737900B3
:10319000593A257831206D6D0003ED030400A0310C
:1031A000BD31B631AF31A831C4310000000000C5D7
:1031B000310000000000D5310000000000E53100C2
:1031C00000000000004D617820656E6473746F70BC
:1031D0003A257358004D696E20656E6473746F7084
:1031E0003A25737800583A257830206D6D0000003C
:1031F000000400F53112320B320432FD3119320075
:10320000000000001F320000000000333200000008
:10321000000037320000000000255566206D005484
:103220006F74616C2046696C616D656E74205573B6
:1032300065640025557400546F74616C2050726988
:103240006E74696E672054696D65000000000400AB
:1032500052326F32683261325A32763200000000E8
:1032600000803200000000008E320000000000A04C
:103270003200000000004861636B65722048320034
:103280005072696E746572204D6F64656C004657AC
:1032900020446174653A20323031373131313300A6
:1032A00046572056657273696F6E3A20302E393258
:1032B0002E32000000000400BA32D732D032C932B8
:1032C000C232DE320000000000E2320000000000E6
:1032D000EB320000000000F4320000000000256F17
:1032E00073005A3A257832206D6D00593A257831AD
:1032F000206D6D00583A257830206D6D000000007B
:103300000400043321331A3313330C332833000001
:103310000000002C330000000000353300000000E6
:10332000004E330000000000256F73005A3A2578E4
:1033300032206D6D0053706565643A256F6D2525EB
:103340002520466C6F773A256F66252525004E4F60
:103350005A3A256563205461726765743A2545635E
:10336000000000000000000000000000FF0000015D
:10337000000000000000000000000000000000004D
:103380000024F403D950C38EB1C2A23D96828B357E
:1033900082127AE372816CCB66A861015DC758EB3B
:1033A000546151204E1E4B5648C14559431A4101A4
:1033B0003F093D2F3B7139CD374036C93465331451
:1033C00032D430A32F802E6B2D632C672B752A8E61
:1033D00029B028DC2710274B268F25D9242B2482BF
:1033E00023E0224322AC211A218D200420801F00DB
:1033F0001F841E0C1E971D261DB81C4E1CE61B822A
:103400001B201BC11A641A0A1AB2195D190A19B9CC
:10341000186A181C18D11788174017FA16B51673B2
:10342000163116F115B31576153A150015C7148F18
:103430001458142214EE13BA13881356132513F6D6
:1034400012C71299126C1240121512EB11C1119889
:1034500011701148112111FB10D610B1108D106997
:1034600010461024100210E10FC00FA00F800F6152
:103470000F420F230F060FE80ECB0EAF0E930E7701
:103480000E5C0E410E270E0D0EF30DDA0DC10DA8C8
:103490000D900D780D600D490D320D1B0D050DEFD2
:1034A0000CD90CC30CAE0C990C850C700C5C0C4840
:1034B0000C350C210C0E0CFB0BE80BD60BC40BB21D
:1034C0000BA00B8E0B7D0B6B0B5A0B4A0B390B2988
:1034D0000B180B080BF80AE90AD90ACA0ABB0AAC8E
:1034E0000A9D0A8E0A800A710A630A550A470A3938
:1034F0000A2C0A1E0A110A040AF709EA09DD09D092
:1035000009C409B709AB099F09920987097B096FAB
:1035100009630958094C09410936092B0920091585
:10352000090A090009F508EB08E008D608CC08C22A
:1035300008B808AE08A4089A08900887087D08749F
:10354000086B08610858084F0846083D0834082CE5
:103550000823081A08120809080108F807F007E804
:1035600007E007D807D007C807C007B807B007A803
:1035700007A1070000420FA1071605D0030D038B1A
:10358000022E02E801B2018601630145012C0117F8
:10359000010401F4005072696E7465722052656115
:1035A0006479005072696E74657220526561647945
:1035B000005072696E7465722052656164790020F2
:1035C0007A3A0020793A0020783A00696E207175C5
:1035D00065756544656C74614D6F766520746F2008
:1035E00063616C63756C61746544656C746153757B
:1035F000625365676D656E74732072657475726E63
:1036000073206572726F722E0043206869742066A1
:103610006C6F6F720043706F7320782073717561E7
:103620007265200043706F73207820737465707327
:10363000200043706F73207920737175617265206B
:103640000043706F7320792073746570732000429B
:103650002068697420666C6F6F720042706F73200F
:103660007820737175617265200042706F732078E5
:10367000207374657073200042706F73207920731B
:103680007175617265200042706F732079207374C8
:103690006570732000412068697420666C6F6F72DA
:1036A0000041706F7320782073717561726520001E
:1036B00041706F73207820737465707320004170BF
:1036C0006F73207920737175617265200041706F8E
:1036D00073207920737465707320006D6F76655266
:1036E000656C617469766544697374616E6365497C
:1036F0006E5374657073202F207175657565446510
:103700006C74614D6F76652072657475726E73208E
:103710006572726F720000000A0B02090C0D0E0830
:10372000070304010000000000000000000000008A
:103730000000000000000000000000000000000089
:103740000000121110000000000000000000000046
:103750000000000000000000000000000102102036
:1037600020080810204010204080020102010804B7
:10377000020101020408102040808040201008044B
:1037800002018004020180402010080402010804A4
:1037900002010102040810204080010204081020E8
:1037A0004080050505050705080808080202020211
:1037B0000A0A0808040404040101010101010101CD
:1037C0000303030303030303040707070C0C0C0C98
:1037D0000C0C0C0C02020202060606060606060681
:1037E0000B0B0B0B0B0B0B0B000020002300260018
:1037F00029002C002F003200000100000301060107
:10380000090100002200250028002B002E003100B5
:10381000340002010000050108010B010000210035
:10382000240027002A002D00300033000101000091
:10383000040107010A01024E414E494E49545949BB
:103840004E46CDCCCC3D0AD7233C17B7D13877CCE8
:103850002B329595E6241FB14F0A0000204100004D
:10386000C84200401C4620BCBE4CCA1B0E5AAEC506
:103870009D74948DD19C95D858FB11241FBECFEF19
:10388000D1E2DEBFCDBF00E00CBF13E0A0E0B2E0AC
:10389000E8ECF9E102E00BBF02C007900D92A633FD
:1038A000B107D9F72EE1A6E3B3E001C01D92A9321A
:1038B000B207E1F718E3CAE7D8E300E006C02297B1
:1038C0000109FE010BBF0F945D08C237D10780E0EC
:1038D0000807A9F70F94C9030D94E20C0C9400009B
:1038E000CF93DF9300D01F92CDB7DEB744E050E016
:1038F000BC01CE0101960F949E0C69817A818B8167
:103900009C810F900F900F900F90DF91CF910895B1
:10391000179A0895169A0895159A089580B182FB12
:10392000882780F9089580B186958170089588E48C
:1039300093E0D6CFCF92DF92EF92FF92CF93DF93B7
:1039400000D01F921F92CDB7DEB76B017C01609350
:1039500018077093190780931A0790931B070E940A
:103960003272C982DA82EB82FC8244E050E065E781
:1039700073E0CE0101960F94C00C23E0B701A601BD
:1039800088EC94E00E94EC9E0E9465CA682F88E64D
:1039900090E06D830F94AE0C6D81681721F088E67E
:1039A00090E00F94C90C0F900F900F900F900F9014
:1039B000DF91CF91FF90EF90DF90CF900895CF935C
:1039C000DF931F92CDB7DEB7BC018DE793E00F9474
:1039D000DC0C0E9465CA682F88E690E069830F942A
:1039E000AE0C6981681739F088E690E00F90DF919E
:1039F000CF910D94C90C0F90DF91CF910895CF9383
:103A0000DF931F92CDB7DEB7BC018FE793E00F9431
:103A1000DC0C0E9465CA682F88E690E069830F94E9
:103A2000AE0C6981681739F088E690E00F90DF915D
:103A3000CF910D94C90C0F90DF91CF910895CF9342
:103A4000DF931F92CDB7DEB7BC0181E893E00F94FE
:103A5000DC0C0E9465CA682F88E690E069830F94A9
:103A6000AE0C6981681739F088E690E00F90DF911D
:103A7000CF910D94C90C0F90DF91CF910895CF9302
:103A8000C82F809147048823D1F0109247040E94E8
:103A9000A25790919002915090939002911109C079
:103AA00080919102833010F40E94495785E0809301
:103AB00090026C2F87E19AE0CF910C94C6C5CF910C
:103AC00008958091CC0B882349F00E94B19580E045
:103AD000D6DF87E19AE00E94C5C5F3CF08954F92E3
:103AE0005F926F927F928F929F92AF92BF92CF928E
:103AF000DF92EF92FF920F931F93CF93DF9300D04B
:103B00001F92CDB7DEB78C018091920790919307F9
:103B1000A0919407B091950789839A83AB83BC8366
:103B2000C0909607D0909707E0909807F09099077B
:103B300080909A0790909B07A0909C07B0909D075B
:103B40009C01AD01BC01CD010F948F0781110FC104
:103B500049805A806B807C80E89477F82FEF3FEFA4
:103B60004FE75FE7C301B2010F948F0781110BC0CC
:103B70002FEF3FEF4FE75FE7C301B2010F943C0423
:103B800018160CF4F4C0A7019601C701B6010F94F2
:103B90008F078111ECC026013701E89477F82FEFE9
:103BA0003FEF4FE75FE7C301B2010F948F07811129
:103BB0000BC02FEF3FEF4FE75FE7C301B2010F9458
:103BC0003C0418160CF4D3C0A5019401C501B4013E
:103BD0000F948F078111CBC024013501E89477F849
:103BE0002FEF3FEF4FE75FE7C301B2010F948F075D
:103BF00081110BC02FEF3FEF4FE75FE7C301B20129
:103C00000F943C0418160CF4B2C020916A0730914E
:103C10006B0740916C0750916D0769817A818B81A8
:103C20009C810F94D8032B013C0120916E073091A9
:103C30006F074091700750917107C701B6010F944B
:103C4000D8036B017C01209172073091730740917A
:103C5000740750917507C501B4010F94D8034B0147
:103C60005C018091F207882329F020E732E441E2E9
:103C70005DE304C020E030E040E85FE3C301B2014F
:103C80000F94E406AB01BC0122E088EF92E20E94AF
:103C9000299F8091F207882329F020E732E441E24E
:103CA0005DE304C020E030E040E85FE3C701B60117
:103CB0000F94E406AB01BC0122E080EF92E20E9487
:103CC000299F8091F207882329F020E732E441E21E
:103CD0005DE304C020E030E040E85FE3C501B401EB
:103CE0000F94E406AB01BC0123E08CEE92E20E944B
:103CF000299F6091AA077091AB078091AC079091C2
:103D0000AD070F940F052091EE073091EF0740911A
:103D1000F0075091F1070F94E4062091F207222357
:103D200029F020E732E441E25DE304C020E030E026
:103D300040E85FE30F94E406AB01BC0124E088EEA9
:103D400092E20F900F900F900F90DF91CF911F9103
:103D50000F91FF90EF90DF90CF90BF90AF909F902A
:103D60008F907F906F905F904F900C94EC9EC80165
:103D70000E940E9D4ACFCF92DF92EF92FF92CF9397
:103D8000DF93EC01893191053CF0C53F81E0D80714
:103D90002CF0C4EFD1E002C0C9E1D0E0BE01882719
:103DA00077FD8095982F0F940F056B017C01609132
:103DB000A2067091A306882777FD8095982F0F940F
:103DC0000F059B01AC01C701B6010F9443049B0191
:103DD000AC016091A4067091A5068091A606909111
:103DE000A7060F94E4066093A4067093A50680933B
:103DF000A6069093A706D093A306C093A206BE0181
:103E00008BEC92E2DF91CF91FF90EF90DF90CF901B
:103E10000C94D29DCF92DF92EF92FF926B017C01C6
:103E200020E030E040E752E40F943C0487FD11C0ED
:103E300020E030E046E153E4C701B6010F9470067C
:103E400018166CF4C12CD12C86E1E82E83E4F82EF0
:103E500006C0C12CD12C90E7E92E92E4F92EC09235
:103E60001807D0921907E0921A07F0921B0722E078
:103E7000B701A60182EB92E2FF90EF90DF90CF9026
:103E80000C94EC9E8F929F92AF92BF92CF92DF9252
:103E9000EF92FF92CF93DF93EC018931910534F0DB
:103EA000893C91052CF0C8ECD0E002C0C9E1D0E01B
:103EB000D093A106C093A006E0913603F09137039A
:103EC000E258FF4FC080D180E280F38020E030E0F4
:103ED000A901C701B6010F943C04AE01662757FD46
:103EE0006095762F18165CF0CB01BA010F940F0580
:103EF0002AE037ED43E25CE30F94E40624C0CB01F3
:103F0000BA010F940F052AE037ED43E25CE30F940A
:103F1000E40620E030E040E850E40F94E4064B0172
:103F20005C01A7019601C701B6010F94E4062BEDD1
:103F30003FE049E450E40F94E4069B01AC01C50165
:103F4000B4010F9443046093960270939702809398
:103F5000980290939902BE018DEB92E2DF91CF918E
:103F6000FF90EF90DF90CF90BF90AF909F908F9099
:103F70000C94D29DCF93DF932091660797FD0DC0DF
:103F8000EC018F3F910519F014F0CFEFD0E02097AE
:103F900021F028602093660705C0277F20936607DD
:103FA000C0E0D0E061118DDD8091251D90E0C81743
:103FB000D90729F0BE0188EA92E20E94D29DC093FF
:103FC000251DDF91CF9108954F925F926F927F925E
:103FD0008F929F92AF92BF92CF92DF92EF92FF9219
:103FE000CF93DF9300D01F92CDB7DEB72FE632E13B
:103FF00043E85AE360918A0670918B0680918C06A3
:1040000090918D060F94E4066B017C0181E890E0AD
:1040100067DC9B01AC01C701B6010F94D803AB016B
:10402000BC0122E086E992E20E94299F84E892E2A4
:104030000E94D49CE0910A02F0910B0220E030E053
:1040400040E751E463857485858596850F947006F5
:1040500018160CF46BC020E030E0A9018DE790E069
:1040600029833A834B835C830F94B60C4B015C012C
:1040700029813A814B815C81820E931EA41EB51E5C
:10408000C501B40120E831E541E050E00F9410088B
:1040900060E87EEA8EEF9FEF0F94AB076B017C0127
:1040A000C80CD91CEA1CFB1CBA01A90187E892E2E2
:1040B0000E94F89DC701B60120E13EE040E050E0DB
:1040C0000F94100849015A01BA01A9018DE792E243
:1040D0000E94F89DA0EFB1EFA50194010F9459083B
:1040E0006C0D7D1D8E1D9F1D2CE330E040E050E0E7
:1040F0000F941008BA01A90185E792E20E94F89D89
:1041000080E792E20F900F900F900F90DF91CF9188
:10411000FF90EF90DF90CF90BF90AF909F908F90E7
:104120007F906F905F904F900C94ED9C0E9473FE77
:10413000C0908E06D0908F06E0909006F090910689
:104140006C197D098E099F0928EE33E040E050E0AC
:104150000F94EE0783CF811102C08EE207C0813039
:1041600011F48DE203C0823019F48CE20C9465FDE9
:104170000895EAE0F1E08081886080838081806139
:10418000808380818062808364E670E08EE20E949A
:1041900065FD64E670E08DE20E9465FD62E870E016
:1041A0008CE20E9465FDE1E2F1E08081887F816020
:1041B0008083089567FD43C08230E9F028F48823A6
:1041C00041F0813061F03BC0833009F1843059F116
:1041D00036C0662311F0A19A69C0A19867C080918A
:1041E0000801662311F0806801C08F778093080171
:1041F00047FF3AC05FC080910801662311F08064D8
:1042000001C08F7B8093080147FF34C055C0809167
:104210000801662311F0886001C0877F8093080140
:1042200047FF32C046C080910501662311F08064CB
:1042300001C08F7B8093050147FF2EC03CC047FD26
:104240003BC08230B9F028F4882341F0813061F01E
:1042500008958330C9F08430F9F00895442311F0B3
:10426000A09A0895A0980895442311F0A29A089561
:10427000A298089580910801442311F0806201C042
:104280008F7D80930801089580910801442311F0E7
:104290008061F7CF8F7EF5CF80910501442311F027
:1042A000806401C08F7B80930501089547FFD6CFBE
:1042B00008950895089508950895643079F028F4D4
:1042C000613041F0623041F00895683051F0603162
:1042D00041F0089540E003C040E004C041E060E0E8
:1042E00002C041E061E066CFCF93DF9381E592E2C7
:1042F0000E94ED9C62B36695617070E088EF92E277
:104300000E94C69D62B3617070E08EE692E20E94E8
:10431000D29DC6E0D1E08881992787FD9095692FCD
:10432000661F6627661F70E089E692E20E94C69DBE
:1043300062B362FB662760F970E08EE692E20E944B
:10434000D29D688166FB662760F970E086E692E29E
:104350000E94C69D688165FB662760F970E08EE665
:1043600092E20E94D29D688163FB662760F970E04B
:1043700082E692E20E94C69D68816295617070E05B
:104380008EE692E20E94D29DC3E0D1E0688166FB96
:10439000662760F970E08EE592E20E94C69D688112
:1043A00066FB662760F970E08EE692E2DF91CF91BE
:1043B0000C94D29DFF920F931F93CF93DF9300D065
:1043C0001F921F92CDB7DEB785E0E8EFF2E0DE0185
:1043D000119601900D928A95E1F7989A9A9A809198
:1043E00007018062809307018091070180618093BB
:1043F0000701809104018064809304018E010F5FA6
:104400001F4FF12CF80161918F018F2D56DFF3942E
:10441000F5E0FF12F7CF0F900F900F900F900F90D5
:10442000DF91CF911F910F91FF9008950C948AD541
:104430000E9475D5209108023091090282179307D6
:1044400024F4909309028093080208956091080271
:10445000709109028091060290910702681779070E
:1044600044F470930702609306028BEF92E20C947F
:10447000D29D0895CF93C82F69E170E080E39DE15C
:104480000E9443FB6C2F80E39DE10E94E4FA60E010
:1044900080E39DE10E9444FB882329F082EA9CE0AE
:1044A000CF910C94ED9CCF910895CF93DF93D82FAB
:1044B000C62F69E170E080E39DE10E9443FB6D2F10
:1044C00080E39DE10E94E4FA6C2F80E39DE10E946D
:1044D000E4FA80E39DE10E9456FB882331F082E8F4
:1044E0009CE0DF91CF910C94ED9CDF91CF910895EA
:1044F000C1DF41E050E069E170E080E39DE10E94AE
:1045000037FB80E39DE10E948DFA892B31F080E337
:104510009DE10E9495FA81E0089583E69CE00E9467
:10452000ED9C80E008958EE39CE00E94ED9C80E38A
:104530009DE10E9422FB8FE0DBDF81E3D9DF80E297
:10454000D7DF6CE980E2B1DF80E2D2DF82E2D0DF48
:1045500060E482E2AADF82E2CBDF85E2C9DF60E0CD
:1045600085E2A3DF85E2C4DF83E2C2DF60E383E2AA
:104570009CDF83E2BDDF84E2BBDF6AE484E295DF97
:1045800084E2B6DF80E3B4DF60E280E38EDF80E3C5
:10459000AFDF81E3ADDF82E3ABDF64E182E385DFA0
:1045A00082E3A6DF83E3A4DF60E083E37EDF83E3CF
:1045B0009FDF84E39DDF60E084E377DF84E398DFBF
:1045C00086E396DF62E386E370DF86E391DF87E3CD
:1045D0008FDF60E087E369DF87E38ADF88E388DFD6
:1045E00060E188E362DF88E383DF89E381DF8AE3D8
:1045F0007FDF62E38AE359DF8AE37ACFCF9381E3F7
:1046000077DFC82F85E374DF811101C0C0E089E343
:104610006FDF811101C0C0E08DE26ADF811101C04E
:10462000C0E08C2FCF9108956DE08AED9AE00E9452
:1046300029D46AE08AED9AE00C9429D4E0913603FB
:10464000F091370342A953A964A975A922E085EE28
:1046500092E20E94299FE0913603F091370346A928
:1046600057A960AD71AD20E08AED92E20E94299FCA
:10467000E0918F02EF3F29F4E0913603F091370388
:10468000E081F0E0EE5DF24E608170E081EE92E25A
:104690000E94C69DC9CF2F923F924F925F926F9218
:1046A0007F928F929F92AF92BF92CF92DF92EF92C2
:1046B000FF920F931F93CF93DF93CDB7DEB7299768
:1046C0000FB6F894DEBF0FBECDBF5C01DC011696BD
:1046D0008D919C9117978C38910509F48BC608F041
:1046E000E7C08235910509F42FC408F08AC08A31E9
:1046F000910509F4D1C208F03FC08531910509F454
:1047000049C278F48231910509F423C284319105BC
:1047100009F424C2419711F00C9474331798169839
:10472000D0C58731910509F46DC208F44FC28831B4
:10473000910509F495C2499711F00C94743360E027
:1047400083EC98E029960FB6F894DEBF0FBECDBF7C
:10475000DF91CF911F910F91FF90EF90DF90CF905D
:10476000BF90AF909F908F907F906F905F904F9091
:104770003F902F900C94A6988E31910509F4E9C2D0
:1047800018F58C31910509F4BCC210F00C94AC33CF
:1047900083EC98E029960FB6F894DEBF0FBECDBF2C
:1047A000DF91CF911F910F91FF90EF90DF90CF900D
:1047B000BF90AF909F908F907F906F905F904F9041
:1047C0003F902F900C94ED9B8A32910509F41BC306
:1047D00028F4809709F4EAC20C947433803591056B
:1047E00009F49DC38135910511F00C94743369D996
:1047F0009B9A809168078F7B80936807A39A0C949B
:10480000AC338B36910511F40C94A82C38F58C350B
:10481000910509F4A4C460F48435910509F49DC39D
:1048200008F496C38535910509F475C40C94743366
:104830008836910509F448C530F48336910509F4AA
:10484000F2C40C9474338936910509F427C68A366C
:10485000910511F40C94972C0C94743383379105C3
:1048600011F40C94F82C80F48F36910511F40C940B
:10487000C92C8237910511F40C94162D8D369105B3
:1048800011F00C9474332CC68537910511F40C94F7
:10489000192D10F40C94512C8737910511F40C94B8
:1048A000442D8837910511F40C948B2D0C9474339E
:1048B0008530B1E09B0711F40C94953008F0B0C03E
:1048C0008F3C910511F40C942F2F08F041C08A3CC5
:1048D000910511F40C94622E70F4883C910511F44A
:1048E0000C94B12D10F00C94042E8E3B910509F41C
:1048F000CBC70C9474338C3C910511F40C94B92EF5
:1049000010F40C94A72E8D3C910511F40C94152FE6
:104910008E3C910511F00C947433C50129960FB6A5
:10492000F894DEBF0FBECDBFDF91CF911F910F91E5
:10493000FF90EF90DF90CF90BF90AF909F908F90BF
:104940007F906F905F904F903F902F900C94B8D0D5
:104950008F3D910511F40C94EA2F88F48C3D91055C
:1049600011F40C94972F8D3D910511F40C94BF2FE9
:10497000813D910511F00C9474330C94772F893E8E
:10498000910511F40C94FF2F40F5883E910511F02C
:104990000C94743360912A1D70912B1D8AE092E271
:1049A0000E94C69D4091261D5091271D6091281D93
:1049B0007091291D22E081E092E20E94EC9E10920B
:1049C0002B1D10922A1D1092261D1092271D109249
:1049D000281D1092291D0C94AC338B3F910511F4C6
:1049E0000C9438308430914011F00C947433299633
:1049F0000FB6F894DEBF0FBECDBFDF91CF911F91F0
:104A00000F91FF90EF90DF90CF90BF90AF909F906D
:104A10008F907F906F905F904F903F902F9083CDBD
:104A20008E3521E0920711F40C94EC31C0F58E32F2
:104A300041E0940711F40C94383198F48931A1E0E5
:104A40009A0711F40C94ED308C32B1E09B0711F40D
:104A50000C94FD308630914011F00C9474330C941A
:104A6000B7308034F1E09F0711F40C94AA3138F488
:104A70008F32914011F40C9477310C94743381345B
:104A800041E0940711F40C94AE318234914011F05E
:104A90000C94743380E00E9466890C94C33182398F
:104AA000A1E09A0711F40C94D73298F58836E1E02A
:104AB0009E0711F40C94A33238F48336914011F41C
:104AC0000C945D320C947433803931E0930711F407
:104AD0000C94BD328139914011F00C9474332996B5
:104AE0000FB6F894DEBF0FBECDBFDF91CF911F91FF
:104AF0000F91FF90EF90DF90CF90BF90AF909F907D
:104B00008F907F906F905F904F903F902F900C947C
:104B1000DE83853F51E0950711F40C94073360F470
:104B2000843F914011F00C94743380E00E947CCA61
:104B300089E89DE10C941233863FE1E09E0711F471
:104B40000C942C338C38934011F40C9446330C9411
:104B500074330E94881C0E948A1C8CC283EC98E0EB
:104B600029960FB6F894DEBF0FBECDBFDF91CF916F
:104B70001F910F91FF90EF90DF90CF90BF90AF907B
:104B80009F908F907F906F905F904F903F902F906D
:104B90000C94369B83EC98E029960FB6F894DEBF10
:104BA0000FBECDBFDF91CF911F910F91FF90EF907E
:104BB000DF90CF90BF90AF909F908F907F906F903D
:104BC0005F904F903F902F900C942A9883EC98E040
:104BD00029960FB6F894DEBF0FBECDBFDF91CF91FF
:104BE0001F910F91FF90EF90DF90CF90BF90AF900B
:104BF0009F908F907F906F905F904F903F902F90FD
:104C00000C942F98D5018D919C9197FD02C00C9426
:104C1000AC3360E083EC98E00E948064F501EE5ACA
:104C2000FF4F6081718140E083EC98E029960FB6D8
:104C3000F894DEBF0FBECDBFDF91CF911F910F91D2
:104C4000FF90EF90DF90CF90BF90AF909F908F90AC
:104C50007F906F905F904F903F902F900C94679B48
:104C600083EC98E029960FB6F894DEBF0FBECDBF57
:104C7000DF91CF911F910F91FF90EF90DF90CF9038
:104C8000BF90AF909F908F907F906F905F904F906C
:104C90003F902F900C949598F5018081918192FD21
:104CA00002C00C94AC33468D578D60A171A18091E8
:104CB0002D09882311F40C94AC33409324095093AC
:104CC0002509609326097093270983E099E02996C6
:104CD0000FB6F894DEBF0FBECDBFDF91CF911F910D
:104CE0000F91FF90EF90DF90CF90BF90AF909F908B
:104CF0008F907F906F905F904F903F902F900C948B
:104D0000C662D5018D919C9197FD02C00C94AC3385
:104D1000F501EE5AFF4F6081718183EC98E029968E
:104D20000FB6F894DEBF0FBECDBFDF91CF911F91BC
:104D30000F91FF90EF90DF90CF90BF90AF909F903A
:104D40008F907F906F905F904F903F902F900C943A
:104D50000E9CF5018081918197FD02C00C94AC33CB
:104D600060E083EC98E00E948064F501EE5AFF4F0A
:104D70006081718183EC98E029960FB6F894DEBFCC
:104D80000FBECDBFDF91CF911F910F91FF90EF909C
:104D9000DF90CF90BF90AF909F908F907F906F905B
:104DA0005F904F903F902F900C94709CD5018D9107
:104DB0009C9197FD02C00C94AC3360E083EC98E0CA
:104DC0000E948064F501EE5AFF4F6081718183EC8F
:104DD00098E029960FB6F894DEBF0FBECDBFDF91E5
:104DE000CF911F910F91FF90EF90DF90CF90BF90E8
:104DF000AF909F908F907F906F905F904F903F907B
:104E00002F900C949E9CF5012081318133FD02C0CE
:104E10000C94AC3312A1E12EF3A0E1ECFCE0449140
:104E200050E04E155F0509F45EC032964DE0E53363
:104E3000F407A9F7F7FC57C032FF2CC0D5015E96E6
:104E40004D915D916D917C9191974F3F5105610519
:104E5000710509F0E0F461E0812F0E9487FFF50100
:104E6000668D812F0E94C0FFD5015E966D917C9169
:104E70005F97812F0E9465FDB70184E492E20E9452
:104E8000C69DF501668D778D8FE392E212C08FE5A6
:104E900094E02BC062E0812F0E9487FFB7018FE36F
:104EA00092E20E94C69D812F0E94F5FFBC018AE319
:104EB00092E229960FB6F894DEBF0FBECDBFDF9108
:104EC000CF911F910F91FF90EF90DF90CF90BF9007
:104ED000AF909F908F907F906F905F904F903F909A
:104EE0002F900C94D29D89E294E029960FB6F89405
:104EF000DEBF0FBECDBFDF91CF911F910F91FF900D
:104F0000EF90DF90CF90BF90AF909F908F907F9069
:104F10006F905F904F903F902F900C940E9D0E9449
:104F2000611D0E9473FE60932C1D70932D1D809354
:104F30002E1D90932F1D9B9A80916807806480930B
:104F40006807A3980C94AC331092AE070C94AC3362
:104F500081E08093AE070C94AC33D5018D919C9188
:104F6000119792FF14C05E962D913D914D915C91E9
:104F70009197A8EEB3E00F944D086093EF02709301
:104F8000F0028093F1029093F2020C94AC3393FF01
:104F9000A5C0F50182A193A1A4A1B5A1823091057C
:104FA000A105B10509F466C02CF50097A105B1056E
:104FB00009F446C00197A105B10511F00C94AC337A
:104FC00029960FB6F894DEBF0FBECDBFDF91CF910B
:104FD0001F910F91FF90EF90DF90CF90BF90AF9017
:104FE0009F908F907F906F905F904F903F902F9009
:104FF0000C948A1C83309105A105B10509F454C0B5
:105000000497A105B10511F00C94AC3329960FB6A5
:10501000F894DEBF0FBECDBFDF91CF911F910F91EE
:10502000FF90EF90DF90CF90BF90AF909F908F90C8
:105030007F906F905F904F903F902F900C94D24F45
:1050400029960FB6F894DEBF0FBECDBFDF91CF918A
:105050001F910F91FF90EF90DF90CF90BF90AF9096
:105060009F908F907F906F905F904F903F902F9088
:105070000C94881C29960FB6F894DEBF0FBECDBFE6
:10508000DF91CF911F910F91FF90EF90DF90CF9024
:10509000BF90AF909F908F907F906F905F904F9058
:1050A0003F902F900C948C1C29960FB6F894DEBF7D
:1050B0000FBECDBFDF91CF911F910F91FF90EF9069
:1050C000DF90CF90BF90AF909F908F907F906F9028
:1050D0005F904F903F902F900C94C44F0E94611DA1
:1050E00081E029960FB6F894DEBF0FBECDBFDF91E9
:1050F000CF911F910F91FF90EF90DF90CF90BF90D5
:10510000AF909F908F907F906F905F904F903F9067
:105110002F900C94CA71D5018D919C91119792FF9B
:1051200014C05E962D913D914D915C919197A8EEA2
:10513000B3E00F944D086093F3027093F4028093F0
:10514000F5029093F6020C94AC331092F302109295
:10515000F4021092F5021092F6020C94AC33F501B1
:10516000808183FF0CC082859385A485B58580935B
:10517000D8029093D902A093DA02B093DB02D50152
:105180008C9184FF0EC01E968D919D910D90BC91C7
:10519000A02D8093DC029093DD02A093DE02B093F9
:1051A000DF02F501808185FF0CC082899389A48983
:1051B000B5898093E0029093E102A093E202B0935C
:1051C000E3020E943272D5018C9186FD02C00C94DC
:1051D000AC33209136033091370356968D919D91D3
:1051E0000D90BC91A02DF90181879287A387B48788
:1051F000808129960FB6F894DEBF0FBECDBFDF9138
:10520000CF911F910F91FF90EF90DF90CF90BF90C3
:10521000AF909F908F907F906F905F904F903F9056
:105220002F900C94044ED501ED91FC911197F2FF53
:105230000DC05E962D913D914D915C919197A8EE98
:10524000B3E00F944D086B017C0106C040E1C42E11
:1052500047E2D42EE12CF12CE3FD0E94881CF501DD
:10526000808184FD0E948A1CD5018C9185FD0E945D
:105270008C1C0E9473FE2B013C014C0C5D1C6E1CAF
:105280007F1C0E9473FEA3019201261B370B480B63
:10529000590BDA01C901803A9648A140B10518F4CA
:1052A0000E942877EECFD5018C9183FD1798F501E8
:1052B000808184FD1698D5018C9185FD02C00C94E7
:1052C000AC3315980C94AC330E947A5781110C942E
:1052D000AC330E9473FE60932C1D70932D1D809340
:1052E0002E1D90932F1D80919B0283FF02C00C9472
:1052F000AC33F5018081918193FF02C00C94973308
:1053000092FF0AC0868D978DA0A1B1A1892B8A2B0F
:105310008B2B11F40C949733D5018D919C9111979F
:1053200092FD02C00C94AC339C012227317091FF96
:1053300023C0232B89F011E020E030E0A9015A9628
:105340006D917D918D919C915D970F9470061816CB
:105350000CF010E0212F01C020E085010C5A1F4FF6
:10536000F501668D778D80A191A129870F940F0596
:105370002985D8014C9124C0232B81F011E020E035
:1053800030E0A901F501628D738D848D958D0F94A8
:10539000700618160CF010E0212F01C020E00091DB
:1053A000360310913703D5015E966D917D918D91F5
:1053B0009C91919729870F940F052985F8014081C9
:1053C00029960FB6F894DEBF0FBECDBFDF91CF9107
:1053D0001F910F91FF90EF90DF90CF90BF90AF9013
:1053E0009F908F907F906F905F904F903F902F9005
:1053F0000C9438530E947A5781110C94AC330E945C
:1054000073FE60932C1D70932D1D80932E1D909321
:105410002F1D80919B0283FF02C00C94AC33D501F9
:105420008D919C91119792FD02C00C94AC3390FF2A
:1054300011C011E020E030E0A9015A966D917D91F4
:105440008D919C915D970F94700618160CF010E0EA
:10545000412F01C040E0F501668D778D80A191A1BB
:1054600049870F940F05498529960FB6F894DEBF3A
:105470000FBECDBFDF91CF911F910F91FF90EF90A5
:10548000DF90CF90BF90AF909F908F907F906F9064
:105490005F904F903F902F900C94BE4FD5018D910F
:1054A0009C9133E0969587953A95E1F7817029961E
:1054B0000FB6F894DEBF0FBECDBFDF91CF911F9125
:1054C0000F91FF90EF90DF90CF90BF90AF909F90A3
:1054D0008F907F906F905F904F903F902F90AEC8CD
:1054E0000E947A5781110C94AC330E9473FE609332
:1054F0002C1D70932D1D80932E1D90932F1D809138
:105500009B0283FF02C00C94AC3340E068E174E07E
:1055100087E19AE00E94CBA887E19AE00E941FAC45
:105520000E94611D2090360330903703F501808181
:10553000918191FF09C0EC5AFF4F2081211104C0D5
:105540002CE0222E22E0322E92FF1EC090FF0FC0D0
:1055500011E020E030E0A901D5015A966D917D91CE
:105560008D919C915D970F94700618160CF010E0C9
:10557000F501668D778D80A191A10F940F05212FE4
:10558000D1014C910E943853F10126A937A940ADB1
:1055900051AD62A973A984A995A90F94D7032B01D2
:1055A0003C0120E030E0A9010F947006181664F465
:1055B00020E030E040EA50E4C301B2010F943C0423
:1055C00087FF0EC00C94AC3320E030E040EA50EC92
:1055D000C301B2010F947006181614F40C94AC3386
:1055E00099249394D101D0962D913C91D1979E9678
:1055F0008D919C919F97821793070CF0912C0E949C
:1056000073FE6D837E838F83988710E0412C512C2D
:1056100032010E9473FE69837A838B839C8360933B
:105620002C1D70932D1D80932E1D90932F1DDC013A
:10563000CB012D813E814F815885821B930BA40B9A
:10564000B50B893E9340A105B10558F080E00E945A
:105650001E2389819A81AB81BC818D839E83AF8318
:10566000B88781E00E943F1D8091360390913703F7
:105670002816390609F064C0D1019396ED90FC908C
:1056800094971E141F040CF05BC0111158C0992090
:1056900009F477C091966D917C919297882777FD58
:1056A0008095982F0F940F059B01AC01F10162A921
:1056B00073A984A995A90F947006181614F00C9478
:1056C000A433662777276E197F09882777FD809591
:1056D000982F0F940F052091E4023091E50240913C
:1056E000E6025091E7020F94E4060F94DC041F9247
:1056F0001F92D10152962C9152972F9351962C9133
:1057000051972F9350962C9150972F931F962C9131
:105710002F935B016C01E12CF12C870120E030E03C
:10572000A90160E070E0CB010E9494F20F900F900D
:105730000F900F900F900F9011E00C94A43311E094
:10574000411451046104710409F050C09920F1F032
:1057500020E030E040E85FE3F10166A977A980AD81
:1057600091AD0F94D7039B01AC01D101D2966D91FD
:105770007D918D919C91D5970F94700687FF1FC0E6
:1057800045CF411451046104710481F520E030E0FB
:1057900040E85FE3F10166A977A980AD91AD0F9470
:1057A000D8039B01AC01D101D2966D917D918D9171
:1057B0009C91D5970F943C0418160CF427CFF10157
:1057C000A78DB0A128EE33E00F9447082B013C01D0
:1057D00029813A814B815C81420E531E641E751EE5
:1057E000411451046104710409F413CFD301C201BF
:1057F00029813A814B815C81821B930BA40BB50BF1
:1058000081159449A543B74708F403CF1123E1F16B
:10581000809136039091370328163906A9F5D101F6
:1058200093966D917C919497882777FD8095982F1A
:105830000F940F052091E4023091E5024091E602B9
:105840005091E7020F94E4060F94DC041F921F921C
:10585000F10122892F9321892F9320892F93278566
:105860002F935B016C01E12CF12C870120E030E0EB
:10587000A90160E070E0CB010E9494F20F900F90BC
:105880000F900F900F900F901092800A0E9473FE5D
:1058900060932C1D70932D1D80932E1D90932F1DB2
:1058A0005BC780919B0283FD57C70E9473FE4B012B
:1058B0005C010E9473FE681979098A099B09693E97
:1058C00073408105910538F080E00E941E230E94FC
:1058D00073FE4B015C0181E00E943F1D00910A02B2
:1058E00010910B02D8011B964D905D906D907C90AD
:1058F0001E9720E030E040EF51E4C301B2010F9465
:10590000700618160CF028C7F801278130854185EC
:105910005285C301B2010F94D7039F7720E030E096
:1059200040E85FE30F94700618161CF215C7D50106
:105930008D919C91119793FB662760F992FF05C0AA
:105940005E968D919C915F970AC08FEF90E007C0A3
:10595000F501618163FB662760F980E090E029969C
:105960000FB6F894DEBF0FBECDBFDF91CF911F9170
:105970000F91FF90EF90DF90CF90BF90AF909F90EE
:105980008F907F906F905F904F903F902F900C94EE
:10599000BA1FD5018D919C91119792FF04C05E961C
:1059A0002C9120939B0293FF12C0F50182A193A139
:1059B000A4A1B5A120919B02181619061A061B0670
:1059C00014F4822B02C08150822380939B02809129
:1059D0009B0283FFC1C620E040E060E070E0CB01A5
:1059E0000E94385320E040E060E070E0CB01E8CC5A
:1059F00081E194E20E94ED9C29960FB6F894DEBFF7
:105A00000FBECDBFDF91CF911F910F91FF90EF900F
:105A1000DF90CF90BF90AF909F908F907F906F90CE
:105A20005F904F903F902F900C94E41F82E194E0A0
:105A300062C3D5018D919C9197FF8EC6F501EE5AF8
:105A4000FF4F6081718140E087E19AE00E9444A9A4
:105A500087E19AE029960FB6F894DEBF0FBECDBF5E
:105A6000DF91CF911F910F91FF90EF90DF90CF903A
:105A7000BF90AF909F908F907F906F905F904F906E
:105A80003F902F900C941FAC0E94611D8DE292E21A
:105A90000E94D49C379903C084E392E202C087E35A
:105AA00092E20E94D49C86E292E20E94D49C0E94E0
:105AB0008E1C882319F087E392E202C084E392E20D
:105AC0000E94D49C8FE192E20E94D49C0E94931C7D
:105AD000882319F087E392E202C084E392E20E94F5
:105AE000D49C29960FB6F894DEBF0FBECDBFDF91D0
:105AF000CF911F910F91FF90EF90DF90CF90BF90CB
:105B0000AF909F908F907F906F905F904F903F905D
:105B10002F900C941423F5018081918188279C702B
:105B200081159C4009F018C6F50162A1868D299661
:105B30000FB6F894DEBF0FBECDBFDF91CF911F919E
:105B40000F91FF90EF90DF90CF90BF90AF909F901C
:105B50008F907F906F905F904F903F902F900C941C
:105B6000FF9FE0913603F09137032081D5018D919D
:105B70009C9191FF06C0F501EC5AFF4F808188236C
:105B800011F0822F01C080E0F501928192FF05C0E3
:105B900046A457A460A871A803C0412C512C32011F
:105BA00093FF07C0D501D2964D905D906D907C908B
:105BB000D597082F10E0B3E88B9FF0011124E6572A
:105BC000FD4F4082518262827382821306C08091AF
:105BD000A0069091A1060E94421F20E030E0A9019A
:105BE000C301B2010F943C04B801811103C086EED9
:105BF00093E05FC98FEB93E00E94C69D22E0B30162
:105C0000A2018AEB93E059C1F501808183FF0CC0AA
:105C100082859385A485B5858093AC029093AD026F
:105C2000A093AE02B093AF02D5018C9184FF0EC059
:105C30001E968D919D910D90BC91A02D8093B002E8
:105C40009093B102A093B202B093B302F5018081A8
:105C500085FF0CC082899389A489B5898093B40299
:105C60009093B502A093B602B093B702D5018C9180
:105C700086FF0EC056968D919D910D90BC91A02DE2
:105C80008093B8029093B902A093BA02B093BB027A
:105C900029960FB6F894DEBF0FBECDBFDF91CF912E
:105CA0001F910F91FF90EF90DF90CF90BF90AF903A
:105CB0009F908F907F906F905F904F903F902F902C
:105CC0000C943272F501808183FF0CC0828593852C
:105CD000A485B58580939C0290939D02A0939E021B
:105CE000B0939F02D5018C9184FF0EC01E968D91BA
:105CF0009D910D90BC91A02D8093A0029093A10244
:105D0000A093A202B093A302F501808185FF0CC08D
:105D100082899389A489B5898093A4029093A5026E
:105D2000A093A602B093A702D5018C9186FFB0CFB5
:105D300056968D919D910D90BC91A02D8093A802B7
:105D40009093A902A093AA02B093AB02A1CFF50150
:105D50008081918192FF00C5868D978DA0A1B1A110
:105D6000181619061A061B060CF4F6C48093910245
:105D7000F3C4E0913603F0913703BB96D5012D9122
:105D80003C91119732FF0DC05E968D919D910D90C3
:105D9000BC91A02D892B8A2B8B2B09F0DDC4E7E366
:105DA000F2E023FF0BC0D5011A964D915D916D91E4
:105DB0007C911D97428F538F648F758FD5018C9185
:105DC00084FF0AC01E964D915D916D917C91519713
:105DD000468F578F60A371A3D5018C9185FF0AC0B0
:105DE00052964D915D916D917C91559742A353A32D
:105DF00064A375A3CF0129960FB6F894DEBF0FBE3A
:105E0000CDBFDF91CF911F910F91FF90EF90DF9069
:105E1000CF90BF90AF909F908F907F906F905F904A
:105E20004F903F902F900C94BE4D29960FB6F8944A
:105E3000DEBF0FBECDBFDF91CF911F910F91FF90BD
:105E4000EF90DF90CF90BF90AF909F908F907F901A
:105E50006F905F904F903F902F900C9465D2F5011A
:105E6000208123FF0CC082859385A485B58580930E
:105E70009C0690939D06A0939E06B0939F0626FFD6
:105E800011C02091360330913703F5018689978937
:105E9000A08DB18DF901878B908FA18FB28F8081FA
:105EA0000E94044E40919C0650919D0660919E0672
:105EB00070919F0622E089E192E229960FB6F8944C
:105EC000DEBF0FBECDBFDF91CF911F910F91FF902D
:105ED000EF90DF90CF90BF90AF909F908F907F908A
:105EE0006F905F904F903F902F900C94EC9ED50157
:105EF0008D919C91119792FF2FC461E05E968D91D8
:105F00009D910D90BC91A02D20916707892B8A2B24
:105F10008B2B21F460E0822F8D7F02C0822F826064
:105F20008093670770E081E293E00C945927F501B4
:105F30008081918192FF05C0868D978DA0A1B1A12E
:105F400004C084E690E0A0E0B0E029960FB6F89493
:105F5000DEBF0FBECDBFDF91CF911F910F91FF909C
:105F6000EF90DF90CF90BF90AF909F908F907F90F9
:105F70006F905F904F903F902F900C94BB1ED50177
:105F80008D919C91119792FF07C05E968D919D9186
:105F90000D90BC91A02D04C084E690E0A0E0B0E09C
:105FA00029960FB6F894DEBF0FBECDBFDF91CF911B
:105FB0001F910F91FF90EF90DF90CF90BF90AF9027
:105FC0009F908F907F906F905F904F903F902F9019
:105FD0000C94421FF5018081918192FFBDC34FB7A0
:105FE000F8948091F3079091F407268D378D820FF6
:105FF000931F9093F4078093F3074FBFADC3F50150
:106000008081209136033091370384FF09C0868553
:106010009785A089B189F90185A396A3A7A3B0A705
:10602000D90195964D915D916D917C91989722E063
:1060300088EE91E20E94299F0E94142329960FB6B0
:10604000F894DEBF0FBECDBFDF91CF911F910F91AE
:10605000FF90EF90DF90CF90BF90AF909F908F9088
:106060007F906F905F904F903F902F900C9418729C
:1060700020919A0730919B0740919C0750919D0772
:106080006091AC067091AD068091AE069091AF061E
:106090000F94D7036093AC067093AD068093AE0661
:1060A0009093AF061092A6071092A7071092A80728
:1060B0001092A9070E94327262EB77E08EE997E0B6
:1060C0000E9480E780E00E943B7E4091AC065091A8
:1060D000AD066091AE067091AF0622E083E99EE1C5
:1060E0000E94EC9E80E00E947CCA82EF91E20E94B6
:1060F000ED9C84EB93E029960FB6F894DEBF0FBEBB
:10610000CDBFDF91CF911F910F91FF90EF90DF9066
:10611000CF90BF90AF909F908F907F906F905F9047
:106120004F903F902F900C946F1D80E10E94F5FFDF
:10613000BC018AEA93E00E94D29D29960FB6F8949A
:10614000DEBF0FBECDBFDF91CF911F910F91FF90AA
:10615000EF90DF90CF90BF90AF909F908F907F9007
:106160006F905F904F903F902F900C94FE2282E3AF
:106170000E947822F5018081918192FFEDC2468DC7
:10618000578D60A171A184E993E00E94109ED50112
:106190005E966C9182E30E945522F501668D8AE33A
:1061A0000E94552282E329960FB6F894DEBF0FBEF7
:1061B000CDBFDF91CF911F910F91FF90EF90DF90B6
:1061C000CF90BF90AF909F908F907F906F905F9097
:1061D0004F903F902F900C94782289E593E00E9495
:1061E000049D80E00E94CA7168EC70E080E090E05D
:1061F0000E94A2FE8FB7F894FFCFD5018D919C919C
:10620000119792FF05C05E966D917C915F9702C0D9
:1062100061E070E093FF04C0F50102A113A102C088
:1062200008EE13E020E030E0A90184E50F9445007A
:10623000B80180E090E00E94A2FE84E529960FB6A6
:10624000F894DEBF0FBECDBFDF91CF911F910F91AC
:10625000FF90EF90DF90CF90BF90AF909F908F9086
:106260007F906F905F904F903F902F900D945603CA
:10627000D5018D919C91119792FF0EC021E05E9601
:106280008D919D910D90BC91A02D892B8A2B8B2BEC
:1062900009F420E0822F01C081E0909168078823F3
:1062A00011F0906801C09F7790936807882319F0D8
:1062B0008AE093E002C080EF92E029960FB6F8944E
:1062C000DEBF0FBECDBFDF91CF911F910F91FF9029
:1062D000EF90DF90CF90BF90AF909F908F907F9086
:1062E0006F905F904F903F902F900C94ED9CF50134
:1062F0000081118112FF03C0668D778D02C066E9AF
:1063000070E013FF0CC0D5019296ED90FC9093972E
:106310001E141F0434F4EE24E394F12C02C0E12C8B
:10632000F12CA3E016950795AA95E1F7017088274F
:1063300077FD8095982F0F940F05AB01BC01F701F5
:10634000EE0FFF1FE65FFD4F2E2D808191810E9491
:10635000145402C281E00E94128515C080E00E94A0
:106360001285D5018D919C91119792FFF5C15E9692
:106370008D919D910D90BC91A02D0097A105B10527
:1063800009F0D9C1E9C1F5018081918192FFE4C191
:10639000868D978DA0A1B1A1892B8A2B8B2B09F417
:1063A000DBC180E029960FB6F894DEBF0FBECDBFEB
:1063B000DF91CF911F910F91FF90EF90DF90CF90E1
:1063C000BF90AF909F908F907F906F905F904F9015
:1063D0003F902F900C947CCA87E493E00E94ED9C40
:1063E000D5018D919C9192FD0FC0F501808183FFB5
:1063F00016C0F50162857385848595850F94E10447
:1064000080E00E945D210BC010E0D5015E966C918A
:10641000812F0E945D211F5F1530B9F7E6CFD501AE
:106420008C9184FF0BC01E966D917D918D919C91F6
:1064300051970F94E10481E00E945D21F501808174
:1064400085FF09C062897389848995890F94E10465
:1064500082E00E945D21D5018C9186FF0BC056968B
:106460006D917D918D919C9159970F94E10483E0FA
:106470000E945D21F5018081918193FF04C062A19A
:1064800084E00E945D2129960FB6F894DEBF0FBE0E
:10649000CDBFDF91CF911F910F91FF90EF90DF90D3
:1064A000CF90BF90AF909F908F907F906F905F90B4
:1064B0004F903F902F900C947421D5018D919C9119
:1064C000119792FF26C081E05E964D915D916D918E
:1064D0007C919197452B462B472B09F480E0299618
:1064E0000FB6F894DEBF0FBECDBFDF91CF911F91E5
:1064F0000F91FF90EF90DF90CF90BF90AF909F9063
:106500008F907F906F905F904F903F902F900C9462
:106510008F8D29960FB6F894DEBF0FBECDBFDF91E9
:10652000CF911F910F91FF90EF90DF90CF90BF9090
:10653000AF909F908F907F906F905F904F903F9023
:106540002F900C94908D29960FB6F894DEBF0FBE55
:10655000CDBFDF91CF911F910F91FF90EF90DF9012
:10656000CF90BF90AF909F908F907F906F905F90F3
:106570004F903F902F900C949E8D29960FB6F894D3
:10658000DEBF0FBECDBFDF91CF911F910F91FF9066
:10659000EF90DF90CF90BF90AF909F908F907F90C3
:1065A0006F905F904F903F902F900C94611DF5017C
:1065B0008081918190FF05C0E28CF38C048D158D54
:1065C00008C0E090A406F090A5060091A6061091E0
:1065D000A7069C0146E0369527954A95E1F721707C
:1065E000AC0165E0569547956A95E1F74170BC01AD
:1065F000E4E076956795EA95E1F76170F3E09695AA
:106600008795FA95E1F781700E943F84A5C00E94AA
:10661000C9CCE0913603F091370380810E94044E8B
:1066200087E69DE129960FB6F894DEBF0FBECDBF79
:10663000DF91CF911F910F91FF90EF90DF90CF905E
:10664000BF90AF909F908F907F906F905F904F9092
:106650003F902F900C94049D29960FB6F894DEBFBE
:106660000FBECDBFDF91CF911F910F91FF90EF90A3
:10667000DF90CF90BF90AF909F908F907F906F9062
:106680005F904F903F902F900C94ADC88EE293E0B6
:106690000E94ED9CD5018D919C9188279C7081155D
:1066A0009C4009F059C0D5015E966D917C915F9731
:1066B00092968C9129960FB6F894DEBF0FBECDBF8F
:1066C000DF91CF911F910F91FF90EF90DF90CF90CE
:1066D000BF90AF909F908F907F906F905F904F9002
:1066E0003F902F900C94AB2080919B0282FF34C08E
:1066F00085E093E20E94D49CC50129960FB6F894D8
:10670000DEBF0FBECDBFDF91CF911F910F91FF90E4
:10671000EF90DF90CF90BF90AF909F908F907F9041
:106720006F905F904F903F902F900C94BE940E947A
:10673000611D0C948C290397A105B10509F031CE98
:1067400080E00E9466892DCE4114510461047104D9
:1067500011F40C94A82B4AC829960FB6F894DEBF02
:106760000FBECDBFDF91CF911F910F91FF90EF90A2
:10677000DF90CF90BF90AF909F908F907F906F9061
:106780005F904F903F902F9008952F923F924F929D
:106790005F926F927F928F929F92AF92BF92CF92B1
:1067A000DF92EF92FF920F931F93CF93DF93CDB7BA
:1067B000DEB7EC970FB6F894DEBF0FBECDBF1C015D
:1067C000DC0118968D919C9119978032910509F4FE
:1067D00069C358F58531910509F45EC198F4843098
:1067E000910509F41BC128F4029708F4EBC00C943E
:1067F0009E42449711F00C949E4281E08093F207F0
:106800000C94A9428D31910509F4AEC128F44C973E
:1068100009F446C10C949E428E31910509F41DC2C3
:106820004F9709F42CC30C949E428C35910511F4BA
:106830000C94C83E40F58534910509F492C7B8F42C
:106840008434910511F00C949E428091A40690919D
:10685000A506A091A606B091A7068D879E87AF8753
:10686000B88B44E1442E512C612C712CA5C58A357E
:10687000910511F40C94AD3E8B35910511F40C94F7
:10688000B93E0C949E428438910511F40C945F41FA
:1068900008F05DC08436910511F40C94AA3F83384A
:1068A000910511F00C949E426091920770919307AC
:1068B00080919407909195072091960730919707C2
:1068C0004091980750919907E0909A07F0909B07A4
:1068D00000919C0710919D074090A4065090A5063A
:1068E0006090A6067090A7061092980610929906DE
:1068F00010929A0610929B0610929406109295069A
:106900001092960610929706E091BF02EF93E091E5
:10691000BE02EF93E091BD02EF93E091BC02EF93D2
:10692000E0EFAE2EE3E2BE2EE4E7CE2EE9E4DE2E6B
:106930000E947E7B4092A4065092A5066092A60615
:106940007092A70680E00E943B7E0C945A418538E5
:10695000910511F40C94EE418638910511F00C94D8
:106960009E424091B2075091B3076091B407709175
:10697000B50780EF94E00E94F89D4091B6075091D2
:10698000B7076091B8077091B9078EE692E20E944E
:10699000F89D4091BA075091BB076091BC07709178
:1069A000BD078EE692E20E94109E80E00E943B7E30
:1069B00082EE94E00E94D49C8CED94E00E946F1DC6
:1069C0000C94A942F1018081918192FF11C0868DC2
:1069D000978DA0A1B1A120916807892B8A2B8B2BC1
:1069E00019F0822F806202C0822F8F7D809368070A
:1069F000C1010E94B27F882359F041E061E081E04B
:106A00000E9464ED811104C082E19CE00E94FA9C26
:106A100061E081E00E9465E70C94A9420E94611D3B
:106A2000D1018D919C91119793FF07C092968D9003
:106A30009D90AD90BC90959703C0812C912C5401F2
:106A400092FF0BC0F101268D378D40A151A1A8EE18
:106A5000B3E00F944D084B015C010E9473FE6B0183
:106A60007C01C80CD91CEA1CFB1C0E9473FEA70108
:106A70009601261B370B480B590BDA01C90181150A
:106A80009449A543B74710F00C94A9420E94B195D0
:106A900081E00E943F1DE9CF1092F2070C94A942B9
:106AA000D1018D919C91AC01487355274115510539
:106AB00051F49C0166E0369527956A95E1F7B1E0BF
:106AC0002B27217001C020E086FF08C01092AA0782
:106AD0001092AB071092AC071092AD07211117C0AE
:106AE000452BD1F0AC0125E0569547952A95E1F765
:106AF000BC0134E0769567953A95E1F753E09695B9
:106B000087955A95E1F761704170817003C061E02B
:106B100041E081E00E942C8580E00E943B7E379915
:106B200002C00C94CC428FEF9BE00E94779387EFDA
:106B30009BE00E94D49C379B04C084EF9BE00E94A2
:106B4000D49C0E948E1C882321F081EF9BE00E9440
:106B5000D49C0E94931C882321F08EEE9BE00E941F
:106B6000D49C8EEC9BE075C00E94FE22811111C066
:106B70006AEF70E080E090E00E94A2FE0E94FE2298
:106B8000811107C08EEA9BE00E94ED9C85E99BE0A5
:106B900072C180E89BE00E9477932091A406309117
:106BA000A5064091A6065091A706298F3A8F4B8FD4
:106BB0005C8F80E090E00E94DF1C80E090E00E940B
:106BC000FF1C80E090E00E941F1D80E00E947CCAB4
:106BD0000E94C9CC84E190E0A0E0B0E0898B9A8B60
:106BE000AB8BBC8B86E1482E512C612C712C1DA2E5
:106BF00029893A894B895C892D873E874F87588B35
:106C000041E061E081E00E942C85379902C00C943C
:106C1000D7428DE69BE00E94779385E69BE00E9439
:106C2000D49C379B04C082E69BE00E94D49C0E94C7
:106C30008E1C882321F08FE59BE00E94D49C0E944B
:106C4000931C882321F08CE59BE00E94D49C8CE36C
:106C50009BE00E94ED9C0C94A942D1012D913C91A6
:106C6000119732FD02C00C94E2475E968D919D9182
:106C70000D90BC91A02D0297A105B10511F00C94C7
:106C8000E2470C945B4881EE9AE00E94ED9C89EC0F
:106C90009AE00E94779383EA9EE10E940E9DEDA107
:106CA000E1110C94A94281E00E943B7E298D3A8D2E
:106CB0004B8D5C8D2093A4063093A5064093A606C9
:106CC0005093A70687E899E00E946F1D8BE09FE133
:106CD0000E947793212C312C8091180790911907ED
:106CE000A0911A07B0911B07898B9A8BAB8BBC8B39
:106CF00080E00E947CCA0E94C9CC81E00E9412857B
:106D000041E061E081E00E942C8580E00E941285D4
:106D10008CE09FE10E9477930E94971C9F938F9332
:106D20007F936F93B0EFAB2EB3E2BB2EB4E7CB2EC5
:106D3000B9E4DB2E8601750120E030E0A901CA012B
:106D4000B9010E94E98220E041E060E081E00E9418
:106D5000BB856B017C0120E041E060E081E00E94A6
:106D6000BB854B015C019B01AC01C701B6010F94CF
:106D7000D7032B013C010F900F900F900F902DEC3B
:106D80003CEC4CEC5DE30F947006181614F00C9478
:106D9000F8454D855E856F85788983E599E00E9489
:106DA000109E2D853E854F85588928323105410535
:106DB000510514F00C94044682E30E9478228D85DC
:106DC0009E85AF85B8890296A11DB11D8D879E87CE
:106DD000AF87B88BAC01BD0185E399E00E94109E9E
:106DE0006D8582E30E9455226D858AE30E945522BB
:106DF00082E30E947822B4E02B1631040CF46CCFAD
:106E000081E00E94128581E00E943B7E86E298E04C
:106E10000E946F1D8BE09FE10E947793298D3A8D30
:106E20004B8D5C8D2093A4063093A5064093A60657
:106E30005093A70641E061E081E00E942C8580E04C
:106E40000E947CCA41E06DEF72E083EC98E00E9402
:106E5000679B882371F083EC98E00E94C5986DEFE2
:106E600072E083EC98E00E94709C83EC98E00E94B2
:106E7000F9978CE098E00E9477930C94A94289E1FD
:106E80009FE10E94D49C8091000181FD02C068E4D2
:106E900001C06CE48AED9AE00E9429D40E94142378
:106EA0000C94A9428CE09FE10E94779310927207A4
:106EB00010927307109274071092750710926E0764
:106EC00010926F07109270071092710710926A0764
:106ED00010926B0710926C0710926D0780E00E9471
:106EE00012852091A4063091A5064091A6065091E6
:106EF000A70629A33AA34BA35CA30E94971C162FB5
:106F0000072FF82EE92E84E393E00E94701C9B016A
:106F1000AC0180E393E029AF3AAF4BAF5CAF0E9486
:106F2000701CEF92FF920F931F9350EFA52E53E228
:106F3000B52E54E7C52E59E4D52E8601750129AD2D
:106F40003AAD4BAD5CAD0E94E98220E041E060E0EB
:106F500081E00E94BB852B013C010F900F900F90A8
:106F60000F9020E030E0A9010F943C0487FF02C09D
:106F70000C94A9420E94971C162F072FF82EE92E79
:106F80008CE393E00E94701C9B01AC0188E393E0CA
:106F900029AF3AAF4BAF5CAF0E94701CEF92FF92EB
:106FA0000F931F938601750129AD3AAD4BAD5CADD2
:106FB0000E94E98221E041E060E080E00E94BB8520
:106FC0006D877E878F87988B0F900F900F900F9013
:106FD00020E030E0A9010F943C0487FF02C00C942C
:106FE000A9420E94971C162F072FF82EE92E84E441
:106FF00093E00E94701C9B01AC0180E493E029AFF8
:107000003AAF4BAF5CAF0E94701CEF92FF920F93B0
:107010001F938601750129AD3AAD4BAD5CAD0E9461
:10702000E98221E041E061E080E00E94BB854B0104
:107030005C010F900F900F900F9020E030E0A901BD
:107040000F943C0487FF02C00C94A942850174018F
:107050002D853E854F855889C301B2010E94618B01
:1070600080913E0790913F07A0914007B091410762
:107070008D879E87AF87B88B209152073091530739
:107080004091540750915507298B3A8B4B8B5C8B61
:10709000C0904607D0904707E0904807F090490716
:1070A00080914A0790914B07A0914C07B0914D07F2
:1070B0008D8B9E8BAF8BB88F2091A2073091A30749
:1070C0004091A4075091A5072DA33EA34FA358A715
:1070D0008091E6079091E707A091E807B091E90752
:1070E00089A79AA7ABA7BCA720914E0730914F075D
:1070F00040915007509151072D8F3E8F4F8F58A3CD
:107100008091420790914307A0914407B0914507B1
:10711000898F9A8FAB8FBC8F20919E0730919F07EC
:107120004091A0075091A1072DA73EA74FA758ABAC
:107130008091E2079091E307A091E407B091E50701
:1071400089AB9AABABABBCAB1092A8061092A90668
:107150001092AA061092AB06D1018D919C911197C5
:1071600092FFDCC05E968D919D910D90BC91A02DFB
:10717000AC01BD014150510961097109423051050D
:107180006105710548F00397A105B10509F0C6C076
:1071900080E00E947CCAC2C029893A894B895C89F7
:1071A0006D857E858F8598890F94E4062B013C01BF
:1071B0002D893E894F89588DC701B6010F94E40689
:1071C0009B01AC01C301B2010F94D7032B013C0119
:1071D0006DA17EA18FA198A50F940F059B01AC0115
:1071E000C301B2010F94E40629A53AA54BA55CA5FD
:1071F0000F94E4062B013C012D8D3E8D4F8D58A13F
:10720000C701B6010F94E4066B017C0129893A8914
:107210004B895C89698D7A8D8B8D9C8D0F94E406EA
:107220009B01AC01C701B6010F94D7036B017C0130
:107230006DA57EA58FA598A90F940F059B01AC01A4
:10724000C701B6010F94E40629A93AA94BA95CA984
:107250000F94E4069B01AC01C301B2010F94D80363
:107260006B017C01F7FAF094F7F8F0942D893E89D0
:107270004F89588D698D7A8D8B8D9C8D0F94E40686
:107280002B013C012D8D3E8D4F8D58A16D857E8546
:107290008F8598890F94E4069B01AC01C301B2016C
:1072A0000F94D7039B01AC01C701B6010F944304AF
:1072B0009B01AC01C501B4010F94D80320919A073A
:1072C00030919B0740919C0750919D070F94D703E5
:1072D0002091AC063091AD064091AE065091AF06BC
:1072E0000F94D803AB01BC014093AC065093AD069C
:1072F0006093AE067093AF0622E083E99EE10E94A0
:10730000EC9E81E00E941285F101868D978DA0A1EF
:10731000B1A10297A105B10509F43ACF81E00E941D
:1073200012850E94327281E00E943B7E84EB97E0DE
:107330000E946F1D41E061E081E00E942C8529A13F
:107340003AA14BA15CA12093A4063093A5064093DB
:10735000A6065093A7060C94A9422DEC3CEC4CECED
:107360005DEBC701B6010F943C0487FF85C0B301F4
:10737000A20184E997E00E94109E38E2431651046E
:1073800061047104CCF482E30E94782242E0440E4E
:10739000511C611C711CB301A20186E797E00E9499
:1073A000109E642D82E30E945522642D8AE30E9480
:1073B000552282E30E947822209118073091190704
:1073C00040911A0750911B07298F3A8F4B8F5C8F82
:1073D00080E00E947CCA0E94C9CC41E061E081E06B
:1073E0000E942C858CE09FE10E94779380E00E94B0
:1073F00012850E94971C9F938F937F936F9330EF1A
:10740000A32E33E2B32E34E7C32E39E4D32E860104
:10741000750120E030E0A901CA01B9010E94E982AA
:1074200020E041E060E081E00E94BB85698B7A8BBF
:107430008B8B9C8B20E041E060E081E00E94BB856B
:107440006D8B7E8B8F8B988F9B01AC0169897A89BC
:107450008B899C890F94D7036B017C010F900F904F
:107460000F900F902DEC3CEC4CEC5DE30F9470060C
:1074700018160CF072CF7BCF0E94971C162F072F87
:10748000F82EE92E84E493E00E94701C9B01AC016D
:1074900080E493E029AF3AAF4BAF5CAF0E94701C21
:1074A000EF92FF920F931F9320EFA22E23E2B22EB2
:1074B00024E7C22E29E4D22E8601750129AD3AAD0A
:1074C0004BAD5CAD0E94E98221E041E061E080E0EB
:1074D0000E94BB854B015C0121E041E061E080E05E
:1074E0000E94BB856B017C019B01AC01C501B4010D
:1074F0000F94D7036D8F7E8F8F8F98A30F900F906F
:107500000F900F902DEC3CEC4CEC5DE30F9470066B
:10751000181664F02DEC3CEC4CEC5DEB6D8D7E8D23
:107520008F8D98A10F943C0487FF13C0B301A20173
:1075300086E597E00E94109E82E30E94782252E046
:10754000450E511C611C711CB301A20188E397E038
:1075500026CF29893A894B895C896D897E898F89F3
:10756000988D0F94D80320E030E040E05FE30F9463
:10757000E406698B7A8B8B8B9C8B20E030E0A90131
:107580000F943C0487FD18CFA5019401C701B601F3
:107590000F94D80320E030E040E05FE30F94E4066E
:1075A0009B01AC0169897A898B899C890F94D703E7
:1075B00020E030E040EA52E40F94E4066B017C01E5
:1075C00020E030E0A9010F943C0487FF31C0F7FAB6
:1075D000F094F7F8F09422E0B701A60187E39FE169
:1075E0000E94EC9E209118073091190740911A07CC
:1075F00050911B07C701B6010F9443049B01AC01D6
:107600000F94D8036B017C0122E0AB01BC0187E33E
:107610009FE10E94EC9EA70196016091180770916E
:10762000190780911A0790911B070F94D70318C070
:107630008090180790901907A0901A07B0901B0728
:10764000A5019401C701B6010F9443049B01AC014D
:107650000F94D8039B01AC01C501B4010F94D8036A
:10766000609318077093190780931A0790931B076C
:107670002CE53FE844EC52E460911807709119073B
:1076800080911A0790911B070F9443046B017C01B2
:107690002DEC3CEC4CE85FE30F947006181654F0A8
:1076A00026E636E646E65FE3C701B6010F943C04E2
:1076B00087FF12C08CE59FE8A4ECB2E48093180722
:1076C00090931907A0931A07B0931B0722E0AC010F
:1076D000BD018DE197E014C022E0498D5A8D6B8D7C
:1076E0007C8D80E197E00E94EC9E409118075091BC
:1076F000190760911A0770911B0722E083E097E059
:107700000E94EC9E8D859E85AF85B8898093A406E6
:107710009093A506A093A606B093A70681E00E94C9
:10772000128581E00E943B7E8EEF96E00E946F1DE5
:107730008BE09FE10E9477932D853E854F85588988
:107740002093A4063093A5064093A6065093A7065F
:1077500041E061E081E00E942C8580E00E947CCACB
:10776000F8C68091A4069091A506A091A606B091B6
:10777000A7068D8F9E8FAF8FB8A324E130E040E045
:1077800050E02D873E874F87588BD1018D919C917A
:10779000119792FF0CC05E968D919D910D90BC91BA
:1077A000A02D0297A105B10511F40C94A74941E061
:1077B00061E081E00E942C858CE09FE10E9477933C
:1077C00080E00E9412850E94971C162F072FF82E2A
:1077D000E92E84E393E00E94701C9B01AC0180E3DE
:1077E00093E029AF3AAF4BAF5CAF0E94701CEF92B1
:1077F000FF920F931F9300EFA02E03E2B02E04E739
:10780000C02E09E4D02E8601750129AD3AAD4BADED
:107810005CAD0E94E98220E041E060E081E00E94EE
:10782000BB85698F7A8F8B8F9C8F20E041E060E071
:1078300081E00E94BB8569A37AA38BA39CA39B01D3
:10784000AC01698D7A8D8B8D9C8D0F94D7036B0164
:107850007C010F900F900F900F902DEC3CEC4CECB6
:107860005DE30F947006181654F02DEC3CEC4CECD4
:107870005DEBC701B6010F943C0487FF2BC04D851B
:107880005E856F8578898EED96E00E94109E2D852D
:107890003E854F85588928323105410551050CF048
:1078A00074CF82E30E947822D1018D919C9192FF46
:1078B0006CCF2D853E854F8558892E5F3F4F4F4FAA
:1078C0005F4F2D873E874F87588BBA01A90180EC07
:1078D00096E086C08DE793E00F94BB0C9A8B898B62
:1078E0000E94971C162F072FF82EE92E8CE393E0A9
:1078F0000E94701C9B01AC0188E393E029AF3AAF72
:107900004BAF5CAF0E94701CEF92FF920F931F93DE
:1079100010EFA12E13E2B12E14E7C12E19E4D12EDF
:107920008601750129AD3AAD4BAD5CAD0E94E9828F
:1079300021E041E060E080E00E94BB856DA37EA372
:107940008FA398A721E041E060E080E00E94BB8522
:1079500069A77AA78BA79CA79B01AC016DA17EA10B
:107960008FA198A50F94D7036B017C010F900F9006
:107970000F900F902DEC3CEC4CEC5DE30F947006F7
:10798000181654F02DEC3CEC4CEC5DEBC701B60145
:107990000F943C0487FF32C04D855E856F857889E2
:1079A00080EA96E00E94109E8D859E85AF85B889FD
:1079B0008897A105B1050CF0E8CE82E30E947822F9
:1079C0002D853E854F8558892E5F3F4F4F4F5F4F26
:1079D0002D873E874F87588BBA01A90182E896E030
:1079E0000E94109E6D8582E30E9455226D858AE378
:1079F0000E94552282E30E947822C7CE8FE793E04F
:107A00000F94BB0C9E8B8D8B0E94971C162F072FFB
:107A1000F82EE92E84E493E00E94701C9B01AC01D7
:107A200080E493E029AF3AAF4BAF5CAF0E94701C8B
:107A3000EF92FF920F931F93B0EFAB2EB3E2BB2EEA
:107A4000B4E7CB2EB9E4DB2E8601750129AD3AAD42
:107A50004BAD5CAD0E94E98221E041E061E080E055
:107A60000E94BB854B015C0121E041E061E080E0C8
:107A70000E94BB856B017C019B01AC01C501B40177
:107A80000F94D7032B013C010F900F900F900F9094
:107A90002DEC3CEC4CEC5DE30F947006181654F0A2
:107AA0002DEC3CEC4CEC5DEBC301B2010F943C04BB
:107AB00087FF25C04D855E856F85788982E696E0D3
:107AC0000E94109E8D859E85AF85B8898897A105F7
:107AD000B1050CF05ACE82E30E9478222D853E85B6
:107AE0004F8558892E5F3F4F4F4F5F4F2D873E8701
:107AF0004F87588BBA01A90184E496E071CFA501A4
:107B00009401C701B6010F94D80320E030E040E0B3
:107B10005FE30F94E4066DA77EA78FA798AB81E87B
:107B200093E00F94BB0C8C01D1018D919C91119726
:107B300092FF0CC05E968D919D910D90BC91A02DF1
:107B4000892B8A2B8B2B11F00C94BA49298D3A8DF5
:107B50004B8D5C8D69A17AA18BA19CA10F94D80358
:107B600020E030E040E05FE30F94E406698F7A8F15
:107B70008B8F9C8F2D8D3E8D4F8D58A12093A40609
:107B80003093A5064093A6065093A70681E00E9475
:107B90001285D1018D919C91119792FFABC05E9699
:107BA0008D919D910D90BC91A02D0297A105B105DD
:107BB00009F0A0C020E030E040EA52E4698D7A8DFF
:107BC0008B8D9C8D0F94E40620E030E048EC54E46B
:107BD0000F94D7030F94DC046B017C0129893A8947
:107BE000442737FD4095542F298B3A8B4B8B5C8B68
:107BF0002DA13EA14FA158A569A57AA58BA59CA54D
:107C00000F94D80320E030E040E05FE30F94E406F7
:107C100020E030E040EA52E40F94E40620E030E057
:107C200048EC54E40F94D7030F94DC042B013C017F
:107C30008D899E89AA2797FDA095BA2F8D8B9E8B43
:107C4000AF8BB88F20E030E040EA52E46DA57EA50E
:107C50008FA598A90F94E40620E030E048EC54E4A6
:107C60000F94D7030F94DC044B015C01222717FD0E
:107C70002095322FC414D504E604F70414F00C94B4
:107C8000D249C814D904EA04FB0414F00C94FA494C
:107C90004C185D086E087F088D899E89AF89B88D64
:107CA000480E591E6A1E7B1E8C189D08AE08BF0820
:107CB000800E911EA21EB31EC2010E94FF1CC401B1
:107CC0000E941F1DC12CD12C7601A1E94A16A1E00A
:107CD0005A066104710414F00C942E4AB1E98B1613
:107CE000B1E09B06A104B10414F00C942E4A80E08C
:107CF0000E947CCA20E030E0A901698D7A8D8B8DCD
:107D00009C8D0F943C0487FD40CD20E030E0A9011C
:107D10006DA57EA58FA598A90F943C0487FD35CD50
:107D200081E00E943B7E8AE096E00E946F1D8BE01E
:107D30009FE10E9477932D8D3E8D4F8D58A120930A
:107D4000A4063093A5064093A6065093A70641E0EB
:107D500061E081E00E942C85FCC31092AF07F10125
:107D6000EB5AFF4F8081882309F4F3C385EF95E038
:107D70000CC081E08093AF07F101EB5AFF4F808187
:107D8000882309F4E6C380EE95E00E94049DE1C3D8
:107D900080906A0790906B07A0906C07B0906D0779
:107DA00040906E0750906F07609070077090710759
:107DB000C0907207D0907307E0907407F090750739
:107DC000D1011C9113FF2BC01A96EC911A971B96A8
:107DD000FC911B971C960C911C971D96BC90809152
:107DE000F207882361F023E333E34BEC51E4BF0156
:107DF000802F9B2D0F94E406FB01DC0102C0A02F15
:107E0000BB2D209192073091930740919407509198
:107E10009507BF01CD010F94D7034B015C0114FFFF
:107E20002CC0D1011E96EC911E971F96FC911F97B6
:107E300050960C91509751967C908091F207882330
:107E400061F023E333E34BEC51E4BF01802F972D26
:107E50000F94E406FB01DC0102C0A02FB72D209196
:107E60009607309197074091980750919907BF0165
:107E7000CD010F94D7032B013C0115FF2CC0D1017C
:107E80005296EC9152975396FC91539754961C91AD
:107E9000549755960C918091F207882361F023E363
:107EA00033E34BEC51E4BF01812F902F0F94E40694
:107EB000FB01DC0102C0A12FB02F20919A07309165
:107EC0009B0740919C0750919D07BF01CD010F94E6
:107ED000D7036B017C0187017601A3019201C501E3
:107EE000B4010E940777F101808186FF32C3E689E1
:107EF000D1015796FC91579758961C9158975996CF
:107F00000C918091F207882361F023E333E34BEC7B
:107F100051E4BF01812F902F0F94E406FB01DC0197
:107F200002C0A12FB02F2091E4023091E5024091D0
:107F3000E6025091E702BF01CD010F94E4060F94D1
:107F4000DC046093AA077093AB078093AC0790930F
:107F5000AD07FFC280909A0790909B07A0909C0766
:107F6000B0909D072091AC063091AD064091AE06D1
:107F70005091AF06C501B4010F9443042DEC3CECC5
:107F80004CEC5DE30F94700618162CF48AEA95E029
:107F90000E940E9DDEC2F10122818081918122FF2B
:107FA0000CC083FF02C00C944A4A80739927892B26
:107FB00011F00C944A4A0C94504A83FF6FC0C2845B
:107FC000D384E484F58420E030E0A901C701B60140
:107FD0000F947006181664F420E030E040E251E49B
:107FE000C701B6010F943C0418160CF459C00AC01E
:107FF00020E030E040E251ECC701B6010F9470067A
:1080000087FD4EC0A5019401C701B6010F94D803A6
:108010009B01AC016091B8067091B9068091BA06D7
:108020009091BB060F94D8036093B8067093B9067D
:108030008093BA069093BB060E9432724091B806B4
:108040005091B9066091BA067091BB0623E08DEAA3
:1080500094E00E94EC9E8091B8069091B906A091A0
:10806000BA06B091BB0689879A87AB87BC8744E084
:1080700050E065E870E0CE0109960F94C00C0E94B4
:1080800065CA682F88E690E069AF0F94AE0C69ADC1
:10809000681721F088E690E00F94C90C10E001C049
:1080A00011E0F101808184FF71C0C684D784E0882B
:1080B000F18820E030E0A901C701B6010F947006F5
:1080C000181664F420E030E040E251E4C701B60144
:1080D0000F943C0418160CF458C00AC020E030E09D
:1080E00040E251ECC701B6010F94700687FD4DC008
:1080F000A5019401C701B6010F94D8039B01AC01FF
:108100006091B0067091B1068091B2069091B3066D
:108110000F94D8036093B0067093B1068093B206B3
:108120009093B3060E9432724091B0065091B1060E
:108130006091B2067091B30623E082E994E00E9458
:10814000EC9E8091B0069091B106A091B206B091DC
:10815000B3068D839E83AF83B88744E050E069E81F
:1081600070E0CE0105960F94C00C0E9465CA682F7E
:1081700088E690E069AF0F94AE0C69AD681731F0F6
:1081800088E690E00F94C90C01C011E0D1018C91F8
:1081900085FF74C05296CD90DD90ED90FC90559780
:1081A00020E030E0A901C701B6010F94700618164F
:1081B0005CF420E030E040E251E4C701B6010F94E6
:1081C0003C0418165CF00EC020E030E040E251ECB8
:1081D000C701B6010F94700687FF04C08BEF94E0CF
:1081E0000C944C4AA5019401C701B6010F94D80321
:1081F0009B01AC016091A8067091A9068091AA0626
:108200009091AB060F94D8036093A8067093A906CB
:108210008093AA069093AB060E9432724091A80602
:108220005091A9066091AA067091AB0623E087E7FA
:1082300094E00E94EC9E8091A8069091A906A091DE
:10824000AA06B091AB0689839A83AB83BC8344E0D2
:1082500050E06DE870E0CE0101960F94C00C0E94D2
:1082600065CA682F88E690E069AF0F94AE0C69ADDF
:10827000681721F088E690E00F94C90C1111AECF79
:1082800089E48F9384E78F9383E28F9380EF8F93BA
:10829000F0EFAF2EF3E2BF2EF4E7CF2EF9E4DF2E9E
:1082A000E12CF12C00E411E4A6019501C601B50111
:1082B0000E94E9820F900F900F900F904AC180E0CA
:1082C0000E94128510926A0710926B0710926C0739
:1082D00010926D0710926E0710926F071092700740
:1082E0001092710710927207109273071092740720
:1082F000109275076091C4027091C5028091C60208
:108300009091C7020E948A778091E8069091E906D1
:10831000A091EA06B091EB064091E0065091E1068B
:108320006091E2067091E306C090E406D090E50605
:10833000E090E606F090E7065A01F62FE72F48177F
:1083400059076A077B071CF45C01FA2FEB2F8501A4
:108350002F2F3E2F0C151D052E053F0514F49701F8
:108360008601480159018C189D08AE08BF086801B4
:108370007901C41AD50AE60AF70A28013901481A10
:10838000590A6A0A7B0AB501A40187EB91E20E94AF
:10839000109EB701A6018EEA91E20E94109EB301E1
:1083A000A20185EA91E20E94109EF10180819181F3
:1083B00092FFCDCC868D978DA0A1B1A1181619067C
:1083C0001A061B060CF0C3CCC4010E94DF1CC601B8
:1083D0000E94FF1CC2010E941F1DB9CC709069074A
:1083E00075FA772470F880E00E94128510929E073B
:1083F00010929F071092A0071092A1071092A20757
:108400001092A3071092A4071092A5071092A60736
:108410001092A7071092A8071092A90710926A0756
:1084200010926B0710926C0710926D0710926E07F6
:1084300010926F07109270071092710710927207D6
:108440001092730710927407109275071092B2077A
:108450001092B3071092B4071092B5071092B607A6
:108460001092B7071092B8071092B9071092BA0786
:108470001092BB071092BC071092BD076091C40216
:108480007091C5028091C6029091C7020E948A77BE
:108490000091CC061091CD062091CE063091CF06EA
:1084A0008091C0069091C106A091C206B091C3060A
:1084B000081B190B2A0B3B0B08511C4F2F4F3F4F2A
:1084C0008091E0069091E106A091E206B091E3066A
:1084D00048015901881A990AAA0ABB0A8091E8063C
:1084E0009091E906A091EA06B091EB066801790146
:1084F000C81AD90AEA0AFB0A8091E4069091E506B7
:10850000A091E606B091E706B901A801481B590BF6
:108510006A0B7B0B87EB91E20E94109EB501A401D0
:108520008EEA91E20E94109EB701A60185EA91E2CF
:108530000E94109E872D0E94128509CC80919B027B
:1085400082FF07C085E093E20E94D49CC1010E9493
:10855000BE940E9473FE60932C1D70932D1D80931A
:108560002E1D90932F1DEC960FB6F894DEBF0FBE14
:10857000CDBFDF91CF911F910F91FF90EF90DF90D2
:10858000CF90BF90AF909F908F907F906F905F90B3
:108590004F903F902F9008950E948E1C81110C9453
:1085A00093350E94931C81110C949335D2CF0E9475
:1085B0008E1C81110C9409360E94931C81110C941D
:1085C00009368CE09FE10E94779380E00E9412853B
:1085D0000E94971C162F072FF82EE92E84E393E0B4
:1085E0000E94701C9B01AC0180E393E029AF3AAF7D
:1085F0004BAF5CAF0E94701CEF92FF920F931F93E2
:1086000050EFA52E53E2B52E54E7C52E59E4D52ED2
:108610008601750129AD3AAD4BAD5CAD0E94E98292
:1086200020E041E060E081E00E94BB8569A77AA775
:108630008BA79CA720E041E060E081E00E94BB8521
:1086400069A37AA38BA39CA39B01AC0169A57AA51E
:108650008BA59CA50F94D7036B017C010F900F9005
:108660000F900F902DEC3CEC4CEC5DE30F947006FA
:10867000181654F02DEC3CEC4CEC5DEBC701B60148
:108680000F943C0487FF1AC049895A896B897C89F9
:1086900082E19BE00E94109E89899A89AB89BC89FE
:1086A0008897A105B10511F40C94433682E30E942A
:1086B0007822B301A20184EF9AE01BC18DE793E019
:1086C0000F94BB0C9E8B8D8BD1018D919C9111973A
:1086D00092FF0BC05E968D919D910D90BC91A02D47
:1086E0000297A105B10509F453C40E94971C162FE7
:1086F000072FF82EE92E8CE393E00E94701C9B015B
:10870000AC0188E393E029AF3AAF4BAF5CAF0E9476
:10871000701CEF92FF920F931F9300EFA02E03E2C5
:10872000B02E04E7C02E09E4D02E8601750129ADD4
:108730003AAD4BAD5CAD0E94E98220E041E060E0E3
:1087400081E00E94BB856DA77EA78FA798AB20E034
:1087500041E060E081E00E94BB8569AB7AAB8BAB06
:108760009CAB9B01AC016DA57EA58FA598A90F942C
:10877000D7036B017C010F900F900F900F902DECA1
:108780003CEC4CEC5DE30F947006181654F02DECA5
:108790003CEC4CEC5DEBC701B6010F943C0487FF49
:1087A00021C049895A896B897C898FE99AE00E94A6
:1087B000109E29893A894B895C8928323105410507
:1087C000510541F082E30E947822B301A20181E8C1
:1087D0009AE08FC08EE69AE00E94ED9C86E59AE0D2
:1087E0000C9449368FE793E00F94BB0C9E8F8D8FCE
:1087F000D1018D919C91119792FF0BC05E968D9146
:108800009D910D90BC91A02D0297A105B10509F491
:10881000CCC30E94971C162F072FF82EE92E84E454
:1088200093E00E94701C9B01AC0180E493E029AFAF
:108830003AAF4BAF5CAF0E94701CEF92FF920F9368
:108840001F9310EFA12E13E2B12E14E7C12E19E4ED
:10885000D12E8601750129AD3AAD4BAD5CAD0E94BC
:10886000E98220E041E060E081E00E94BB856B018D
:108870007C0120E041E060E081E00E94BB856DABBF
:108880007EAB8FAB98AF9B01AC01C701B6010F94D3
:10889000D7034B015C010F900F900F900F902DECC0
:1088A0003CEC4CEC5DE30F947006181654F02DEC84
:1088B0003CEC4CEC5DEBC501B4010F943C0487FF2C
:1088C00042C049895A896B897C898CE29AE00E946E
:1088D000109E29893A894B895C89283231054105E6
:1088E000510549F182E30E947822B301A2018EE092
:1088F0009AE00E94109E642D82E30E945522642D0E
:108900008AE30E94552282E30E947822F2E04F0E11
:10891000511C611C711C29893A894B895C892E5F25
:108920003F4F4F4F5F4F298B3A8B4B8B5C8B31E026
:108930003DA30C94F8358BEF99E00E94ED9C83EEFB
:1089400099E00C94493629A13AA14BA15CA169A5F3
:108950007AA58BA59CA50F94D80320E030E040E0D9
:108960005FE30F94E40620E030E040EA52E40F9425
:10897000E40620E030E048EC54E40F94D7030F9471
:10898000DC044B015C018D899E89AA2797FDA09587
:10899000BA2F8D8B9E8BAF8BB88F29A93AA94BA983
:1089A0005CA96DA57EA58FA598A90F94D80320E09A
:1089B00030E040E05FE30F94E40620E030E040EA7E
:1089C00052E40F94E40620E030E048EC54E40F94C5
:1089D000D7030F94DC042B013C012D8D3E8D4427E1
:1089E00037FD4095542F2D8F3E8F4F8F58A32DA9C3
:1089F0003EA94FA958ADC701B6010F94D80320E096
:108A000030E040E05FE30F94E40620E030E040EA2D
:108A100052E40F94E40620E030E048EC54E40F9474
:108A2000D7030F94DC046B017C0181E893E00F9481
:108A3000BB0C9C01442737FD4095542F29A33AA332
:108A40004BA35CA380E00E943B7E0E94327288E2CE
:108A50009FE10E94049D4091AC065091AD0660914B
:108A6000AE067091AF0622E083E99EE10E94EC9E83
:108A7000898D9A8DAB8DBC8D8093A4069093A506AD
:108A8000A093A606B093A70684149504A604B70481
:108A900014F58C149D04AE04BF040CF042C04818B9
:108AA00059086A087B082D8D3E8D4F8D58A1420EC6
:108AB000531E641E751EC818D908EA08FB0889A150
:108AC0009AA1ABA1BCA1C80ED91EEA1EFB1E812C27
:108AD000912C540152C0481459046A047B040CF5CB
:108AE0004C145D046E047F04E4F484189508A60811
:108AF000B7082D893E894F89588D820E931EA41E7A
:108B0000B51EC418D508E608F70889A19AA1ABA13B
:108B1000BCA1C80ED91EEA1EFB1E412C512C3201ED
:108B200025C0C814D904EA04FB0404F5C414D50410
:108B3000E604F704DCF48C189D08AE08BF082D8904
:108B40003E894F89588D820E931EA41EB51E4C1867
:108B50005D086E087F088D8D9E8DAF8DB8A1480E83
:108B6000591E6A1E7B1EC12CD12C760191E98916F3
:108B700091E09906A104B10474F4A1E94A16A1E0B8
:108B80005A06610471043CF4B1E9CB16B1E0DB068E
:108B9000E104F104FCF049895A896B897C8982EBF4
:108BA00099E00E94109E88E999E00E947793B501B0
:108BB000A40184E999E00E94109EB301A20180E91A
:108BC00099E00E94109EB701A6018CE899E00E94EE
:108BD000109EBFCCC4010E94DF1CC2010E94FF1C7A
:108BE000C6010E941F1D80E00E947CCA0C9453366F
:108BF0002DEC3CEC4CEC5DEBC301B2010F943C045A
:108C000087FF09C00C94C93682E299E00E94ED9C6E
:108C10008AE099E0D0C09FEF291A390AA501940192
:108C2000C701B6010F94D80320E030E040E05FE3D5
:108C30000F94E4062B013C014091AC065091AD0627
:108C40006091AE067091AF0622E08CEF98E00E9432
:108C5000EC9E20919A0730919B0740919C07509180
:108C60009D07C301B2010F94D7039B01AC01609132
:108C7000AC067091AD068091AE069091AF060F9450
:108C8000D8036093AC067093AD068093AE069093C4
:108C9000AF060E9432724091AC065091AD066091D1
:108CA000AE067091AF0622E08EEE98E00E94EC9E38
:108CB0000E94971C162F072FF82EE92E84E493E0CC
:108CC0000E94701C9B01AC0180E493E029AF3AAF95
:108CD0004BAF5CAF0E94701CEF92FF920F931F93FB
:108CE000A0EFAA2EA3E2BA2EA4E7CA2EA9E4DA2E98
:108CF0008601750129AD3AAD4BAD5CAD0E94E982AC
:108D000020E041E060E081E00E94BB856B017C01D6
:108D100020E041E060E081E00E94BB856D8B7E8BAE
:108D20008F8B988F9B01AC01C701B6010F94D703BD
:108D30004B015C010F900F900F900F902DEC3CECCD
:108D40004CEC5DE30F947006181654F02DEC3CECDF
:108D50004CEC5DEBC501B4010F943C0487FF33C0BC
:108D60004D855E856F8578898FEB98E00E94109E17
:108D70002D853E854F85588928323105410551059D
:108D8000A4F482E30E9478228D859E85AF85B88900
:108D90000296A11DB11D8D879E87AF87B88BAC0150
:108DA000BD0181EA98E00C94EE368EE898E00E94CE
:108DB000ED9C86E798E00E94779383EA9EE10E940B
:108DC0000E9D0C9400372D893E894F89588DC7011F
:108DD000B6010F94D80320E030E040E05FE30F9449
:108DE000E4069B01AC01C301B2010F94D70320E05C
:108DF00030E040EA52E40F94E4066B017C0120E08D
:108E000030E0A9010F943C0487FF27C0C701B601D9
:108E10009058209118073091190740911A075091E6
:108E20001B070F9443049B01AC010F94D8036B0103
:108E30007C0122E0AB01BC0187E39FE10E94EC9E34
:108E4000A7019601609118077091190780911A0780
:108E500090911B070F94D70318C08090180790902B
:108E60001907A0901A07B0901B07A5019401C7012C
:108E7000B6010F9443049B01AC010F94D8039B01EE
:108E8000AC01C501B4010F94D80360931807709327
:108E9000190780931A0790931B07C0901807D0906A
:108EA0001907E0901A07F0901B072CE53FE844EC07
:108EB00052E4C701B6010F9443044B015C012DEC51
:108EC0003CEC4CE85FE30F947006181654F026E66D
:108ED00036E646E65FE3C501B4010F943C0487FF24
:108EE00013C022E0B701A6018BE598E00E94EC9E3A
:108EF0008CE59FE8A4ECB2E48093180790931907DF
:108F0000A0931A07B0931B0722E049895A896B89FD
:108F10007C8983E498E00E94EC9E40911807509170
:108F2000190760911A0770911B0722E08BE298E005
:108F30000E94EC9E94E02916310414F00C94003742
:108F400029893A894B895C896091180770911907C2
:108F500080911A0790911B070F94D7036B017C0136
:108F60002DEC3CEC4CEC5DE30F947006181614F4F9
:108F70000C946C362DEC3CEC4CEC5DEBC701B6016F
:108F80000F943C0487FF02C00C946C360C9400379D
:108F900041E061E081E00E942C858CE09FE10E942D
:108FA000779380E00E941285A0CB41E061E081E0F0
:108FB0000E942C858CE09FE10E94779380E00E94C4
:108FC000128527CCC90188719927489709F474C183
:108FD00020E041E060E081E00E94BB8520919A079B
:108FE00030919B0740919C0750919D070F94D703A8
:108FF0004B015C0120E041E061E080E00E94BB8524
:1090000020919A0730919B0740919C0750919D07B2
:109010000F94D7032B013C019B01AC01C501B401A6
:109020000F94D7036B017C012DEC3CEC4CEC5DE321
:109030000F947006181654F02DEC3CEC4CEC5DEBE4
:10904000C701B6010F943C0487FF21C022E0B7019D
:10905000A6018AEE97E00E94EC9E82E30E947822AD
:1090600046E150E060E070E08CEC97E00E94109EDA
:1090700066E182E30E94552266E18AE30E9455225E
:1090800082E30E94782288EC97E00C943B37A3019E
:109090009201C501B4010F94D80320E030E040E014
:1090A0005FE30F94E406AB01BC0122E089EB97E09B
:1090B0000E94EC9E4ECA8091A4069091A506A091B4
:1090C000A606B091A7068D879E87AF87B88BF10162
:1090D0008081918192FF09C0868D978DA0A1B1A159
:1090E0000297A105B10509F4AEC041E061E081E05D
:1090F0000E942C858CE09FE10E94779380E00E9483
:1091000012850E94971C9F938F937F936F93F0EF2C
:10911000AF2EF3E2BF2EF4E7CF2EF9E4DF2E860167
:10912000750120E030E0A901CA01B9010E94E9827D
:1091300020E041E060E081E00E94BB854B015C01E2
:1091400020E041E060E081E00E94BB856B017C0192
:109150009B01AC01C501B4010F94D7032B013C0165
:109160000F900F900F900F902DEC3CEC4CEC5DE3CA
:109170000F947006181654F02DEC3CEC4CEC5DEBA3
:10918000C301B2010F943C0487FF05C083EA9EE14E
:109190000E940E9D9CCFA5019401C701B6010F94BA
:1091A000D80320E030E040E05FE30F94E4066B0179
:1091B0007C0120E030E040E85FE30F943C0487FD51
:1091C00086CFD1018D919C91119792FF0BC05E9635
:1091D0008D919D910D90BC91A02D892B8A2B8B2B6D
:1091E00009F043C02D853E854F8558892093A406FC
:1091F0003093A5064093A6065093A70681E00E94EF
:109200001285D1018D919C91119792FF0BC05E96B2
:109210008D919D910D90BC91A02D0297A105B10556
:1092200009F446C081E00E943B7E87E098E00E94FE
:109230006F1D8BE09FE10E9477932D853E854F85C2
:1092400058890C949F3E20E030E843E953E4209392
:10925000AC063093AD064093AE065093AF0680E067
:109260000E947CCA0E94C9CC40CF20919A073091BD
:109270009B0740919C0750919D07C701B6010F9431
:10928000D7039B01AC016091AC067091AD06809153
:10929000AE069091AF060F94D8036093AC0670931E
:1092A000AD068093AE069093AF060E9432729ACFBD
:1092B00080E00E947CCAB6CF30FF27C0D1011E9645
:1092C0002D913D914D915C9151971A966D917D91A3
:1092D0008D919C911D975D96EC915D97EF935C96B7
:1092E000EC915C97EF935B96EC915B97EF935A96BA
:1092F000EC91EF93E0EFAE2EE3E2BE2EE4E7CE2E4C
:10930000E9E4DE2E860175011BC00E94971CF10165
:1093100026853785408951894284538464847584C5
:109320009F938F937F936F9360EFA62E63E2B62E89
:1093300064E7C62E69E4D62E86017501C301B20129
:109340000E94E9820F900F900F900F9041CE80E025
:1093500090E00E94DF1C80E090E00E94FF1C80E013
:1093600090E00E941F1D80E00E947CCA0E94C9CC30
:109370000C94D73B80E00E943B7E0E94327288E2D0
:109380009FE10E94049D4091AC065091AD06609112
:10939000AE067091AF0622E083E99EE10E94EC9E4A
:1093A0000C94A63D4C145D046E047F041CF5481417
:1093B00059046A047B04F4F4C418D508E608F708D5
:1093C00089899A89AB89BC89C80ED91EEA1EFB1E01
:1093D00084189508A608B708800E911EA21EB31E19
:1093E000C6010E94DF1CC4010E941F1D412C512C8C
:1093F00032012BC08C149D04AE04BF0434F58414D8
:109400009504A604B7040CF5C818D908EA08FB08A7
:1094100029893A894B895C89C20ED31EE41EF51E48
:10942000481859086A087B088D899E89AF89B88DCC
:10943000480E591E6A1E7B1EC6010E94DF1CC20117
:109440000E94FF1C812C912C540191E9C91691E0D6
:10945000D906E104F10414F40C94653E4D855E8553
:109460006F8578898BE196E00E94109EB701A60176
:1094700087E196E00E94109EB301A20183E196E08D
:109480000E94109EB501A4018FE096E00E94109EFC
:109490000C94C53B80E895E00E940E9D0C944041E1
:1094A000C6A4D7A4E0A8F1A820E030E0A901C70134
:1094B000B6010F943C04882361F120E030E0A9015B
:1094C000C701B6010F94700618165CF420E030E076
:1094D00040E251E4C701B6010F943C041816B4F001
:1094E0000AC020E030E040E251ECC701B6010F9421
:1094F000700687FD0BC085E793E00E94701C9B01FE
:10950000AC01C701B6010F94D8034DC087E595E0C3
:10951000C3CF20E030E0A9016091920770919307DA
:1095200080919407909195070F943C04811161C03C
:1095300020E030E0A9016091960770919707809133
:109540009807909199070F943C04811152C0809123
:10955000690787FF2CC0C0902407D0902507E090B2
:109560002607F09027076091B6077091B7078091A2
:10957000B8079091B9070F940D059B01AC010F94AA
:10958000E4069B01AC01C701B6010F94D7030F9409
:1095900051072091EA073091EB074091EC07509179
:1095A000ED070F94E4060E949A1C0C944041C09071
:1095B0002407D0902507E0902607F09027076091B8
:1095C000B6077091B7078091B8079091B9079B01D2
:1095D000AC010F94AB07C61AD70AE80AF90AC7010B
:1095E000B6010E949BD4BC0180E090E00F940D0571
:1095F000D0CF84E295E050CFCF93DF93EC01409140
:109600009B028881998144FF09C082FD2AC081FFA5
:1096100005C02E813F812F36310519F582FF05C027
:10962000CE01DF91CF910C94C53381FF05C0CE01EF
:10963000DF91CF910C944B2391FF08C00E94611DD4
:10964000CC5ADF4F8881DF91CF91DEC242FF13C039
:1096500085E093E20E94D49CCE01DF91CF910C94DF
:10966000BE940E9473FE60932C1D70932D1D8093F9
:109670002E1D90932F1DDF91CF9108958091670744
:1096800080FD1DC00E94B1950E943D90EC0187E1D4
:109690009AE00E94C5C52097B1F080912E098823D9
:1096A00041F0888181FF12C08E819F814D9771F4B6
:1096B00016C0CE01A1DFCE010E949C9504C087E1B7
:1096C0009AE00E94C5C50E942877D8CFBE0183ECDE
:1096D00098E00E94DD98CE010E948B95ECCF83EC40
:1096E00098E00E94529CF7CF0E94B9890C94932273
:1096F000C5CFCF93DF93FC01E05CFF4F208121FDBC
:109700001FC0DB014D915D916D917C91DC01AF5BE0
:10971000BF4F4D935D936D937C931397EC01CB5B9F
:10972000DF4FDC0117964D915D916D917C911A97F9
:10973000488359836A837B83822F897F82608083F9
:10974000DF91CF9108959F92AF92BF92CF92DF9217
:10975000EF92FF920F931F93CF93DF93EC015B0186
:109760008C01005C1F4FF801908092FC32C0CB84CA
:10977000DC84ED84FE84A70196016F81788589855C
:109780009A850F94D7039F7720E030E040E85FE3AD
:109790000F94D80320E030E040EA51E40F947006C3
:1097A0001816BCF0F50180819181A281B381FE0180
:1097B000EF5BFF4F80839183A283B383CB5BDF4F4B
:1097C000C882D982EA82FB82892D897F8460F80170
:1097D0008083DF91CF911F910F91FF90EF90DF90E9
:1097E000CF90BF90AF909F9008958091690784605B
:1097F00080936907089508952F923F924F925F9248
:109800006F927F928F929F92AF92BF92CF92DF9290
:10981000EF92FF920F931F93CF93DF93CDB7DEB7F5
:1098200064970FB6F894DEBF0FBECDBF382E292E39
:109830007A8769875A834983098B1A8B2B8B3C8BD8
:109840004AA45BA46CA47DA423E333E948E853E471
:10985000C501B4010F94D8036D837E838F839887ED
:1098600020E030E0A901C301B2010F943C04882339
:1098700059F12EA53FA548A959A9C301B2010F94DA
:10988000D8034B015C0120E030E040EA50E4C30122
:10989000B2010F94E406A50194010F9443046D876F
:1098A0007E878F87988BA30192016EA57FA588A9DB
:1098B00099A90F94E406A50194010F9443046EA79F
:1098C0007FA788AB99AB08C080E090E0A0EAB0E445
:1098D0008D879E87AF87B88B2D813E814F815885BC
:1098E00069897A898B899C8990580F9443040F94D5
:1098F000B0049B01AC01C701B6010F94E4066D836F
:109900007E838F83988769817A81A985BA856A1B4E
:109910007B0B882777FD8095982F0F940F0520E00B
:1099200030E040E05DE30F94E40669877A878B8737
:109930009C87032D122D212C312C89819A81AA27F5
:1099400097FDA095BA2F89839A83AB83BC83A89592
:1099500069817A818B819C810F940F056B017C0159
:10996000B101882777FD8095982F0F940F052985E1
:109970003A854B855C850F94E4069B01AC01C701D9
:10998000B6010F94D7036B017C0123E333E548E86C
:1099900053E40F94D8039B01AC0169897A898B89C0
:1099A0009C890F9443040F94B0042D813E814F8114
:1099B00058850F94E4064B015C0120E030EC4FE742
:1099C00055E40F94E4062D853E854F8558890F9404
:1099D000E4062B013C01A50194016EA57FA588A991
:1099E00099A90F94D80320E030E040EA50E40F94A6
:1099F000E4069B01AC01C301B2010F9443040F9430
:109A0000DC046D3F9FE0790714F06CEF7FE0D80134
:109A10006D937C9320E030E040E051E4C701B60153
:109A20000F94E4060F94DC04F80173836283FFEF64
:109A30002F1A3F0A0C5F1F4F81E22816310409F0EC
:109A400086CF64960FB6F894DEBF0FBECDBFDF9110
:109A5000CF911F910F91FF90EF90DF90CF90BF902B
:109A6000AF909F908F907F906F905F904F903F90BE
:109A70002F9008957F928F929F92AF92BF92CF9234
:109A8000DF92EF92FF920F931F93CF93DF938CE0BF
:109A900092E0909337038093360385E4782E7F928B
:109AA000D2E9DF93C0EECF931F921F921F921F92B5
:109AB0001F92812C912C98ECA92E91E4B92EC12CE7
:109AC00020E5D22E23ECE22E27E4F22E00E010E176
:109AD0002BE835E44CE251E06EEC7FEF8DEB93E048
:109AE0008BDE7F92DF93CF931F921F921F921F9264
:109AF0001F9200E018E728E835E44CE251E06CEEF4
:109B00007FEF89E393E078DE80910A01806480939F
:109B10000A013B9A809119022DB73EB7205F3F4F53
:109B20000FB6F8943EBF0FBE2DBF87FD0CC061E09D
:109B30000E9487FF80911A02811105C061E0809127
:109B400019020E94C0FF0E9473FE60934602709348
:109B5000470280934802909349029D9AA598DF910D
:109B6000CF911F910F91FF90EF90DF90CF90BF901A
:109B7000AF909F908F907F900C948FD5CF92DF9273
:109B8000EF92FF92CF93DF93EC018B898130A9F59F
:109B9000CE8CDF8CE8A0F9A020E030E0A901C7015D
:109BA000B6010F943C04882341F1688D70E080E099
:109BB00090E00F940D0520E030E040E251E40F9476
:109BC000E406A70196010F9443046FA378A789A721
:109BD0009AA7698D70E080E090E00F940D0520E079
:109BE00030E040E251E40F94E406A70196010F949F
:109BF00043046BA77CA78DA79EA7DF91CF91FF9011
:109C0000EF90DF90CF9008954F925F926F927F9286
:109C1000AF92BF92CF92DF92EF92FF920F931F937A
:109C2000CF93DF93CDB7DEB72C970FB6F894DEBF96
:109C30000FBECDBF8091AA079091AB07A091AC0752
:109C4000B091AD07E0913603F0913703838F948F85
:109C5000A58FB68F2CE032E0309337032093360384
:109C60008093820790938307A0938407B09385071E
:109C700040901502509016026090170270901802E2
:109C80004092E4025092E5026092E6027092E7028E
:109C9000A301920160E070E080E89FE30F94430429
:109CA0006093EE077093EF078093F0079093F107AE
:109CB000C0901B02D0901C02E0901D02F0901E028A
:109CC000C092D402D092D502E092D602F092D7028E
:109CD00060911F02709120028091210290912202D6
:109CE0006093A8027093A9028093AA029093AB029A
:109CF0006093B8027093B9028093BA029093BB024A
:109D0000A30192010F94E4060F94E1046093DE072F
:109D10007093DF078093E0079093E1076093CE078D
:109D20007093CF078093D0079093D107209123029F
:109D3000309124024091250250912602C301B201C4
:109D40000F94E4069B01AC0160E074E284E798E4C0
:109D50000F9443040F944A050F94E104162F609367
:109D6000F607A3019201C701B6010F94E4069B0117
:109D7000AC0160E074E284E798E40F9443040F942C
:109D80004A050F94E104603118F46093F50703C0AD
:109D90008FE08093F5078091F507811710F01093FD
:109DA000F5076091F50770E080E090E00F940D05F5
:109DB000A30192010F94E4069B01AC0160E074E200
:109DC00084E798E40F9443042B013C01A70196011A
:109DD0000F943C0487FF08C04092D4025092D502F1
:109DE0006092D6027092D70287E392E0C7DE20919C
:109DF00092073091930740919407509195072D83D6
:109E00003E834F8358874090960750909707609005
:109E100098077090990780919A0790919B07A0915D
:109E20009C07B0919D0789879A87AB87BC87209153
:109E3000A4063091A5064091A6065091A706298355
:109E40003A834B835C83E0903603F0903703F7014D
:109E500081819281A381B4819C01AD01662777271E
:109E6000CB01621B730B840B950B0F940F05209194
:109E7000E2073091E3074091E4075091E5070F9422
:109E8000E406609398067093990680939A069093DF
:109E90009B06F70185819681A781B0859C01AD0164
:109EA00066277727CB01621B730B840B950B0F94EE
:109EB0000F052091E6073091E7074091E8075091A0
:109EC000E9070F94E40660939406709395068093D7
:109ED0009606909397068091A0069091A1060E9405
:109EE000BB1E8091680780FF24C08091BF028F93C2
:109EF0008091BE028F938091BD028F938091BC02AE
:109F00008F9330EFA32E33E2B32E34E7C32E39E420
:109F1000D32EE984FA840B851C85A30192016D81FF
:109F20007E818F8198850E947E7B0F900F900F908D
:109F30000F9089819A81AB81BC818093A406909314
:109F4000A506A093A606B093A70680E00E943B7EDC
:109F50002C960FB6F894DEBF0FBECDBFDF91CF9128
:109F60001F910F91FF90EF90DF90CF90BF90AF9037
:109F70007F906F905F904F900C9460D7089560E051
:109F800070E080E89FEB0895E0913603F09137038D
:109F9000858587FD06C061E09685911160E00C948F
:109FA000C0FF08958091190287FD07C061E090917C
:109FB0001A02911160E00C94C0FF08952F923F9215
:109FC0004F925F926F927F928F929F92AF92BF92C9
:109FD000CF92DF92EF92FF920F931F93CF93DF9375
:109FE00000D01F92CDB7DEB79C838B83DC01119626
:109FF000EC91E53338F4E23348F5EE2369F0ED30C7
:10A0000090F50DC0E43628F4E13648F4EC33F1F075
:10A010002AC0E436D9F027C049E150E026C0AB8120
:10A02000BC8112968C91A82FB0E0AA0FBB1FAF5B2A
:10A03000BB4F4D915C918CEF9FE0841B950BAB81E6
:10A04000BC8114969C938E93139715C0AB81BC81F1
:10A0500012968C91A82FB0E0AA0FBB1FAF5BBB4F2D
:10A060004D915C9102C04FEF5FE0AB81BC811496D3
:10A070005C934E931397AB81BC8113960D911C9109
:10A080001497E53338F5E23308F0A0C0EE2309F465
:10A0900050C0ED3008F081C1E1508E2F90E0FC01FE
:10A0A000E455F24F4491440FFC01EE0FFF1FE854BA
:10A0B000F24F85919491FC0185909490FC01329629
:10A0C000A590B4907CEF672E7FE0772E601A710A1E
:10A0D00052E03CC0E436C0F4E13608F0DBC0EC33BB
:10A0E00009F05BC1B801882777FD8095982F0F9400
:10A0F0000F0520E030E04AE754E40F94E40620E046
:10A1000030E040E859E325C1E43609F046C1B80122
:10A11000882777FD8095982F0F940F0520E030E079
:10A120004AEF53E40F94E40620E030E040E859E3BE
:10A130002CC180E090E0A8ECB1E4EB81FC81878346
:10A140009087A187B28729C151014801541708F0AF
:10A1500011C1FC01E50FF11DE50FF11D05911491F1
:10A16000FC0161E0650FE60FF11D5E5FE60FF11D7A
:10A1700025903490601671063CF7B501882777FD6D
:10A180008095982F0F940F056B017C01B30168191E
:10A190007909882777FD8095982F0F940F052B015B
:10A1A0003C01B1016A197B09882777FD8095982FBA
:10A1B0000F940F059B01AC01C301B2010F94E4069B
:10A1C0002B013C01B80168197909ADC0EE528E2F00
:10A1D00090E0FC01E455F24F6491660FFC01EE0F34
:10A1E000FF1FE854F24F85919491FC012590349023
:10A1F000FC0132968590949072E0761708F044C086
:10A20000FC01E70FF11DE70FF11DA590B490FC01D3
:10A2100021E0270FE20FF11D7E5FE20FF11D259176
:10A2200034910A151B056CF5B401882777FD8095DC
:10A23000982F29833A830F940F056B017C01B80195
:10A2400062197309882777FD8095982F0F940F0561
:10A250002B013C0129813A81B901681979098827C4
:10A2600077FD8095982F0F940F059B01AC01C301DA
:10A27000B2010F94E4062B013C01B5016219730988
:10A2800052C049011501B9CFB901882777FD8095E2
:10A29000982F75C0E23639F0A090BD03B090BE0390
:10A2A000EDEBF3E006C0A0903903B0903A03E9E388
:10A2B000F3E0828093804CEF642E4FE0742E601A9E
:10A2C000710A82E0048115818E5F268037806016D6
:10A2D00071060CF049C0B401882777FD8095982F4E
:10A2E0000F940F056B017C01B3016A197B09882764
:10A2F00077FD8095982F0F940F052B013C01B1013C
:10A3000068197909882777FD8095982F0F940F0594
:10A310009B01AC01C301B2010F94E4062B013C0187
:10A32000B8016A197B09882777FD8095982F0F94CB
:10A330000F059B01AC01C301B2010F9443049B01C3
:10A34000AC01C701B6010F94D80320E030E040E033
:10A350005EE30F94E406AB81BC8117966D937D9309
:10A360008D939C931A9719C03496823419F0410149
:10A370005801A8CFB101882777FD8095982F0F94B9
:10A380000F0520E030E040E05EE30F94E406EB814F
:10A39000FC8167837087818792870F900F900F9061
:10A3A0000F90DF91CF911F910F91FF90EF90DF9071
:10A3B000CF90BF90AF909F908F907F906F905F9065
:10A3C0004F903F902F9008958F929F92AF92BF929F
:10A3D000CF92DF92EF92FF920F931F93CF93DF9371
:10A3E000EC01CB01BA016B877C878D879E87FE01CC
:10A3F000E05CFF4F2081297F208320E030E040E0B7
:10A4000051E40F94E4060F94DC044B0129812533B9
:10A4100018F5223308F08AC0222309F448C02D30F1
:10A4200008F019C1215030E0F901E455F24FB49021
:10A43000BB0CF901EE0FFF1FE854F24F2591349148
:10A44000F901E590F490F901329645915491C12CAF
:10A45000D12CB2E0AB2E30C02436B0F4213608F057
:10A46000B4C02C3309F0F7C0882777FD8095982F6A
:10A470002CE0660F771F881F991F2A95D1F728EEC9
:10A4800033E040E050E09CC0243609F0E4C0882767
:10A4900077FD8095982F0CE0660F771F881F991F16
:10A4A0000A95D1F724EF31E040E050E089C01E82E8
:10A4B0001D82D1C0A8017D01AB1498F5F901EA0D08
:10A4C000F11DEA0DF11DA591B4916D01F90111E0A5
:10A4D0001A0DE10FF11DA394A394E10FF11D059155
:10A4E00014910815190534F79A01261B370BC7017B
:10A4F0008A1B9B0BDC016CEFC62E6FE0D62ECE18AC
:10A50000DF080F9432089A01201B310B442737FDD6
:10A510004095542F0F941008C20ED31EDE82CD82B8
:10A520009AC08CEF9FE08C199D0993C02E5230E0A9
:10A53000F901E455F24FA491AA0FF901EE0FFF1FA4
:10A54000E854F24F25913491F90105911491F901E4
:10A55000329645915491C12CD12CB2E0BA1768F5CE
:10A56000F901EB0FF11DEB0FF11DA590B490650102
:10A57000F901FF24F394FB0EEF0DF11DBE5FEF0D0B
:10A58000F11DE590F4908E149F04A4F49A01261B0B
:10A59000370BD801AA19BB090F9432089A012E195A
:10A5A0003F09442737FD4095542F0F941008200F82
:10A5B000311F08C0A7018501D1CFCD82DE824BC0FB
:10A5C0000F9410083E832D8346C0223639F0E09068
:10A5D000BD03F090BE03ADEBB3E006C0E0903903DD
:10A5E000F0903A03A9E3B3E012964D915C91139772
:10A5F00022E014960D911C9115972E5F1696ED9101
:10A60000FC911797E815F905D4F49A01261B370B2E
:10A61000D701A01BB10B0CEF1FE00E191F090F94FF
:10A6200032089A012E1B3F0B442737FD4095542FCB
:10A630000F941008020F131F1E830D830CC0149675
:10A64000223419F0AF017801D4CF8CEF9FE0801B4A
:10A65000910B9E838D83DF91CF911F910F91FF907E
:10A66000EF90DF90CF90BF90AF909F908F90089524
:10A670009F92AF92BF92CF92DF92EF92FF920F9391
:10A680001F93CF93DF936B017C01042F922EE091F7
:10A690000A02F0910B02C1E020E030E040E751E413
:10A6A00063857485858596850F94700618160CF061
:10A6B000C0E011E01C2720E030E041E953E4C7018D
:10A6C000B6010F94700618166CF020E030E0A90176
:10A6D000C701B6010F943C0487FF0AC0C12CD12CDE
:10A6E000760106C0C12CD12C91E9E92E93E4F92E14
:10A6F000C02FD0E0FE01EE0FFF1FE65FFD4FA080F0
:10A70000B180F5018181811103C0C12CD12C76016A
:10A71000B701A601C50158DE992081F020E030E0A4
:10A7200040EF51E4C701B6010F947006181634F4D7
:10A73000F501E05CFF4F80818160808320E030E0A4
:10A7400040E252E4C701B6010F94700687FD0EC0C7
:10A7500023E82C9FC0012D9F900D1124845F9D4FF5
:10A76000FC01E458FF4F208131962083602F70E078
:10A7700080E090E00F940D05AB01BC0120E08BED73
:10A7800090E20E94299F20E0B701A6018FED92E29E
:10A790000E94EC9EE0910A02F0910B0220E030E072
:10A7A00040E751E463857485858596850F9470062E
:10A7B00018167CF0111119C0DF91CF911F910F91E4
:10A7C000FF90EF90DF90CF90BF90AF909F900C9450
:10A7D0004CD1112351F00E9473FE60938E0670934A
:10A7E0008F068093900690939106DF91CF911F91F1
:10A7F0000F91FF90EF90DF90CF90BF90AF909F9020
:10A800000895E0910A02F0910B02168215821386D8
:10A81000148615861686E081F0E0EE5DF24E108219
:10A820008FEF80938F0208952F923F924F925F9205
:10A830006F927F928F929F92AF92BF92CF92DF9250
:10A84000EF92FF920F931F93CF93DF93CDB7DEB7B5
:10A85000E5970FB6F894DEBF0FBECDBF9DAB8CABB6
:10A860004E8B5F8B688F798F2E8F0BAB0E9473FEA0
:10A870006A8F7B8F8C8F9D8FACA9BDA996968C918A
:10A8800090E0959587952C01662457FC6094762C72
:10A8900088EC90E20E94049DB4DFBE8DB0938F02DD
:10A8A000ACA9BDA9EC91F0E0EE5DF24E96968C91CC
:10A8B0008083BE8DB11104C080918802809389028B
:10A8C000530142012A8D3B8D4C8D5D8D2BA33CA302
:10A8D0004DA35EA32F8F38A349A35AA319821F86C5
:10A8E00030EA388B41E4498B1A8A1B8A50EA5C8B28
:10A8F00081E48D8B1BA61CA61DA61EA61FA218A652
:10A9000019A61AA6C12CD12C76011FA618AA19AA1D
:10A910001AAA91E099871E861D86A8958CA99DA9E3
:10A920004DDBACA9BDA917963C90179718960C91D2
:10A93000189719961C9119971A962C900E9473FEDD
:10A940006D837E838F839887232D302F412F522D47
:10A950006A897B898C899D890F943C0487FF04C098
:10A960003A8A0B8B1C8B2D8A232D302F412F522D91
:10A9700069817F85888999890F943C0487FD04C08B
:10A9800039820F87188B298AB985BB2309F449C0FE
:10A990002E893F89488D598D632D702F812F922DDF
:10A9A0000F94700618160CF086C08D819E81AF81C1
:10A9B000B8852BA13CA14DA15EA1821B930BA40BDA
:10A9C000B50B3E8D311105C044EC59E060E070E0FC
:10A9D00004C04CED55E060E070E0481759076A0785
:10A9E0007B0708F068C0ECA9FDA92081E22FF0E008
:10A9F000EE5DF24E242D281920838FA798ABA9ABCA
:10AA0000BAABFE89FA8B2F892B8B388D3C8B498D05
:10AA10004D8B8D819E81AF81B8858F8F98A3A9A31F
:10AA2000BAA32E893F89488D598D632D702F812FB0
:10AA3000922D0F943C0487FF11C28D819E81AF81BE
:10AA4000B8852F8D38A149A15AA1821B930BA40B65
:10AA5000B50B3E8D3111EFC048E853E160E070E086
:10AA6000481759076A077B0708F0F8C14D855E85CE
:10AA7000452B09F0E5C0ACA9BDA9EC91F0E0EE5D75
:10AA8000F24E882D840D8083ED85FE853196FE87FC
:10AA9000ED87FE89F9832F892F87388D388B498D73
:10AAA000498B8D819E81AF81B8858BA39CA3ADA37B
:10AAB000BEA391E0998720E030E040E252E46E8945
:10AAC0007F89888D998D0F94D8039B01AC01632DEC
:10AAD000702F812F922D0F94700618161CF489E5A3
:10AAE00090E23BC08D819E81AF81B8852A8D3B8DE0
:10AAF0004C8D5D8D821B930BA40BB50B893E93404F
:10AB0000A105B10558F080E00E941E238D819E8131
:10AB1000AF81B8858A8F9B8FAC8FBD8F8D819E81D1
:10AB2000AF81B885880F991FAA1FBB1F2BA13CA11D
:10AB30004DA15EA1821B930BA40BB50B2F8D38A1E9
:10AB400049A15AA1821B930BA40BB50B81389F44DA
:10AB5000A241B105E8F08CE390E20E940E9DE596DB
:10AB60000FB6F894DEBF0FBECDBFDF91CF911F911E
:10AB70000F91FF90EF90DF90CF90BF90AF909F909C
:10AB80008F907F906F905F904F903F902F9039CE35
:10AB90004D855E85463051050CF443C081EE9FE142
:10ABA0000E94049D2EDE5BA9552309F459C1ACA96E
:10ABB000BDA95A96CD92DD92ED92FC925D972FA1A0
:10ABC00038A549A55AA55E962D933D934D935C9368
:10ABD00091972BA53CA54DA55EA592962D933D93EF
:10ABE0004D935C93959781E053968C9380E0E59626
:10ABF0000FB6F894DEBF0FBECDBFDF91CF911F918E
:10AC00000F91FF90EF90DF90CF90BF90AF909F900B
:10AC10008F907F906F905F904F903F902F900C940B
:10AC20007CCA87E19AE00E94C5C561E087E19AE0AD
:10AC30000E94C6C572CE48EB5BE060E070E010CFCA
:10AC40002FA538A949A95AA9280F391F4A1F5B1FE8
:10AC500029873A874B875C872FA538A949A95AA924
:10AC6000281B390B4A0B5B0BCA01B901A5019401E2
:10AC70000F94AB0729853A854B855C850F941008A6
:10AC8000240D351D461D571D243131054105510543
:10AC9000A4F0ACA9BDA996968C9190E04497AA2700
:10ACA00097FDA095BA2F29013A0182179307A407AF
:10ACB000B50744F42C013D0105C034E1432E512C6D
:10ACC000612C712CECA9FDA926A1822F869590E01C
:10ACD000A0E0B0E084159505A605B7056CF4822FB9
:10ACE00090E001974C01AA2497FCA094BA2C8418F8
:10ACF0009508A608B70802C053014201B301A2019A
:10AD000080EC90E20E94F89DB501A4018BEB90E2EB
:10AD10000E94F89D22E049815F856889798984EBEA
:10AD200090E20E94299F22E04A895B896C897D8993
:10AD30008DEA90E20E94EC9E2D853E852330310500
:10AD40000CF499CEC501B4010F940F0520E030E05A
:10AD500040E850E40F94E4066B017C0129813F85B3
:10AD6000488959896A897B898C899D890F94D70381
:10AD700020ED3FE049E450E40F94E4069B01AC0170
:10AD8000C701B6010F9443046B017C0169857A8584
:10AD90008B859C850F940F0520E030E04AE754E452
:10ADA0000F94430469837A838B839C8322E0B701E9
:10ADB000A60187EA90E20E94299F22E049815A81F8
:10ADC0006B817C8181EA90E20E94EC9E2AE939E95C
:10ADD00049E15FE3C701B6010F94E4066B017C0112
:10ADE0009B01AC010F94D80329813A814B815C818E
:10ADF0000F9443046FA378A789A79AA729813A8162
:10AE00004B815C81C701B6010F94E40620E030E07D
:10AE100040E05EE30F94E4066BA77CA78DA79EA796
:10AE200084E990E20E94ED9C22E0B701A6018EE841
:10AE300090E20E94EC9E22E04FA158A569A57AA558
:10AE400088E890E20E94EC9E22E04BA55CA56DA5EF
:10AE50007EA582E890E20E94EC9E0DCE19862BCE54
:10AE6000E5960FB6F894DEBF0FBECDBFDF91CF9150
:10AE70001F910F91FF90EF90DF90CF90BF90AF9018
:10AE80009F908F907F906F905F904F903F902F900A
:10AE90000895CF93DF930E9473FEAB01BC018AED4E
:10AEA0009FE10E94F89DE0919102F0E0EE0FFF1FFC
:10AEB000E65FFD4FC081D1814F81588569857A85D4
:10AEC00022E08CE692E20E94299F4B855C856D858D
:10AED0007E8520E08CE692E20E94299FE881F0E0E6
:10AEE000EE5DF24E608170E08CE692E2DF91CF91F0
:10AEF0000C94D29D8091690782FF22C060E070E0CF
:10AF000080ED9FE10E94C69DE0910A02F0910B0244
:10AF100067817085818592850F94DC046051710989
:10AF20006D31714018F08BEB9FE102C081EB9FE126
:10AF30000E94ED9C84E89FE10E940E9D81E00895AF
:10AF400080E008952F923F924F925F926F927F928E
:10AF50008F929F92AF92BF92CF92DF92EF92FF9229
:10AF60000F931F93CF93DF9300D01F921F92CDB703
:10AF7000DEB7A8950E9473FE69837A838B839C83D6
:10AF800000910A0210910B0220E030E040E252E40E
:10AF9000D80117966D917D918D919C911A970F9480
:10AFA0003C0487FF10C020E030E040E252E4F801AA
:10AFB00063857485858596850F943C0487FF03C05F
:10AFC0001092890204C08091880280938902809146
:10AFD0008F02811109C080913803882309F46FC260
:10AFE0008150809338036BC2C8010E94DE4F80916C
:10AFF000690782FD1CC0D8011796CD90DD90ED90B9
:10B00000FC901A9720E030E040E851E4C701B60117
:10B010000F943C0487FD66C220E030E046E953E42B
:10B02000C701B6010F94700618160CF45BC2812C90
:10B030008091690782FD40C2FF24F394F8012385C3
:10B0400034854585568567817085818592850F9405
:10B05000700687FDF12C992493949F2441F4780184
:10B06000F0E4EF0EF11CD7018C9180FD48C2C9803D
:10B07000DA80EB80FC80F801E75BFF4F4080518075
:10B08000628073805801B1E4AB0EB11CF501808180
:10B090009181A281B381A7019601281B390B4A0B2C
:10B0A0005B0B421653066406750698F5180130E4EA
:10B0B000230E311CD101BC91BD838B2F867049F1C9
:10B0C0008091680786FF25C0FD81F1FF5DC2780190
:10B0D000E5E4EE0EF11CD7012D913D914D915C916F
:10B0E000F80167817085818592850F94D70320E0F0
:10B0F00030E040E85FE30F943C0487FD09C28D8196
:10B10000897FD1018C93BE016F5F7F4FC8010E9480
:10B11000794BD8019F968C919F971796CD90DD9093
:10B12000ED90FC901A97F801B4E08B9FE00DF11DB3
:10B130001124C0AAD1AAE2AAF3AA8F5F8370F801F2
:10B1400087A78389813009F0BCC043845484658417
:10B15000768420E030E040EA51E4C301B2010F946C
:10B160003C0487FDC0C0A7019601C301B2010F9442
:10B17000D7036B017C0120E030E040EA51E40F94FA
:10B18000700618160CF4C6C020E030E040EA51EC1E
:10B19000C701B6010F943C0487FDD0C0BE016F5FAC
:10B1A0007F4FC8010E94A34BF801228D338D448D3F
:10B1B000558DC701B6010F94E4062B013C01D8015F
:10B1C00054962D913D914D915C915797C701B601D1
:10B1D0000F94D8036B017C01F80123A434A4A5A427
:10B1E000B6A49101A5010F943C0487FD16C0D801B7
:10B1F00097962C90979798963C9098979996AC90A4
:10B2000099979A96BC909101A501B601C7010F9438
:10B210007006181614F016015701C101D501F80186
:10B22000848B958BA68BB78B268D378D40A151A132
:10B23000B101C5010F94E4062DEC3CEC4CEC5DE350
:10B240000F94E4069B01AC01C301B2010F94D80333
:10B250006B017C01D8019F968C91F801B4E08B9F23
:10B26000E00DF11D1124D80117962D913D914D91BE
:10B270005C911A9760A971A982A993A90F94D70329
:10B28000F80122A133A144A155A10F94E4062FEDAA
:10B290003FE445E550E40F94E4069B01AC01C7018F
:10B2A000B6010F94D8030F94DC0477FD47C0D80192
:10B2B00096962C9130E0261737070CF4B901F62E3C
:10B2C00098C0833009F09CC0F8014384548465849D
:10B2D000768420E030E040EA51E4C301B2010F94EB
:10B2E0003C0487FF07C0F801E05CFF4F8081897F45
:10B2F000808324C0A7019601C301B2010F94D70334
:10B300006B017C0120E030E040EA51E40F947006CC
:10B31000181654F4D8019696FC90BE016F5F7F4FCB
:10B32000C8010E94794B65C020E030E040EA51EC52
:10B33000C701B6010F943C0487FF02C0F12C59C02D
:10B34000BE016F5F7F4FC8010E94A34BF801C78009
:10B35000D084E184F28420E030E040E450E4648969
:10B360007589868997890F94E4062B013C01D801E1
:10B370009F968C91F801B4E08B9FE00DF11D112494
:10B3800020A931A942A953A9C701B6010F94D70337
:10B390002FED3FE445E550E40F94E4069B01AC013A
:10B3A000C301B2010F94D80320E030E040E85EE32F
:10B3B0000F94E406F801648B758B868B978B228D36
:10B3C000338D448D558D0F94E4069B01AC01C7016C
:10B3D000B6010F94D803D8011B962D913D914D9144
:10B3E0005C911E970F94700618160CF4A7CFF80105
:10B3F000F08CD801EC91F0E0EE5DF24EF0823CC0B2
:10B40000823021F589819A81AB81BC81F801478521
:10B410005089618972896C017D01C41AD50AE60AD6
:10B42000F70A29E8C21623E1D206E104F10420F16B
:10B430002081E22FF0E0EE5DF24E292D2195208350
:10B44000F8018787908BA18BB28B07C0E081F0E079
:10B45000EE5DF24E892D81958083992039F0BE01F1
:10B460006F5F7F4FC8010E94794B06C0F801E05C16
:10B47000FF4F8081897F808320E030E041E953E401
:10B48000F80167817085818592850F947006181682
:10B4900034F4D801EC91F0E0EE5DF24E1082809130
:10B4A0003603909137038B960817190729F49920D2
:10B4B00011F02F9A01C02F98882009F48CCD80912B
:10B4C000690782FFB8C0E0910A02F0910B02E081A7
:10B4D000F0E0EE5DF24E108280919B0288608093D6
:10B4E0009B02A9C0809138038F5F809338038B3013
:10B4F00018F00E94F54BFEDC8824839499CD63E01C
:10B5000082E30E94FF9FF70180818E7F8083AFCD11
:10B51000809138038F5F809338038B3008F478C0B4
:10B520000E94F54B41E068EE77E187E19AE00E94E6
:10B53000CBA881EA97E10E940E9DD7012D913D9104
:10B540004D915C91F80167817085818592850F949A
:10B55000D703AB01BC0122E08CE39DE00E94299F50
:10B5600049815A816B817C81F50180819181A28121
:10B57000B381481B590B6A0B7B0B84E39DE00E944F
:10B58000F89D80E39DE042C0F80123853485458520
:10B59000568567817085818592850F94D7039F7743
:10B5A00020E030E040EA51E40F94700618169CF554
:10B5B000809138038F5F809338038B3048F10E946D
:10B5C000F54B41E068EE77E187E19AE00E94CBA875
:10B5D00081EA97E10E940E9DF801EB5BFF4F4081ED
:10B5E00051816281738122E08EE09DE00E94299F5B
:10B5F000D80117964D915D916D917C911A9722E03B
:10B6000083E09DE00E94299F8BEF9CE00E94ED9CCF
:10B61000882483947ECDB8EECB0EB3E0DB1EE11C14
:10B62000F11CC418D508E608F708F501C082D182DC
:10B63000E282F3826ECD0F900F900F900F900F90DB
:10B64000DF91CF911F910F91FF90EF90DF90CF90FE
:10B65000BF90AF909F908F907F906F905F904F9032
:10B660003F902F9008958FEF8EBD0DB407FEFDCF54
:10B670008EB50895DC01680F791F80E090E0A61771
:10B68000B70779F02D91E92FFF27E227EE0FFF1F73
:10B69000EF5CFD4E25913491982F882782279327C0
:10B6A000EECF089522E090E0281728F4963019F0A4
:10B6B000220F9F5FF9CF209A289A219A229A2398E5
:10B6C000809164008B7F80936400892F806A8695C7
:10B6D0008CBD90FD03C081E0963009F480E08DBD03
:10B6E00008958EBD0DB407FEFDCF0895CF93FB01E5
:10B6F00020E030E22F5F31932B30E1F7DC0190E066
:10B7000037E02A2FEB2F8D9181110AC0DA012C939B
:10B710001196EC9381E0FB019081903241F526C0B7
:10B720008F32A1F3282F8E3219F0E1E3F4E108C043
:10B730003A30E1F098E03AE0E4CF3196C817B1F042
:10B74000C491C111FACF391718F080528F3508F023
:10B750002FE581E0890FFB01E90FF11D9FE9920FB1
:10B760009A3108F420522083982FCBCF80E0CF91DC
:10B7700008959B01255F3F4F80E0FB019191BF0140
:10B78000482F4695F0E88F9F400D1124842F890F94
:10B790006217730791F7089561E0FC0180810E94B0
:10B7A000C0FF8FEF9ECFCF93DF93EC018A817ADFCA
:10B7B00060E08881DF91CF910C94C0FFCF92DF923F
:10B7C000EF92FF920F931F93CF93DF93EC018B01C6
:10B7D0007A010E9473FE6B0146DF8B838F3F49F431
:10B7E0000E9473FE6C197D096D327140A8F381E1EE
:10B7F00031C08E3F11F08FE02DC0E114F104D9F07B
:10B80000C70101972FEF2EBDF8014FEF9F01201BBD
:10B81000310B2817390738F40DB407FEFDCF2EB5CC
:10B8200021934EBDF3CF0DB407FEFDCF2EB5F80129
:10B83000E80FF91F20831B8216DFD82E14DFC82ED5
:10B84000B701C80117DF2C2D30E03D292817390733
:10B8500031F08BE18983CE019FDF80E003C0CE0110
:10B860009BDF81E0DF91CF911F910F91FF90EF90CF
:10B87000DF90CF9008950F931F93CF93DF931F9284
:10B880001F92CDB7DEB78C0169837A838CDF40E0ED
:10B8900052E069817A81C8010F900F90DF91CF91BA
:10B8A0001F910F918BCF0F931F93CF93DF93EB01DA
:10B8B0000E9473FE8B01D7DE8F3F49F00E9473FE1A
:10B8C000601B710B6C177D07B0F380E001C081E055
:10B8D000DF91CF911F910F910895BF92CF92DF9288
:10B8E000EF92FF920F931F93CF93DF93CDB7DEB705
:10B8F0002A970FB6F894DEBF0FBECDBF8C01B62ECF
:10B900002F83388749875A874EDF6CE271E0C80180
:10B91000CADFFE01319686E0DF011D928A95E9F7C4
:10B920008B2D806489838A858A8389858B8388852A
:10B930008C838F818D83CE010696DF0120E059E054
:10B940004D9138E0220F642F622767FD2527440FB1
:10B950003150C1F7A817B90799F7220F21602E833C
:10B960007F016E01B7E0CB0ED11CF70181917F0101
:10B97000B8DEEC14FD04C9F7FCE0BF1201C073DEB1
:10B98000F12C71DED80113968C9387FF05C0BFEFB1
:10B99000FB1611F0F394F5CF2A960FB6F894DEBF9C
:10B9A0000FBECDBFDF91CF911F910F91FF90EF9010
:10B9B000DF90CF90BF900895BF92CF92DF92EF9229
:10B9C000FF920F931F93CF93DF93EC01B62E1C824F
:10B9D000198248830E9473FE8B0161E088810E9476
:10B9E00087FF61E088810E94C0FF2398229A219AF4
:10B9F000209A8BE08A8356DEE4E1FE2E8FEF71DE23
:10BA0000FA94E1F720E030E0A90160E0CE0165DFC3
:10BA1000813049F00E9473FE601B710B613D7740DD
:10BA200088F381E057C021E030E040E050E06BE374
:10BA3000CE0153DF813011F08AE14CC02AEA31E0B7
:10BA400040E050E068E0CE0148DF853011F481E04D
:10BA500009C074E0F72E07DE8B83FA94E1F78A3A87
:10BA600059F482E08C838C81823079F4C12CD12C02
:10BA7000E12C60E4F62E0CC00E9473FE601B710B7B
:10BA8000613D7740D8F282E025C0C12CD12C7601EF
:10BA900020E030E0A90167E3CE011FDFA701960196
:10BAA00069E2CE011ADF882349F00E9473FE601B11
:10BAB000710B613D774060F38AE00CC08C8182306D
:10BAC000B1F420E030E0A9016AE3CE0106DF88236B
:10BAD00029F088E08983CE015FDE14C0C4DD807C5C
:10BAE000803C11F483E08C83BEDDBDDDBCDDCE0186
:10BAF00053DE8EE08B1518F488E1898303C0BA8287
:10BB000081E001C080E0DF91CF911F910F91FF9004
:10BB1000EF90DF90CF90BF9008950F931F93CF9336
:10BB2000DF93EC0189018C81833039F0F9E0440F17
:10BB3000551F661F771FFA95D1F79A01AB0161E196
:10BB4000CE01CBDE811109C040E052E0B801CE0148
:10BB5000DF91CF911F910F9131CE84E08983CE0187
:10BB60001BDE80E0DF91CF911F910F910895CF935D
:10BB7000DF93EC018C81833039F089E0440F551F4D
:10BB8000661F771F8A95D1F79A01AB0162E1CE015A
:10BB9000A4DE882331F085E08983CE01FDDD80E0DD
:10BBA00003C0CE01F9DD81E0DF91CF910895CF93FD
:10BBB000DF93EC01F8DD20E030E0A9016CE0CE017C
:10BBC0008CDE882331F083E08983CE01E5DD80E0DF
:10BBD00003C0CE01E1DD81E0DF91CF910895CF92E6
:10BBE000DF92EF92FF920F931F93CF93DF931F92F9
:10BBF000CDB7DEB78C01E62E6A0160E072E0CA01C3
:10BC000039DDF82E8E2D99836CDDF60180818EBD95
:10BC1000418122E030E099810DB407FEFDCF4EBD99
:10BC20002115F2E03F0739F0F601E20FF31F4081E2
:10BC30002F5F3F4FF1CF0DB407FEFDCF892F51DDB0
:10BC40008F2D4FDD10DDF80183838F71853031F04A
:10BC500083E18183C801A0DD80E001C081E00F9015
:10BC6000DF91CF911F910F91FF90EF90DF90CF90D8
:10BC700008950F931F93CF93DF93EC0189018C817B
:10BC8000833039F039E0440F551F661F771F3A950E
:10BC9000D1F79A01AB0168E1CE011FDE882311F0D4
:10BCA00086E01EC0A8016EEFCE0199DF8823C9F09F
:10BCB00068E572E0CE01F7DD182F811102C087E13F
:10BCC0000FC020E030E0A9016DE0CE0106DE811159
:10BCD00006C0C9DC811103C0CE015EDD05C086E16E
:10BCE0008983CE0159DD10E0812FDF91CF911F9123
:10BCF0000F9108950F931F93CF93DF93EC018B0166
:10BD000052DD68E572E0CE01CEDD882351F0A80156
:10BD10006CEFCE0164DF182F882319F0CE013CDDD3
:10BD200005C085E18983CE0137DD10E0812FDF91E9
:10BD3000CF911F910F9108958F929F92AF92BF92D2
:10BD4000CF92DF92EF92FF920F931F93CF93DF93E7
:10BD5000EC016A017B014801590120E030E0A901B2
:10BD600067E3BBDDA501940167E1CE01B6DD882361
:10BD700011F089E012C08C81833039F049E0CC0C9D
:10BD8000DD1CEE1CFF1C4A95D1F7A701960169E165
:10BD9000CE01A3DD882331F087E08983CE01FCDC6E
:10BDA00080E003C0CE01F8DC81E0DF91CF911F91EC
:10BDB0000F91FF90EF90DF90CF90BF90AF909F904A
:10BDC0008F9008951F93CF93DF93EC01ECDC68E52F
:10BDD00072E0CE0168DD882361F08DEF82DC68E5DA
:10BDE00072E0CE0160DD182F882319F0CE01D4DC7B
:10BDF00005C082E18983CE01CFDC10E0812FDF9185
:10BE0000CF911F9108950F931F93CF93809150046A
:10BE100080FF41C0409151045091520460915304FD
:10BE20007091540425E534E080914A0490914B04CC
:10BE300020DFC82F811102C0C0E02EC080915004C5
:10BE400081FD06C0809150048E7F8093500424C0F1
:10BE500000914C0410914D0420914E0430914F04F8
:10BE6000011511052105310569F3409151045091E7
:10BE700052046091530470915404400F511F621F8B
:10BE8000731F25E534E080914A0490914B04F1DE64
:10BE90008111D8CFD1CFC1E08C2FCF911F910F91BD
:10BEA0000895CF92DF92EF92FF92CF936B017C01C6
:10BEB000C42F8091510490915204A0915304B091E9
:10BEC00054048C159D05AE05BF05F9F09CDF81116A
:10BED00003C080E090E021C0C2FF0BC0109250046C
:10BEE000C0925104D0925204E0925304F092540450
:10BEF0000CC025E534E0B701A60180914A04909179
:10BF00004B040BDE8111EACFE4CFC3708091500463
:10BF10008C2B8093500485E594E0CF91FF90EF90B7
:10BF2000DF90CF900895CF93DF93EC01462F6F857C
:10BF3000788989899A89B5DF009739F02C8130E2B8
:10BF4000239F800D911D112402C080E090E0DF91BD
:10BF5000CF9108950F931F93CF93DF93EC018B81C3
:10BF60008823D1F1898187FF32C061E0CE01DBDF18
:10BF70008C01009789F1FC018081853E69F18B81FC
:10BF8000823040F44B895C896D897E89448F558F5E
:10BF9000668F778F4F89588D698D7A8DF801538F11
:10BFA000428F758B648BE0915506F0915606309761
:10BFB00059F0B8016A5E7F4FC80148961995F8019B
:10BFC000808D918D938B828B89818F778983DF918F
:10BFD000CF911F910F9117CF81E0888380E0DF918F
:10BFE000CF911F910F910895CF93DF93EC01B2DFB2
:10BFF0001B82DF91CF9108958FEF9FEFDC0180933B
:10C00000510490935204A0935304B093540410929B
:10C01000500408958F929F92AF92BF92CF92DF9279
:10C02000EF92FF920F931F93CF93DF93EC016A017E
:10C030007B018901423051056105710508F454C046
:10C0400089859A85AB85BC850196A11DB11D841794
:10C050009507A607B70708F447C08F89803129F4F0
:10C060009927872F762F652F0BC08032E9F5CB01FA
:10C07000BA0127E096958795779567952A95D1F728
:10C080008B889C88AD88BE88680D791D8A1D9B1D94
:10C0900042E007DF009741F12F89203169F4DD2468
:10C0A000EE24FF24F601EE0FFF1FE80FF91F808139
:10C0B0009181A0E0B0E011C0E894C7F8DD24EE243F
:10C0C000FF24F601EE0FFF1FEE0FFF1FE80FF91F11
:10C0D00080819181A281B381BF70F80180839183B7
:10C0E000A283B38381E001C080E0DF91CF911F91F3
:10C0F0000F91FF90EF90DF90CF90BF90AF909F9007
:10C100008F9008952F923F924F925F927F928F92DD
:10C110009F92AF92BF92CF92DF92EF92FF920F93D6
:10C120001F93CF93DF93EC017B016A018B81811117
:10C1300003C08FEF9FEF17C1898180FFFACF4B8932
:10C140005C896D897E898B859C85AD85BE85460120
:10C15000A12CB12C8A019B01081B190B2A0B3B0B4C
:10C1600080169106A206B30618F06A01C81AD90A09
:10C1700086014E0127E0820E911C0115110509F47C
:10C180006EC02B843C844D845E84510181E0B822D2
:10C190008D819E81B201A101E9E076956795579561
:10C1A0004795EA95D1F7FC0174807A9474222B812B
:10C1B000223049F4228C338C448C558C240E351E4D
:10C1C000461E571E37C0A114B104C1F4711016C029
:10C1D00023282428252849F48F89988DA98DBA8D84
:10C1E0008F839887A987BA8709C04F815885698549
:10C1F0007A8594010FDF882309F49BCFED81FE81BE
:10C20000A4812F81388549855A85225031094109F9
:10C210005109B0E00F944D081B012C0186859785CC
:10C22000A089B189280E391E4A1E5B1E270C311CBD
:10C23000411C511CA114B104A1F40115F2E01F0727
:10C2400080F08091510490915204A0915304B091D8
:10C250005404281639064A065B06D9F402C0C60102
:10C2600082C040E0C201B1011CDE009709F461CF39
:10C2700020E032E02A193B0928012017310708F491
:10C280002901BC016A0D7B1DA201C7010F94550C49
:10C290002AC00115E4E01E07B8F1B12EB6942B8137
:10C2A000223009F040C0281639064A065B0608F01D
:10C2B00043C0B201A10180914A0490914B0457DC24
:10C2C000882309F436CF1701412C80914A049091BC
:10C2D0004B044B103BC06BDC882309F42ACF512C54
:10C2E000542C4424550CE40CF51C8B859C85AD85A1
:10C2F000BE85840D951DA11DB11D8B879C87AD87C3
:10C30000BE870419150939CF9701B201A1018091A7
:10C310004A0490914B0401DC882309F40ACF412C94
:10C3200042E0542EE0CFED81FE81248127192B15A8
:10C3300008F0B9CFB22EB7CF8B0D911DA11DB11D45
:10C34000281639064A065B0650F0B3CFB10193DADE
:10C350002EEF321A882309F4ECCE4394B6CF53DD86
:10C360008111A7CFE6CEDF91CF911F910F91FF9062
:10C37000EF90DF90CF90BF90AF909F908F907F9085
:10C380005F904F903F902F900895CF93DF931F922F
:10C39000CDB7DEB741E050E0BE016F5F7F4FB2DE48
:10C3A000019719F4898190E002C08FEF9FEF0F9001
:10C3B000DF91CF9108951F93CF93DF93EC018B8191
:10C3C000823018F480E090E023C04B855C856D8559
:10C3D0007E85A5E07695679557954795AA95D1F7FF
:10C3E000142F1F70CE01D1DF97FDECCF4B855C85FC
:10C3F0006D857E85415E5F4F6F4F7F4F4B875C87BA
:10C400006D877E8720E2129FC00111248B5A9B4FBB
:10C41000DF91CF911F910895AF92BF92CF92DF929B
:10C42000EF92FF920F931F93CF93DF931F92CDB79D
:10C43000DEB77C018A014115510511F0DA011C9229
:10C4400041E0BDE0CB2EA895C7014983B4DF5C0174
:10C450004981009709F47AC0FC012081222309F464
:10C4600075C0253009F467C0253E09F464C0FC019D
:10C470008385982F9F739F3009F054C001151105D3
:10C4800011F3828D938D892BF1F62F71E1F2233018
:10C49000D4F6332727FD309521503109C29EF00193
:10C4A000C39EF00D1124E00FF11FD50111968C9160
:10C4B0001197808313968C911397818315968C9195
:10C4C0001597828317968C911797838319968C9171
:10C4D000199784831E968C911E97858350968C9114
:10C4E0005097868352968C915297878354968C915D
:10C4F0005497808756968C915697818758968C9141
:10C50000589782875C968C915C9783875E968C9116
:10C510005E978487442309F496CF1D96DC90158698
:10C5200040E091CF982F967031F42E3261F4F501EE
:10C5300091819E3241F00115110511F441E083CF44
:10C54000D8011C92FBCF83FD7ECF03C080E090E03A
:10C5500011C00115110569F0411105C0B501C701F0
:10C5600008D9D81631F0A501B80183EC98E00E94F3
:10C57000B29AC5010F90DF91CF911F910F91FF905B
:10C58000EF90DF90CF90BF90AF9008954F925F9261
:10C590006F927F92AF92BF92CF92DF92EF92FF9213
:10C5A0000F931F93CF93DF93EC016A017B012B81E3
:10C5B000222349F08B899C89AD89BE898417950710
:10C5C000A607B70710F480E073C0223049F4CB8689
:10C5D000DC86ED86FE861F82188619861A8667C05D
:10C5E000C114D104E104F10449F41F8218861986AC
:10C5F0001A861B861C861D861E8659C08B859C85C7
:10C60000AD85BE85ED81FE81E585F0E03996AC0112
:10C61000BD0141505109610971090E2E04C0769582
:10C620006795579547950A94D2F79701860101506F
:10C6300011092109310904C03695279517950795E9
:10C64000EA95D2F7041715072607370720F0892B3C
:10C650008A2B8B2B49F48F89988DA98DBA8D8F8366
:10C660009887A987BA8704C0041B150B260B370BC4
:10C67000280139015E0187E0A80EB11C4114510464
:10C680006104710481F04F81588569857A8595012F
:10C690008D819E81BFDC91E0491A510861087108C3
:10C6A0008111ECCF05C0CB86DC86ED86FE8681E06D
:10C6B000DF91CF911F910F91FF90EF90DF90CF907E
:10C6C000BF90AF907F906F905F904F90089540E043
:10C6D00050E0BA015BCFAF92BF92CF92DF92EF9260
:10C6E000FF920F931F93CF93DF936C01A42E7901D8
:10C6F000E801FC018381823008F43DC0C601E7DF18
:10C70000B12CA895C60157DE0097B9F1FC01208134
:10C71000222399F1253011F0253E91F7FC01838504
:10C720008F738F3031F1209721F11A1414F5BA1458
:10C7300004F1088119812A813B81012B022B032BF3
:10C74000C1F4F60183859485A585B6858097A109F6
:10C75000B109FB2D40E2F40290011124821B930BDE
:10C76000A109B10988839983AA83BB83F701B082A9
:10C7700002C0B394C6CF81E001C080E0DF91CF91C9
:10C780001F910F91FF90EF90DF90CF90BF90AF90EF
:10C790000895AF92BF92CF92DF92EF92FF920F93E4
:10C7A0001F93CF93DF9300D01F92CDB7DEB78C01DC
:10C7B000FC018789908DA18DB28D89839A83AB838B
:10C7C000BC83A12CB12C49815A816B817C819E0153
:10C7D0002F5F3F4FD80115968D919C9116971ADCCB
:10C7E0008823C1F1D8011596ED91FC9116978481AB
:10C7F000A80EB11CA114B0E1BB0658F5C980DA80BF
:10C80000EB80FC808789803149F481E0E8EFCE1627
:10C81000EFEFDE06E104F10450F4D5CF81E0F8EF4C
:10C82000CF16FFEFDF06EF06FFE0FF0660F2A5017F
:10C8300060E070E099E0440F551F661F771F9A95DE
:10C84000D1F7D80153964D935D936D937C93569792
:10C8500001C080E00F900F900F900F90DF91CF916B
:10C860001F910F91FF90EF90DF90CF90BF90AF900E
:10C870000895CF93DF93EC01FB018B81882311F0A6
:10C8800080E03BC07E836D838789803101F18032F7
:10C89000B9F783E08B83428D538D648D758D4F8BFB
:10C8A000588F698F7A8FCE0174DF882349F381E036
:10C8B00089831F82188619861A861B861C861D8608
:10C8C0001E861F86188A198A1A8A1C8216C082E060
:10C8D0008B831F8A188E198E1A8E408D518D60E0C1
:10C8E00070E025E0440F551F661F771F2A95D1F78A
:10C8F0004B8B5C8B6D8B7E8BDACFDF91CF91089564
:10C900000F931F93CF93DF938C01EC01A3966623C3
:10C9100021F0D0935806C0935706F80186A18823CA
:10C9200011F0CE0161DBB8016B5F7F4FCE01DF916B
:10C93000CF911F910F919DCF8F929F92AF92BF92F7
:10C94000CF92DF92EF92FF920F931F93CF93DF93DB
:10C95000EC016A017B014801590142305105610532
:10C96000710508F44DC049855A856B857C854F5FFC
:10C970005F4F6F4F7F4F4C155D056E057F0508F4C7
:10C980003FC08F89803129F499278F2D7E2D6D2D01
:10C990000BC08032A9F5C701B60157E0969587957F
:10C9A000779567955A95D1F70B891C892D893E8912
:10C9B000600F711F821F931F43E073DA009701F12C
:10C9C0002F89203159F4DD24EE24FF24F601EE0FE7
:10C9D000FF1FE80FF91F9182808210C0E894C7F80A
:10C9E000DD24EE24FF24F601EE0FFF1FEE0FFF1FE4
:10C9F000E80FF91F80829182A282B38281E001C098
:10CA000080E0DF91CF911F910F91FF90EF90DF9029
:10CA1000CF90BF90AF909F908F9008952F923F92AC
:10CA20004F925F926F927F928F929F92AF92BF923E
:10CA3000CF92DF92EF92FF920F931F93CF93DF93EA
:10CA4000CDB7DEB72F970FB6F894DEBF0FBECDBFC0
:10CA50001C014C875D876E877F873B872A87DC01B7
:10CA600019960D911D912D913C911C970F5F1F4FB1
:10CA70002F4F3F4F0D831E832F833887EA85FB8519
:10CA800080809180A280B38081149104A104B104BC
:10CA900031F0FFEF8F1A9F0AAF0ABF0A10C0DC0106
:10CAA0008D909D90AD90BC90B1E0B9870C851D85AF
:10CAB0002E853F85013011052105310509F01986C4
:10CAC00075016401412C512C3201F101818592855F
:10CAD000A385B485481659066A067B0608F04EC041
:10CAE0000D811E812F8138850C151D052E053F05F2
:10CAF00050F472E0C72ED12CE12CF12CE2E08E2E06
:10CB0000912CA12CB12C9E012F5F3F4FB701A601A4
:10CB1000C10180DA882391F149815A816B817C813E
:10CB2000D701C6010196A11DB11D452B462B472BF0
:10CB300019F04C015D010FC0AC01BD014819590944
:10CB40006A097B090C851D852E853F854017510795
:10CB50006207730741F01FEF411A510A610A710A17
:10CB60006C017D01B2CF0FEF1FEF2FEF3FE0B70158
:10CB7000A601C101E1DE8D83811113C01D823DC07C
:10CB80002601370121E0421A510861087108970116
:10CB90008601B301A201C101CFDE882379F37301BD
:10CBA00062018C149D04AE04BF0450F3AA85BB85BA
:10CBB0004D915D916D917C91411551056105710516
:10CBC000A9F4EA85FB8580829182A282B382F985ED
:10CBD000FF2399F00FEF801A900AA00AB00AD10142
:10CBE0008D929D92AD92BC92139707C095018401DE
:10CBF000C101A2DE8111E5CFC1CF8D812F960FB685
:10CC0000F894DEBF0FBECDBFDF91CF911F910F9182
:10CC1000FF90EF90DF90CF90BF90AF909F908F905C
:10CC20007F906F905F904F903F902F900895CF939B
:10CC3000DF93EC019C01295F3F4F41E050E060E051
:10CC400070E08D819E81EADE882399F04F89588DAE
:10CC5000698D7A8D452B462B472B59F44F8158858A
:10CC600069857A854F8B588F698F7A8F9981906803
:10CC70009983DF91CF9108952F923F924F925F92C7
:10CC80006F927F928F929F92AF92BF92CF92DF92DC
:10CC9000EF92FF920F931F93CF93DF93CDB7DEB741
:10CCA00028970FB6F894DEBF0FBECDBF7C015B01A5
:10CCB0004A01DC0111968C9181FFB0C182FD02C056
:10CCC00064018DC0F701438954896589768983851C
:10CCD0009485A585B68584179507A607B70781F3C0
:10CCE000C70154DC8111ECCF99C1D70115968D9104
:10CCF0009C911697FC0134803A94B901A80129E06F
:10CD000076956795579547952A95D1F734221170F6
:10CD1000332009F470C0D70113968C9113971596A0
:10CD2000ED91FC911697823009F0A9C01B964D90A9
:10CD30005D906D907C901E9789E0769467945794EF
:10CD400047948A95D1F7828D938DA48DB58D480E29
:10CD5000591E6A1E7B1E0115110509F4AFC080E043
:10CD600092E0801B910B16018C159D0508F41C01A7
:10CD70000115110509F0A7C0F701438554856585A4
:10CD8000768583899489A589B689481759076A07E2
:10CD90007B0708F498C045E0C301B20182D8009730
:10CDA00009F43CC1A101B501800F911F0F94550CEE
:10CDB000020D131D0115124009F487C0F701838588
:10CDC0009485A585B685820D931DA11DB11D838710
:10CDD0009487A587B687A20CB31CC218D308D701C5
:10CDE0001B960D911D912D913C911E97C114D1045C
:10CDF00009F07BCFE7C00115110509F08CCF17961C
:10CE00004D915D916D917C911A9741155105610588
:10CE1000710509F19E012F5F3F4FFCD8882309F46B
:10CE2000FDC089819A81AB81BC81F7012581368162
:10CE3000F9012789203139F4883FFFEF9F07A105C9
:10CE4000B10590F416C0883F2FEF9207A2072FE09C
:10CE5000B20778F009C0F7018789908DA18DB28D56
:10CE60000097A105B10529F4C701E1DE811153CF77
:10CE7000D5C0F70187839087A187B2874CCF848183
:10CE8000D70117962D913D914D915C911A972250A3
:10CE9000310941095109A82FB0E00F944D082B0129
:10CEA0003C0186859785A089B189480E591E6A1E66
:10CEB0007B1E430C511C611C711C4DCFC114B2E090
:10CEC000DB0640F44CCF41E067CF0E94035F811145
:10CED00075CFA4C0C11424E0D206F0F480915104AF
:10CEE00090915204A0915304B09154048415950577
:10CEF000A605B70509F480D89501B301A201809178
:10CF00004A0490914B040E94395E882309F486C03C
:10CF1000212CA2E03A2E52CF848183193D2C3694E5
:10CF2000831508F4382E032D10E020E030E0B30123
:10CF3000A20180914A0490914B040E949C5E882338
:10CF400009F46CC085014D825E826F8278868D8186
:10CF50008419831548F58091510490915204A09151
:10CF60005304B09154042D813E814F815885281778
:10CF700039074A075B0709F43FD8B80180914A0492
:10CF800090914B040E947A5E1E5F2D813E814F81FD
:10CF900058852F5F3F4F4F4F5F4F2D833E834F8309
:10CFA00058878111D4CF3AC080914A0490914B04A4
:10CFB0000E94E25E882391F1232C312C322C222412
:10CFC000330CFCCE53968D919D910D90BC91A02D6C
:10CFD000F701418180179107A207B30738F4038B4B
:10CFE000148B258B368B406841830CC0809155068D
:10CFF00090915606892B31F08114910419F0406804
:10D00000F7014183D70111968C9183FD02C0C401C1
:10D010000AC0C7010E94AA5F8111F9CF81E0F70120
:10D0200080838FEF9FEF28960FB6F894DEBF0FBE78
:10D03000CDBFDF91CF911F910F91FF90EF90DF90C7
:10D04000CF90BF90AF909F908F907F906F905F90A8
:10D050004F903F902F900895AF92BF92CF92DF9262
:10D06000EF92FF920F931F93CF93DF9300D01F9205
:10D07000CDB7DEB75C016A017B0182E090E0A0E001
:10D08000B0E0F50180839183A283B3839E012F5F7B
:10D090003F4FB701A601C5010E940A60811102C07D
:10D0A00080E023C000E010E09801B701A601C501AF
:10D0B00043DC8823A9F3C980DA80EB80FC80F5018A
:10D0C0008789803149F481E0F8EFCF16FFEFDF0662
:10D0D000E104F10450F4DACF81E098EFC9169FEF34
:10D0E000D906E9069FE0F90688F20F900F900F909D
:10D0F0000F90DF91CF911F910F91FF90EF90DF90F4
:10D10000CF90BF90AF9008954F925F926F927F92B1
:10D11000AF92BF92CF92DF92EF92FF920F931F9345
:10D12000CF93DF9300D01F92CDB7DEB75C016A01C9
:10D130007B01FC0183818130E9F4818181FF1AC088
:10D14000F50183899489A589B68984179507A6076F
:10D15000B70780F0892B8A2B8B2B09F474C0F5015B
:10D160004384548465847684B701A601C5010EDA30
:10D17000811102C080E068C0F50185819681C114EB
:10D18000D104E104F10469F44789508D618D728DF9
:10D1900063DF882379F3F501178A108E118E128EC2
:10D1A00038C0F50147815085618572859E012F5FEA
:10D1B0003F4F0E940A608823E9F249815A816B81BE
:10D1C0007C81F50185819681FC012789203139F424
:10D1D000483FFFEF5F0761057105D8F407C0483F7E
:10D1E0002FEF520762072FE0720798F435DF88238C
:10D1F00009F4C0CFF50147815085618572850FEF35
:10D200001FEF2FEF3FE08581968196DB882309F49D
:10D21000B1CFF501C38AD48AE58AF68A8181806814
:10D220008183C5010E94AA5F882309F4A3CFB701B7
:10D23000A6014C145D046E047F0410F4B301A20136
:10D24000C501A4D901C081E00F900F900F900F90FD
:10D25000DF91CF911F910F91FF90EF90DF90CF90D2
:10D26000BF90AF907F906F905F904F900895BF9266
:10D27000CF92DF92EF92FF920F931F93CF93DF93A2
:10D28000EC01B42E80E2689FF0011124EB5AFB4FB1
:10D290008091510490915204A0915304B091540490
:10D2A0008F87988BA98BBA8B6C830489158920E0B2
:10D2B00030E0980111270027C28CD38CE12CF12C8F
:10D2C0000C291D292E293F290F8B188F298F3A8F62
:10D2D0008385887151F4048D158D268D378D0B8BC8
:10D2E0001C8B2D8B3E8B81E00BC08031F1F4CE0185
:10D2F00050DA811104C01B8A1C8A1D8A1E8A84E0B0
:10D300008B838B2D8F7089831F82188619861A86CE
:10D310001B861C861D861E86B4FE0AC040E050E0B7
:10D32000BA01CE01F1DE811103C01B8280E012C080
:10D33000B5FE0FC04B895C896D897E89CE01DF9176
:10D34000CF911F910F91FF90EF90DF90CF90BF9002
:10D350001DC981E0DF91CF911F910F91FF90EF9058
:10D36000DF90CF90BF900895DF92EF92FF920F93DE
:10D370001F93CF93DF938C01EB017A01D22E8D8125
:10D380009E81F801968385838381811128C020972F
:10D3900031F127FD24C0A70165E0440F551F6A95B0
:10D3A000E1F760E070E0CE01F1D88823C1F0CE0152
:10D3B00002D80097A1F0FC018081882381F0853E8E
:10D3C00071F08E3261F06E2D6F704D2DC801DF91BE
:10D3D000CF911F910F91FF90EF90DF9048CF80E0A9
:10D3E000DF91CF911F910F91FF90EF90DF90089503
:10D3F0002F923F924F925F926F927F928F929F9265
:10D40000AF92BF92CF92DF92EF92FF920F931F9352
:10D41000CF93DF93CDB7DEB7C454D1090FB6F894DC
:10D42000DEBF0FBECDBF4C017B016A01422E302E04
:10D430001EAA1FAA18AE19AEDB0115968D919C91FC
:10D440001697F40196838583CB0141D946FE1AC015
:10D45000F60101900020E9F73197EC1977247394D5
:10D46000E9300CF0712C8E2F6DE00F94BA0721E09B
:10D47000911101C020E08E2F6DE00F94BA07582E55
:10D48000520E03C055245A94712C8E010A5C1F4F12
:10D49000252D45E859E0B501C7010E940C625C01E9
:10D4A000009779F1A895D7011B968D919D910D90CC
:10D4B000BC91A02D23968CAF9DAFAEAFBFAF23978D
:10D4C000B60185E899E00E94C99A8111DECF47FE36
:10D4D00002C080E08FC123968CAD9DADAEADBFADD7
:10D4E00023974F97A109B109F5E0B695A7959795B0
:10D4F0008795FA95D1F7682F6F70442DC401B7DE78
:10D5000079C1842D8274823421F79E01265C3F4FBD
:10D51000452DFE0131965F01BF01C701DCD88EA900
:10D520009FA9A8ADB9AD892B8A2B8B2BA9F4D70164
:10D5300013962C9113971B968D919D910D90BC91F4
:10D54000A02D223009F046C18115E0E49E07A10517
:10D55000B10508F0BECF3EC122242394D701119615
:10D560008C911197826011968C934EA95FA968AD3A
:10D5700079ADC7010BD8711037C06EE270E0C601FB
:10D580000F94690C3C0186010A5F1F4F009761F000
:10D5900044E050E0BC01CE01C1960F94840C1DAA5A
:10D5A0000615170518F401C019AA38016C187D0872
:10D5B0007724A301B601CE0181960F94550CE1E2C8
:10D5C000F0E0EC0FFD1FE60DF71D10826AE073E03E
:10D5D000CE0181960F945E0CBE016F5C7F4FCE0131
:10D5E00081960F945E0C05C0B601CE0181960F9412
:10D5F0007D0CAE014F5C5F4FB501CE0181960E945C
:10D60000765BB501C4010E94B95B782EF6010190EA
:10D610000020E9F78F01015011090C191D09652C33
:10D62000252D332727FD309525963FAF2EAF259723
:10D6300011279E01215F3F4F3CAF2BAF225F3F4F31
:10D640003EAF2DAF662009F460C0862D90E0BC018E
:10D65000615071093DE0639F602D1124D501E0E226
:10D660001D92EA95E9F72FE02C8725962EAD3FAD68
:10D6700025978217930711F480E401C080E0862982
:10D68000898340E050E0FE01329670E0C601860FCB
:10D69000971F21969FAF8EAF2197CF0102969A01D7
:10D6A000260F371F0217130734F49C01AFEFBFEFAB
:10D6B000B183A0830DC09C012196AEADBFAD219773
:10D6C000A40FB51F8C91992787FD90959183808336
:10D6D000443029F04A3029F42DAD3EAD02C02BADC7
:10D6E0003CAD4F5F5F4F4D30510511F0F901D5CF83
:10D6F0007E8640E250E0B501C701BEDA97FDE9CE73
:10D70000C7010E94AA5F6A949DCF80E2F501119241
:10D710008A95E9F7AE014F5C5F4FB501CE01819666
:10D720000E94765B332011F080E101C080E28C879B
:10D7300081E298E29A8B898B20E038E0388B2F8742
:10D740009C8B8B8B9A8F898F388F2F8B40E250E088
:10D75000B501C70191DA97FDBCCEC7010E94AA5F4F
:10D7600080E2D5011D928A95E9F7222011F085EE1D
:10D770008983D12C052D112707FD10958AAD992796
:10D7800087FD9095801B910B2D2D332727FD30951C
:10D790002817390764F440E250E0B501C7016CDA9C
:10D7A00097FD97CEC7010E94AA5FD394E7CF242D9F
:10D7B0002F774EA95FA968AD79ADE5E076956795BD
:10D7C00057954795EA95D1F7400F511FB701C4010E
:10D7D000CBDD10C021E0250D2AAF0097A105B105D2
:10D7E00039F08097A109B1098EAB9FABA8AFB9AF53
:10D7F000212CB4CECC5BDF4F0FB6F894DEBF0FBE4A
:10D80000CDBFDF91CF911F910F91FF90EF90DF90EF
:10D81000CF90BF90AF909F908F907F906F905F90D0
:10D820004F903F902F900895BF92CF92DF92EF924A
:10D83000FF920F931F93CF93DF93CDB7DEB7A097DF
:10D840000FB6F894DEBF0FBECDBF7C016B01FB01AC
:10D850008381823088F101E023ECC701C9DDB82E55
:10D86000882351F18E010F5F1F4F80E2F801119262
:10D870008A95E9F721E238E23A8B298B80E098E03B
:10D88000988B8F873C8B2B8B3A8F298F988F8F8B20
:10D890008EE2898380E18C87FE013296CE010C9660
:10D8A00020E22193E817F907E1F740E250E0B801E0
:10D8B000C701E2D997FF02C0B12C37C0C7010E944F
:10D8C000AA5F8EE28A83F60183818250823028F437
:10D8D0001C8E1B8E1E8A1D8A09C0F6014789508D39
:10D8E000618D728D5C8F4B8F7E8B6D8B40E250E033
:10D8F000B801C701C1D997FDDFCFC7010E94AA5F58
:10D9000080E2F80111928A95E9F740E250E0B8010F
:10D91000C701B2D997FDD0CFC7010E94AA5F84E0AA
:10D92000F70183838181806881838B2DA0960FB658
:10D93000F894DEBF0FBECDBFDF91CF911F910F9145
:10D94000FF90EF90DF90CF90BF9008952F923F927D
:10D950004F925F926F927F928F929F92AF92BF92FF
:10D96000CF92DF92EF92FF920F931F93CF93DF93AB
:10D97000CDB7DEB7C154D1090FB6F894DEBF0FBEE4
:10D98000CDBF4B016A0139011801EFAE1E8E19A2FD
:10D9900019821C82F90110826115710511F480E071
:10D9A0008AC0FC0183818111FACFFA0180818F3214
:10D9B00061F4CA016C010196F60120812F32D1F386
:10D9C000F40183818250823010F454010CC0F401C0
:10D9D00065817681CE0101960E9439648823F9F22F
:10D9E000CE0101965C017E019EE1E90EF11CFCAEC8
:10D9F000EBAEFE013196FEAFEDAF2196EFAE219773
:10DA00002296FFAE229734C092012C193D09022FB5
:10DA1000112707FD1095A801B601C3010F94550CFD
:10DA2000F301E00FF11F1082F20181818823D9F107
:10DA300000E021E0A301B501C701DADC882309F188
:10DA4000A814B90419F0C5010E94F45F8BAD9CAD18
:10DA5000E816F90609F121969FAD219722968FAD20
:10DA600022976201EFEFCE1ADE0A5701E92EF82E57
:10DA70006FE270E0C6010F94690C2C01009721F64B
:10DA80000EC0FFADFF2309F48ACFA301B501C70182
:10DA9000CBDE8111D5CF83CF9DAD8EADE2CFB60168
:10DAA000C3010F947D0C8DE1F501D10101900D9220
:10DAB0008A95E1F781E0CF5BDF4F0FB6F894DEBFC8
:10DAC0000FBECDBFDF91CF911F910F91FF90EF90CF
:10DAD000DF90CF90BF90AF909F908F907F906F908E
:10DAE0005F904F903F902F900895CF92DF92EF92EA
:10DAF0000F931F93CF93DF93CDB7DEB7E9970FB6A0
:10DB0000F894DEBF0FBECDBF6C0119821C82E22EDD
:10DB10008E010F5F1F4F9E01225E3F4F17DF88234C
:10DB200039F0AE01425E5F4FB801C6017DDE01C033
:10DB300080E0E9960FB6F894DEBF0FBECDBFDF914F
:10DB4000CF911F910F91EF90DF90CF900895CF93D9
:10DB5000DF93CDB7DEB76D970FB6F894DEBF0FBE7B
:10DB6000CDBF242F19821C828396AB01BC01CE014C
:10DB70000196BBDF6D960FB6F894DEBF0FBECDBF2A
:10DB8000DF91CF910895CF92DF92EF92FF920F93A2
:10DB90001F93CF93DF93CDB7DEB7E9970FB6F89415
:10DBA000DEBF0FBECDBF6C01F22E19821C82E12CAC
:10DBB0008E010F5F1F4F9E01225E3F4FC7DE8823FD
:10DBC00071F08E8D882369F000E02F2DAE01425E4A
:10DBD0005F4FBE016F5F7F4FC6010ADC03C080E06C
:10DBE00001C081E0E9960FB6F894DEBF0FBECDBF4D
:10DBF000DF91CF911F910F91FF90EF90DF90CF9029
:10DC00000895FF920F931F93CF93DF93CDB7DEB7A5
:10DC10006D970FB6F894DEBF0FBECDBFFB01F42E9B
:10DC200019821C8220812F3239F42181211104C0F4
:10DC3000642F0E9480641EC08C010D5D1F4F21E087
:10DC4000AF01B801CE0101969EDF882399F09C8137
:10DC5000923078F09DE1FE013196D80101900D924D
:10DC60009A95E1F7FF2031F010935806009357067C
:10DC700001C080E06D960FB6F894DEBF0FBECDBF39
:10DC8000DF91CF911F910F91FF900895FB01242FF9
:10DC90006091570670915806AF0175CFCF93DF930F
:10DCA000EC0140E050E0BA012FDA882371F061E026
:10DCB000CE010E94935F009741F025EEFC01208386
:10DCC0001B82DF91CF910C94035F80E0DF91CF91B5
:10DCD0000895CF93DF93CDB7DEB76D970FB6F89465
:10DCE000DEBF0FBECDBFAB0119821C8222E0BC019A
:10DCF000CE01019648DF882319F0CE010196CEDFD0
:10DD00006D960FB6F894DEBF0FBECDBFDF91CF91F9
:10DD100008958396DECF0F931F93CF93DF93EC018B
:10DD20008B81843061F5CE010E9467630B851C8571
:10DD30002D853E854B895C896D897E890417150781
:10DD40002607370748F4CE010E94DB610097B9F03F
:10DD5000FC01208121110BC081E08B8389818260CD
:10DD60008983CE01DF91CF911F910F9197CF253EEF
:10DD7000E9F22E32D9F2FC01838583FDD7CF80E012
:10DD8000DF91CF911F910F910895CF93DF93CDB77E
:10DD9000DEB76D970FB6F894DEBF0FBECDBF198208
:10DDA0001C8241E0CE01019671DF882319F0CE017B
:10DDB0000196B1DF6D960FB6F894DEBF0FBECDBFF2
:10DDC000DF91CF9108954F925F926F927F92AF92C1
:10DDD000BF92CF92DF92EF92FF920F931F93CF9358
:10DDE000DF93EC01142F70934B0460934A041F8A55
:10DDF00082E090E0A0E0B0E088839983AA83BB83AF
:10DE0000109250048FEF9FEFDC01809351049093A8
:10DE10005204A0935304B093540410924C041092F3
:10DE20004D0410924E0410924F04442361F145308A
:10DE300008F0D6C040E060E070E0CB010E94515F86
:10DE4000009709F4CDC0FC0120E1129FE00DF11D07
:10DE50001124E255FE4F80818F7709F0C1C04485BF
:10DE6000558566857785443651056105710508F449
:10DE7000B7C0C084D184E284F384C114D104E10426
:10DE8000F10421F4ADC0C12CD12C760140E0C701D2
:10DE9000B6010E94515FFC01009709F4A1C083857F
:10DEA00094858115924009F09BC02089222309F4B2
:10DEB00097C086859785892B09F492C0858588232C
:10DEC00009F48EC02A8B25852C831D8630E041E025
:10DED00050E06D85062FCA01062E02C0880F991FDB
:10DEE0000A94E2F72817390731F081E0860F8D8711
:10DEF000683078F375C0268937892115310519F006
:10DF000040E050E004C024A135A146A157A12D83D3
:10DF10003E834F83588720934C0430934D044093A5
:10DF20004E0450934F048685978526013701480E8D
:10DF3000591E611C711C4B8A5C8A6D8A7E8AA1887D
:10DF4000B288B98EA88EA089B0E00F944D08640DF8
:10DF5000751D861D971D6A8F7B8F8C8F9D8F15E099
:10DF6000AA0CBB1C1A95E1F741E0A41A4EEFB40AC3
:10DF7000AB2CBB24A694DC01CB018A0D9B1DA11DFB
:10DF8000B11D8E879F87A88BB98B43885488411415
:10DF9000510419F0612C712C04C040A051A062A062
:10DFA00073A0A7019601281B390B4A0B5B0BDA0102
:10DFB000C901840D951DA61DB71D04C0B695A79572
:10DFC000979587950A95D2F789879A87AB87BC87FB
:10DFD000853F3FE09307A105B10520F48CE08F8BCE
:10DFE00080E012C0853F9F4FA105B10510F480E18C
:10DFF00009C084A595A5A6A5B7A58A8F9B8FAC8FD0
:10E00000BD8F80E28F8B81E0DF91CF911F910F91C7
:10E01000FF90EF90DF90CF90BF90AF907F906F9088
:10E020005F904F9008950F931F93CF93DF93EC0170
:10E03000842F462F682FCE010E94DC5C8823B9F024
:10E040008E010B5F1F4F41E0BE01C801BCDE88237B
:10E0500041F061E0CE01DF91CF911F910F910C94BF
:10E06000806440E0BE01C801AEDE8111F2CF80E0E5
:10E07000DF91CF911F910F9108950C943C66682F0A
:10E080008AED9AE00C9429D42F923F924F925F929E
:10E090006F927F928F929F92AF92BF92CF92DF92B8
:10E0A000EF92FF920F931F93CF93DF93CDB7DEB71D
:10E0B0006D970FB6F894DEBF0FBECDBF7B01342E37
:10E0C00059014801CB010E946763C12CD12C222445
:10E0D0002394230C00E010E020E045E859E0B6016D
:10E0E000C7010E940C626C01009739F0A895D60117
:10E0F0001B961C9113FF03C0EDCF80E0C2C06FE000
:10E1000073E085E899E00F94740C892B19F318716A
:10E11000103109F067C0B1E0B315E0F2A114B10409
:10E1200091F4332041F08CE499E00E94189D8DED2C
:10E1300092E20E94D49C85E899E00E94189D8DEDA2
:10E1400092E20E94ED9C19821C82332031F06DE036
:10E1500073E08CE499E00F945E0C65E879E08CE460
:10E1600099E00F945E0CF7014384548465847684AF
:10E17000FFE14F1A51086108710845E076946794F1
:10E18000579447944A95D1F721E0A201B701CE01F7
:10E190000196EAD8882351F084019501422DBE01F1
:10E1A0006F5F7F4FCB0170DF81116AC08FEF481A1C
:10E1B000580A35E0440C551C3A95E1F7A20160E09D
:10E1C00070E0C7010E94C6626FE270E08CE499E0E3
:10E1D0000F94930C009719F0DC011C927BCF1092E6
:10E1E0004C0978CFA114B10489F1ECE4F9E0DF0126
:10E1F0000D900020E9F78D01015011090C541940D0
:10E20000702E402F552747FD5095B501CF010E9434
:10E21000069B81115FCF10161CF477247394700E47
:10E22000B501670D711D77FC7A9585E899E00E942C
:10E23000C99A81114FCF8114910411F18DE1F70139
:10E24000D40101900D928A95E1F71AC0332041F074
:10E250008CE499E00E94189D8DED92E20E94D49C7E
:10E2600085E899E00E94189DF601448D558D668DD4
:10E27000778D8CE692E20E94F89D0E9414232ACFAB
:10E2800081E06D960FB6F894DEBF0FBECDBFDF9173
:10E29000CF911F910F91FF90EF90DF90CF90BF90A3
:10E2A000AF909F908F907F906F905F904F903F9036
:10E2B0002F900895EF92FF920F931F93CF93DF93C8
:10E2C000CDB7DEB76D970FB6F894DEBF0FBECDBFEA
:10E2D0007C0119821C820E946763ECE4F9E01082E1
:10E2E000D7015C96FC93EE935B978DE1F701DE011D
:10E2F000119601900D928A95E1F700E010E020E080
:10E3000030E040E0BE016F5F7F4FC701BDDE6D961C
:10E310000FB6F894DEBF0FBECDBFDF91CF911F9136
:10E320000F91FF90EF900895882321F080910B01C9
:10E330008D7F03C080910B01826080930B01089553
:10E34000882321F080910B018E7F03C080910B0107
:10E35000816080930B010895882321F080910B0147
:10E360008B7F03C080910B01846080930B01089523
:10E37000FB01DC018091F207882349F023E333E3BA
:10E380004BEC51E4CD010F94E406FB01DC01BF012D
:10E39000CD010895CF93DF931F92CDB7DEB7909153
:10E3A000690790FF02C081113FC02091680723FDDB
:10E3B0003BC0916090936907179A169A159A8983C2
:10E3C0000E94D24F8981811121C020E040E060E0AD
:10E3D00070E0CB010E94385340E060E070E0CB0178
:10E3E0000E94BE4F40E068ED76E187E19AE00E942E
:10E3F000CBA887E19AE00E941FAC9B9AA39A8091D8
:10E4000068078F7B8860809368070EC040E067ECE8
:10E4100076E187E19AE00E94CBA887E19AE00F902D
:10E42000DF91CF910C941FAC0F90DF91CF910895A5
:10E43000CF93C0916907CD7FC093690720E030E09A
:10E44000A901609131027091320280913302909162
:10E4500034020F943C04882319F0C260C09369070A
:10E46000CF9108952F923F924F925F926F927F9239
:10E470008F929F92AF92BF92CF92DF92EF92FF92D4
:10E480000F931F93CF93DF93CDB7DEB76D970FB682
:10E49000F894DEBF0FBECDBF8BE793E00F94BB0CAB
:10E4A0009093EF068093EE0689E793E00F94BB0C00
:10E4B0009093ED068093EC06C090E002D090E102CC
:10E4C000E090E202F090E302C092DC02D092DD0222
:10E4D000E092DE02F092DF02C092D802D092D9021E
:10E4E000E092DA02F092DB028091B4029091B502E0
:10E4F000A091B602B091B7028093B0029093B1029E
:10E50000A093B202B093B3028093AC029093AD0299
:10E51000A093AE02B093AF028091C4029091C50265
:10E52000A091C602B091C7028093C0029093C1022D
:10E53000A093C202B093C3028093BC029093BD0229
:10E54000A093BE02B093BF028091D0029091D102FD
:10E55000A091D202B091D3028093CC029093CD02CD
:10E56000A093CE02B093CF028093C8029093C902C9
:10E57000A093CA02B093CB028091A4029091A5020D
:10E58000A091A602B091A7028093A0029093A1024D
:10E59000A093A202B093A30280939C0290939D0249
:10E5A000A0939E02B0939F022091AC063091AD06DD
:10E5B0004091AE065091AF06C701B6010F94E40634
:10E5C0000F94DC046093CC067093CD068093CE0646
:10E5D0009093CF062091B8063091B9064091BA06C3
:10E5E0005091BB06C701B6010F94E4060F94DC04FA
:10E5F0006093C8067093C9068093CA069093CB06B1
:10E600002091B0063091B1064091B2065091B30608
:10E61000C701B6010F94E4060F94DC046093C406AE
:10E620007093C5068093C6069093C7062091A806EE
:10E630003091A9064091AA065091AB06C701B601D8
:10E640000F94E4060F94DC046093C0067093C10637
:10E650008093C2069093C306C0901807D090190704
:10E66000E0901A07F0901B0781E993E00E94701C6C
:10E670009B01AC01C701B6010F94D8032B013C01EB
:10E68000C0901807D0901907E0901A07F0901B0768
:10E6900085E993E00E94701C9B01AC01C701B601A3
:10E6A0000F94D8034B015C01C0901807D090190754
:10E6B000E0901A07F0901B0789E993E00E94701C14
:10E6C0009B01AC01C701B6010F94D8036B017C011B
:10E6D00085E893E00E94701C2BED3FE049E450E494
:10E6E0000F94E40620E030E044E353E40F94430445
:10E6F0000F9440049B01AC01C301B2010F94E406E6
:10E700002091E0023091E1024091E2025091E30257
:10E710000F94E40620E030E040E05FE30F94D8037C
:10E720000F944A050F94DC0460931007709311074F
:10E73000809312079093130785E893E00E94701C62
:10E740002BED3FE049E450E40F94E40620E030E094
:10E7500044E353E40F9443040F9447079B01AC0137
:10E76000C301B2010F94E4062091E0023091E1026E
:10E770004091E2025091E3020F94E40620E030E081
:10E7800040E05FE30F94D8030F944A050F94DC0434
:10E7900060930C0770930D0780930E0790930F07FB
:10E7A00089E893E00E94701C2BED3FE049E450E4BF
:10E7B0000F94E40620E030E044E353E40F94430474
:10E7C0000F9440049B01AC01C501B4010F94E40611
:10E7D0002091E0023091E1024091E2025091E30287
:10E7E0000F94E40620E030E040E05FE30F94D803AC
:10E7F0000F944A050F94DC0460930807709309078F
:10E8000080930A0790930B0789E893E00E94701C9D
:10E810002BED3FE049E450E40F94E40620E030E0C3
:10E8200044E353E40F9443040F9447079B01AC0166
:10E83000C501B4010F94E4062091E0023091E10299
:10E840004091E2025091E3020F94E40620E030E0B0
:10E8500040E05FE30F94D8030F944A050F94DC0463
:10E86000609304077093050780930607909307074A
:10E870008DE893E00E94701C2BED3FE049E450E4EA
:10E880000F94E40620E030E044E353E40F944304A3
:10E890000F9440049B01AC01C701B6010F94E4063C
:10E8A0002091E0023091E1024091E2025091E302B6
:10E8B0000F94E40620E030E040E05FE30F94D803DB
:10E8C0000F944A050F94DC046093000770930107CE
:10E8D00080930207909303078DE893E00E94701CD9
:10E8E0002BED3FE049E450E40F94E40620E030E0F3
:10E8F00044E353E40F9443040F9447079B01AC0196
:10E90000C701B6010F94E4062091E0023091E102C4
:10E910004091E2025091E3020F94E40620E030E0DF
:10E9200040E05FE30F94D8030F944A050F94DC0492
:10E930006093FC067093FD068093FE069093FF069D
:10E9400085EA93E00E94701C6B017C0181E793E0F3
:10E950000E94701C9B01AC01C701B6010F94D80343
:10E960002091E0023091E1024091E2025091E302F5
:10E970000F94E4060F94E10460932807709329072D
:10E9800080932A0790932B0789EA93E00E94701CDA
:10E990006B017C0181E793E00E94701C9B01AC013C
:10E9A000C701B6010F94D8032091E0023091E10233
:10E9B0004091E2025091E3020F94E4060F94E104C7
:10E9C0006093240770932507809326079093270769
:10E9D0008DEA93E00E94701C6B017C0181E793E05B
:10E9E0000E94701C9B01AC014090E0025090E1023B
:10E9F0006090E2027090E302C701B6010F94D80361
:10EA0000A30192010F94E4060F94E1044B015C0111
:10EA1000C0902807D0902907E0902A07F0902B0794
:10EA2000109169078FEFC816D806E104F104C0F40D
:10EA3000609118077091190780911A0790911B0730
:10EA40009B01AC010F94D803A30192010F94E4063B
:10EA500020E03EEF4FE757E40F9470061816D4F508
:10EA6000106810936907C701B6010F940D059B014B
:10EA7000AC010F94E40660932807709329078093F4
:10EA80002A0790932B0760912407709125078091A6
:10EA90002607909127070F940D059B01AC010F9459
:10EAA000E4066093240770932507809326079093CC
:10EAB0002707C501B4010F940D059B01AC010F940C
:10EAC000E4066093200770932107809322079093B8
:10EAD000230733C01F7710936907A7019601C70169
:10EAE000B6010F94AB0760932807709329078093B2
:10EAF0002A0790932B076091240770912507809136
:10EB00002607909127079B01AC010F94AB076093F8
:10EB10002407709325078093260790932707A50164
:10EB20009401C501B4010F94AB0760932007709363
:10EB3000210780932207909323078DE993E00E9499
:10EB4000701C9B01AC010F94E40660931C0770934A
:10EB50001D0780931E0790931F07198A1A8A1B8A24
:10EB60001C8A1D861E861F86188A8091CC0690916D
:10EB7000CD06A091CE06B091CF068D8B9E8BAF8B2C
:10EB8000B88FBE016F5F7F4FCE010D960E9480E768
:10EB900089819A81AB81BC8180932C0790932D074A
:10EBA000A0932E07B0932F078091CC069091CD06AD
:10EBB000A091CE06B091CF068093D0069093D10657
:10EBC000A093D206B093D3068093D4069093D50633
:10EBD000A093D606B093D7061092C0061092C10635
:10EBE0001092C2061092C3061092C4061092C50677
:10EBF0001092C6061092C7061092C8061092C90657
:10EC00001092CA061092CB064090E0025090E102AA
:10EC10006090E2027090E30220E030E040E751E4CF
:10EC2000C301B2010F94E4060F94DC04609314074F
:10EC300070931507809316079093170788ED882E19
:10EC400082E0982E92EEA92E97E0B92E0CEA12E0FF
:10EC500022ED222E27E0322EECE9F2E0FD8FEC8F40
:10EC600082EC97E09B8F8A8F198EF401C190D1902E
:10EC7000E190F1904F01A701960160E070E080E81B
:10EC80009FE30F944304F5016193719381939193F2
:10EC90005F01F80161917191819191918F01A701BB
:10ECA00096010F94E4060F94E104F10161937193CE
:10ECB000819391931F01EC8DFD8D619171918191F3
:10ECC0009191FD8FEC8FA70196010F94E4060F94AC
:10ECD000E104EA8DFB8D6193719381939193FB8F96
:10ECE000EA8FF98DFF5FF98FF43009F0BECFA09065
:10ECF0009C02B0909D02C0909E02D0909F02E09036
:10ED0000AC02F090AD020091AE021091AF029501FD
:10ED1000A601B701C8010F943C0487FF02C075012A
:10ED200086012091D8023091D9024091DA025091A7
:10ED3000DB02B701C8010F94E4069B01AC0160E05F
:10ED400070E080E090E40F9443040F9451079B011E
:10ED5000AC01B701C8010F94E4066093DC06709320
:10ED6000DD068093DE069093DF06A090A402B090AB
:10ED7000A502C090A602D090A702E090B402F09045
:10ED8000B5020091B6021091B7029501A601B70134
:10ED9000C8010F943C0487FF02C0750186019701EA
:10EDA000A801C301B2010F94E4069B01AC0160E02D
:10EDB00070E080E090E40F9443040F9451079B01AE
:10EDC000AC01B701C8010F94E4066093D8067093B4
:10EDD000D9068093DA069093DB062ADB6D960FB690
:10EDE000F894DEBF0FBECDBFDF91CF911F910F9181
:10EDF000FF90EF90DF90CF90BF90AF909F908F905B
:10EE00007F906F905F904F903F902F900895EF927A
:10EE1000FF920F931F9360936A0770936B07809321
:10EE20006C0790936D0720936E0730936F074093A4
:10EE3000700750937107E0927207F0927307009386
:10EE40007407109375071F910F91FF90EF9008952D
:10EE5000CF92DF92EF92FF9281E00E943F1D87E107
:10EE60009AE00E94C5C50E9473FE2091CC0B21112F
:10EE700048C02091660722FD44C0C0902C1DD09050
:10EE80002D1DE0902E1DF0902F1D9B01AC012C1923
:10EE90003D094E095F0969017A018091F302909161
:10EEA000F402A091F502B091F6020097A105B10518
:10EEB00041F08C159D05AE05BF0518F480E06ADAB7
:10EEC00005C080916807877F809368078091EF0273
:10EED0009091F002A091F102B091F2020097A10589
:10EEE000B10539F08C159D05AE05BF0510F481E024
:10EEF00051DA83EC98E0FF90EF90DF90CF900C9484
:10EF0000469860932C1D70932D1D80932E1D909319
:10EF10002F1DEFCFAF92BF92CF92DF92EF92FF9271
:10EF20000F931F93CF93DF93EB01D82EC92E10922E
:10EF30009E0710929F071092A0071092A1071092AF
:10EF4000A2071092A3071092A4071092A50710928F
:10EF5000A6071092A7071092A8071092A90762EBC4
:10EF600077E08EE997E00E9480E76091CC0670918F
:10EF7000CD068091CE069091CF060F940F0520E02C
:10EF800030E040EC5FE30F94E4060F94DC047B0177
:10EF90008C0121E02F932F93CF92DF92DF93CF93B9
:10EFA000A12CB12C650120E030E0A90160E070E007
:10EFB000CB010E9494F2109298061092990610923A
:10EFC0009A0610929B061092940610929506109243
:10EFD0009606109297060F900F900F900F900F903B
:10EFE0000F90DF91CF911F910F91FF90EF90DF90E5
:10EFF000CF90BF90AF9008954F925F926F927F92A3
:10F000008F929F92AF92BF92CF92DF92EF92FF9238
:10F010000F931F93CF93DF9300D01F92CDB7DEB72E
:10F020006091C4027091C5028091C6029091C7029E
:10F0300071DF6091E0027091E1028091E2029091B3
:10F04000E3029B01AC010F94D80320E030E040EADA
:10F0500050EC0F94E4060F94DC042B013C011F924A
:10F06000992493949F9220E030E040E05FE3609128
:10F07000C4027091C5028091C6029091C7020F949C
:10F08000E4069F938F937F936F93A12CB12C65011E
:10F090008301720120E030E0A90160E070E0CB0163
:10F0A0000E9494F220E030E040E05FE36091C4020F
:10F0B0007091C5028091C6029091C7020F94E40638
:10F0C00029DF20E030E040EA50EC6091E0027091EE
:10F0D000E1028091E2029091E3020F94E4060F9422
:10F0E000DC041F929F922091C7022F932091C602A9
:10F0F0002F932091C5022F932091C4022F937B015F
:10F100008C0120E030E0A90160E070E0CB010E94BA
:10F1100094F28DE793E00F94BB0C8090C80690901A
:10F12000C906A090CA06B090CB06B094A094909463
:10F130008094811C911CA11CB11CAA2797FDA0954D
:10F14000BA2F881A990AAA0ABB0A8FE793E00F948C
:10F15000BB0CC090C406D090C506E090C606F090E7
:10F16000C706F094E094D094C094C11CD11CE11C5B
:10F17000F11CAA2797FDA095BA2FC81AD90AEA0A46
:10F18000FB0A81E893E00F94BB0C4091C0065091BC
:10F19000C1066091C2067091C30670956095509546
:10F1A00041955F4F6F4F7F4FAA2797FDA095BA2FCC
:10F1B000481B590B6A0B7B0B0FB6F894DEBF0FBED2
:10F1C000CDBF2A013B018C149D04AE04BF0444F45E
:10F1D00084169506A606B70654F42401350107C027
:10F1E000C416D506E606F70614F42601370184187E
:10F1F0009508A608B708C418D508E608F708DB0183
:10F20000CA0184199509A609B70989839A83AB8332
:10F21000BC8310929E0710929F071092A007109235
:10F22000A1071092A2071092A3071092A4071092B0
:10F23000A5078091CC069091CD06A091CE06B09105
:10F24000CF068093A6079093A707A093A807B09333
:10F25000A90762EB77E08EE997E00E9480E7809152
:10F26000B2079091B307A091B407B091B507881980
:10F270009909AA09BB098093B2079093B307A09399
:10F28000B407B093B5078091B6079091B707A091E6
:10F29000B807B091B9078C199D09AE09BF098093D1
:10F2A000B6079093B707A093B807B093B9078091BA
:10F2B000BA079091BB07A091BC07B091BD07298107
:10F2C0003A814B815C81821B930BA40BB50B80931D
:10F2D000BA079093BB07A093BC07B093BD071F92DA
:10F2E00081E08F938091C7028F938091C6028F93A4
:10F2F0008091C5028F938091C4028F93A12CB12C71
:10F3000065018301720120E030E0A90160E070E056
:10F31000CB010E9494F210929E0710929F071092C8
:10F32000A0071092A1071092A2071092A3071092B3
:10F33000A4071092A5078091CC069091CD06A091CC
:10F34000CE06B091CF068093A6079093A707A0930F
:10F35000A807B093A90710926A0710926B07109242
:10F360006C0710926D0710926E0710926F07109243
:10F370007007109271071092720710927307109223
:10F3800074071092750762EB77E08EE997E00E94B0
:10F3900080E78091B2079091B307A091B407B09134
:10F3A000B5078093F0069093F106A093F206B09310
:10F3B000F3068091B6079091B707A091B807B09176
:10F3C000B9078093F4069093F506A093F606B093E0
:10F3D000F7068091BA079091BB07A091BC07B09146
:10F3E000BD078093F8069093F906A093FA06B093B0
:10F3F000FB0660912C0770912D0780912E0790914C
:10F400002F070F940F056B017C0120E030E040EAEC
:10F4100050E46091E0027091E1028091E2029091EB
:10F42000E3020F94E4069B01AC01C701B6010F94FF
:10F43000D8030F94DC0460932C0770932D078093FE
:10F440002E0790932F070F900F900F900F900F9013
:10F450000F90E0913603F091370380810F900F9069
:10F460000F900F90DF91CF911F910F91FF90EF9030
:10F47000DF90CF90BF90AF909F908F907F906F90D4
:10F480005F904F900C94044E0F931F93CF93DF9394
:10F490008091B007C1E018161CF0C0E08F5F01C07A
:10F4A00081508093B0071798169815988091690736
:10F4B0008E7F809369070091090110910901D09115
:10F4C00009018C2F0E9494718C2F0E94A0718C2FA7
:10F4D0000E94AC7181E090E00E94C7FE409A419A80
:10F4E000429A82E090E00E94C7FE4098419842987C
:10F4F000C1E001FB882780F98C270E949471812F3D
:10F5000081708C270E94A071D2FB882780F98C27FC
:10F51000DF91CF911F910F910C94AC714F925F923C
:10F520006F927F928F929F92AF92BF92CF92DF9213
:10F53000EF92FF920F931F93CF93DF93CDB7DEB778
:10F5400028970FB6F894DEBF0FBECDBF2B013C014C
:10F5500029833A834B835C83ED82FE820F83188775
:10F560008501740120913E0730913F07409140078B
:10F57000509141070F94E4064B015C0120914A072A
:10F5800030914B0740914C0750914D0769817A812A
:10F590008B819C810F94E4069B01AC01C501B401F1
:10F5A0000F94D8034B015C01209156073091570707
:10F5B00040915807509159076D817E818F819885C0
:10F5C0000F94E4069B01AC01C501B4010F94D8036C
:10F5D000F601608371838283938320914207309187
:10F5E00043074091440750914507C301B2010F946E
:10F5F000E4064B015C0120914E0730914F0740918A
:10F6000050075091510769817A818B819C810F94B9
:10F61000E4069B01AC01C501B4010F94D8034B0172
:10F620005C0120915A0730915B0740915C07509133
:10F630005D076D817E818F8198850F94E4069B0123
:10F64000AC01C501B4010F94D803F8016083718344
:10F650008283938320914607309147074091480762
:10F6600050914907C301B2010F94E4064B015C01BC
:10F6700020915207309153074091540750915507FC
:10F6800069817A818B819C810F94E4069B01AC0196
:10F69000C501B4010F94D8034B015C0120915E07B2
:10F6A00030915F0740916007509161076D817E81C5
:10F6B0008F8198850F94E4069B01AC01C501B401CC
:10F6C0000F94D803F7016083718382839383289614
:10F6D0000FB6F894DEBF0FBECDBFDF91CF911F9163
:10F6E0000F91FF90EF90DF90CF90BF90AF909F90E1
:10F6F0008F907F906F905F904F9008954F925F92A0
:10F700006F927F928F929F92AF92BF92CF92DF9231
:10F71000EF92FF920F931F93CF93DF93CDB7DEB796
:10F7200064970FB6F894DEBF0FBECDBF69837A83AE
:10F730008B839C832D833E834F835887E986FA868B
:10F740000B871C8725013601E62EF72E082F192F6F
:10F7500020EF33E244E759E4B701C8010F943C04B9
:10F7600081110DC08091920790919307A091940709
:10F77000B091950789839A83AB83BC830AC0C70184
:10F78000D8018093920790939307A0939407B09326
:10F790009507CD80DE80EF80F88420EF33E244E7E8
:10F7A00059E4C701B6010F943C0481110DC080914A
:10F7B000960790919707A0919807B09199078D832C
:10F7C0009E83AF83B88708C0C0929607D0929707F0
:10F7D000E0929807F0929907C984DA84EB84FC845C
:10F7E00020EF33E244E759E4C701B6010F943C042B
:10F7F00081110DC080919A0790919B07A0919C0761
:10F80000B0919D0789879A87AB87BC8708C0C09253
:10F810009A07D0929B07E0929C07F0929D078091F7
:10F82000690785FF3DC029853A854B855C852D8715
:10F830003E874F87588B20919406309195064091D2
:10F840009606509197066D817E818F8198850F94E1
:10F85000D803698B7A8B8B8B9C8B20919806309187
:10F86000990640919A0650919B0669817A818B8115
:10F870009C810F94D803AE01475F5F4F4A01DE01C0
:10F8800015965D019E012F5F3F4F6901ED84FE8457
:10F890000F85188929893A894B895C893FDE24C004
:10F8A000209198063091990640919A0650919B06B6
:10F8B00069817A818B819C810F94D80369837A83D3
:10F8C0008B839C83209194063091950640919606F7
:10F8D000509197066D817E818F8198850F94D80312
:10F8E0006D837E838F8398872091D8023091D902CF
:10F8F0004091DA025091DB0269817A818B819C818F
:10F900000F94E40620E030E040E05FE30F94D8037A
:10F910000F944A050F94DC04609376077093770781
:10F9200080937807909379072091DC023091DD0273
:10F930004091DE025091DF026D817E818F8198853A
:10F940000F94E40620E030E040E05FE30F94D8033A
:10F950000F944A050F94DC0460937A0770937B0739
:10F9600080937C0790937D072091E0023091E10223
:10F970004091E2025091E30269857A858B859C85EE
:10F980000F94E40620E030E040E05FE30F94D803FA
:10F990000F944A050F94DC0460937E0770937F07F1
:10F9A000809380079093810720EF33E244E759E486
:10F9B000C301B2010F943C048823C1F080919B02E3
:10F9C00083FD14C0E0913603F091370320E030E06E
:10F9D00046E153E462A973A984A995A90F9470061E
:10F9E00018165CF18091680787FD27C020EF33E28D
:10F9F00044E759E468A579A58AA59BA50F943C0422
:10FA0000882361F088A599A5AAA5BBA58093A40623
:10FA10009093A506A093A606B093A70641E061E0E7
:10FA200081E00E9464ED811106C087E796E10E94A3
:10FA3000FA9C80E019C081E017C02091E402309167
:10FA4000E5024091E6025091E702C301B2010F9432
:10FA5000E4060F94DC04609382077093830780931D
:10FA6000840790938507C2CF64960FB6F894DEBFE3
:10FA70000FBECDBFDF91CF911F910F91FF90EF90FF
:10FA8000DF90CF90BF90AF909F908F907F906F90BE
:10FA90005F904F9008954F925F926F927F928F92F6
:10FAA0009F92AF92BF92CF92DF92EF92FF920F930D
:10FAB0001F93CF93DF93CDB7DEB728970FB6F89497
:10FAC000DEBF0FBECDBF2B013C0129833A834B83A0
:10FAD0005C83ED82FE820F8318878501740120917B
:10FAE0003E0730913F0740914007509141070F94E6
:10FAF000E4064B015C01209142073091430740919D
:10FB000044075091450769817A818B819C810F94CC
:10FB1000E4069B01AC01C501B4010F94D8034B016D
:10FB20005C0120914607309147074091480750916A
:10FB300049076D817E818F8198850F94E4069B0132
:10FB4000AC01C501B4010F94D803F6016083718341
:10FB50008283938320914A0730914B0740914C0751
:10FB600050914D07C301B2010F94E4064B015C01B3
:10FB700020914E0730914F07409150075091510707
:10FB800069817A818B819C810F94E4069B01AC0191
:10FB9000C501B4010F94D8034B015C0120915207B9
:10FBA0003091530740915407509155076D817E81E4
:10FBB0008F8198850F94E4069B01AC01C501B401C7
:10FBC0000F94D803F801608371838283938320911B
:10FBD0005607309157074091580750915907C30174
:10FBE000B2010F94E4064B015C0120915A07309159
:10FBF0005B0740915C0750915D0769817A818B8139
:10FC00009C810F94E4069B01AC01C501B4010F94E3
:10FC1000D8034B015C0120915E0730915F07409152
:10FC20006007509161076D817E818F8198850F9467
:10FC3000E4069B01AC01C501B4010F94D803F701A0
:10FC4000608371838283938328960FB6F894DEBF16
:10FC50000FBECDBFDF91CF911F910F91FF90EF901D
:10FC6000DF90CF90BF90AF909F908F907F906F90DC
:10FC70005F904F9008953F924F925F926F927F9264
:10FC80008F929F92AF92BF92CF92DF92EF92FF92AC
:10FC90000F931F93CF93DF9300D01F92CDB7DEB7A2
:10FCA000382E60919E0770919F078091A0079091D8
:10FCB000A1070F940F052091E2073091E3074091CF
:10FCC000E4075091E5070F94E4062B013C01609393
:10FCD0009207709393078093940790939507609190
:10FCE000A2077091A3078091A4079091A5070F9494
:10FCF0000F052091E6073091E7074091E807509102
:10FD0000E9070F94E40669837A838B839C8360936D
:10FD1000960770939707809398079093990760913F
:10FD2000A6077091A7078091A8079091A9070F9443
:10FD30000F052091EA073091EB074091EC075091B5
:10FD4000ED070F94E40660939A0770939B078093E6
:10FD50009C0790939D072091690725FF15C04AE9EC
:10FD6000842E47E0942E56E9A52E57E0B52EE2E901
:10FD7000CE2EE7E0DE2E7B018C0129813A814B817A
:10FD80005C81C301B20187DE20919806309199060B
:10FD900040919A0650919B0660919207709193074B
:10FDA00080919407909195070F94D7032B013C0104
:10FDB00060939207709393078093940790939507AD
:10FDC00020919406309195064091960650919706A1
:10FDD0006091960770919707809198079091990785
:10FDE0000F94D703609396077093970780939807B3
:10FDF00090939907332001F140928607509287072C
:10FE0000609288077092890760938A0770938B07C6
:10FE100080938C0790938D0780919A0790919B0710
:10FE2000A0919C07B0919D0780938E0790938F07B8
:10FE3000A0939007B09391070F900F900F900F90A1
:10FE4000DF91CF911F910F91FF90EF90DF90CF90B6
:10FE5000BF90AF909F908F907F906F905F904F90EA
:10FE60003F9008954F925F926F927F928F929F92F0
:10FE7000AF92BF92CF92DF92EF92FF920F931F93B8
:10FE8000CF93DF932B013C0149015A0167017801AF
:10FE90008091680785FD53C020E030E048EC52ECCB
:10FEA000C701B6010F94700687FD1DC02DEC3CEC18
:10FEB0004CE45DE36091AC067091AD068091AE06B6
:10FEC0009091AF060F94D80320E030E040EA50E470
:10FED0000F94D8039B01AC01C1E0C701B6010F9498
:10FEE0003C0418160CF4C0E0A3019201C301B20156
:10FEF0000F94E4066B017C01A5019401C501B401D6
:10FF00000F94E4069B01AC01C701B6010F94D8031E
:10FF1000D1E020911C0730911D0740911E075091A0
:10FF20001F070F943C0418160CF4D0E0CD2341F4C5
:10FF300081E0A1DE8FED96E10E946F1D01C0C1E05E
:10FF40008C2FDF91CF911F910F91FF90EF90DF9059
:10FF5000CF90BF90AF909F908F907F906F905F9069
:10FF60004F9008952F923F924F925F926F927F929F
:10FF70008F929F92AF92BF92CF92DF92EF92FF92B9
:10FF80000F931F93CF93DF93CDB7DEB760970FB674
:10FF9000F894DEBF0FBECDBF1C018091AF07F10109
:10FFA0001081811169C013FF20C06285738584852B
:10FFB00095850E94B87120916A0730916B07409136
:10FFC0006C0750916D070F94D7036093920770935D
:10FFD0009307809394079093950760938607709397
:10FFE0008707809388079093890714FF21C0F10148
:10FFF00066857785808991890E94B87120916E0706
:020000021000EC
:1000000030916F0740917007509171070F94D7039B
:10001000609396077093970780939807909399073A
:1000200060938A0770938B0780938C0790938D075A
:1000300015FF8BC0F10162897389848995890E94BB
:10004000B8712091720730917307409174075091F5
:1000500075070F94D70360939A0770939B0780935B
:100060009C0790939D0760938E0770938F078093F2
:1000700090079093910769C013FF21C0F101628539
:100080007385848595850E94B8712091860730918B
:10009000870740918807509189070F94D803609390
:1000A00086077093870780938807909389076093EA
:1000B000920770939307809394079093950714FF8A
:1000C00021C0F10166857785808991890E94B87188
:1000D00020918A0730918B0740918C0750918D07B2
:1000E0000F94D80360938A0770938B0780938C07D3
:1000F00090938D0760939607709397078093980766
:100100009093990715FF21C0F10162897389848951
:1001100095890E94B87120918E0730918F07409188
:100120009007509191070F94D80360938E077093B6
:100130008F07809390079093910760939A0770932D
:100140009B0780939C0790939D078091690740903F
:100150008E0750908F07609090077090910785FFF1
:100160003BC020919406309195064091960650919F
:10017000970660918A0770918B0780918C07909108
:100180008D070F94D8036D877E878F87988B20917A
:1001900098063091990640919A0650919B0660917D
:1001A00086077091870780918807909189070F943F
:1001B000D8039E012F5F3F4F4901AE014B5F5F4F58
:1001C0005A01FE0139966F01830172012D853E852A
:1001D0004F855889A3D930C020919806309199064F
:1001E00040919A0650919B0660918607709187070F
:1001F00080918807909189070F94D80369877A873F
:100200008B879C87209194063091950640919606A5
:100210005091970660918A0770918B0780918C07A7
:1002200090918D070F94D8036D837E838F83988779
:1002300049825A826B827C822091D8023091D90205
:100240004091DA025091DB0269857A858B859C8525
:100250000F94E40620E030E040E05FE30F94D80321
:100260000F944A050F94DC04609376077093770728
:1002700080937807909379072091DC023091DD021A
:100280004091DE025091DF026D817E818F819885E1
:100290000F94E40620E030E040E05FE30F94D803E1
:1002A0000F944A050F94DC0460937A0770937B07E0
:1002B00080937C0790937D072091E0023091E102CA
:1002C0004091E2025091E30269817A818B819C81A5
:1002D0000F94E40620E030E040E05FE30F94D803A1
:1002E0000F944A050F94DC0460937E0770937F0798
:1002F0008093800790938107F1010081118106FFAF
:1003000035C180919B0283FD31C1F101C688D78838
:10031000E08CF18C8090E4029090E502A090E602DF
:10032000B090E702A5019401C701B6010F94E4065D
:100330000E94B8710F94DC042B013C018091AF073F
:10034000E0913603F0913703811104C08091AE072C
:100350008823B1F120E030E046E153E462A973A9BB
:1003600084A995A90F943C0487FF08C08091680771
:1003700087FD04C0412C512C320115C0C701B601C4
:100380009F77209196023091970240919802509168
:1003900099020F94E40620E030E04AE754E40F9419
:1003A000700618163CF38091AA079091AB07A091B4
:1003B000AC07B091AD07840D951DA61DB71DDEC01D
:1003C00020E030E046E153E462A973A984A995A92D
:1003D0000F943C0487FF04C08091680787FFD7C053
:1003E0008091AA079091AB07A091AC07B091AD079F
:1003F000A3019201281B390B4A0B5B0BCA01B901FF
:100400000F940F059F7720919602309197024091AB
:100410009802509199020F94E4066B017C0120E050
:1004200030E04AE754E4C501B4010F94E4069B01AF
:10043000AC01C701B6010F94700618160CF4A7C0E2
:1004400040928207509283076092840770928507DA
:1004500010FF3DC08091F2070091A2061091A30603
:100460008823C9F02FE737EB4AE85BE3F101628D9F
:10047000738D848D958D0F94E4066B017C01B8011A
:10048000882777FD8095982F0F940F059B01AC016D
:10049000C701B60112C0B801882777FD8095982F53
:1004A0000F940F05F101228D338D448D558D0F94DE
:1004B000E4062EE333EC4EE259E30F94E406609336
:1004C000A4067093A5068093A6069093A706E090D5
:1004D0008E07F0908F07009190071091910720915F
:1004E0008A0730918B0740918C0750918D0760915E
:1004F0008607709187078091880790918907B2DC01
:10050000811111C08091820790918307A091840787
:10051000B09185078093AA079093AB07A093AC078F
:10052000B093AD070AC0F101808191819C012873CD
:100530003327232BC9F486FD02C080E031C04091EF
:10054000820750918307609184077091850780919D
:10055000AA079091AB07A091AC07B091AD074817DF
:1005600059076A077B0749F381E01AC08091AA07FF
:100570009091AB07A091AC07B091AD078093820733
:1005800090938307A0938407B093850761CF40922F
:10059000AA075092AB076092AC077092AD0750CF9C
:1005A00060960FB6F894DEBF0FBECDBFDF91CF913E
:1005B0001F910F91FF90EF90DF90CF90BF90AF9081
:1005C0009F908F907F906F905F904F903F902F9073
:1005D00008954F925F926F927F92AF92BF92CF92A7
:1005E000DF92EF92FF920F931F93CF93DF93CDB7DC
:1005F000DEB728970FB6F894DEBF0FBECDBF698374
:100600007A838B839C8329013A01ED82FE820F83DA
:10061000188720EF33E244E759E40F943C04882321
:1006200011F1209198063091990640919A065091C7
:100630009B0669817A818B819C810F94D8032091DC
:10064000D8023091D9024091DA025091DB020F9426
:10065000E4060F94DC046093760770937707809329
:1006600078079093790720EF33E244E759E4C30118
:10067000B2010F943C04882301F12091940630913B
:1006800095064091960650919706C301B2010F94CA
:10069000D8032091DC023091DD024091DE025091BE
:1006A000DF020F94E4060F94DC0460937A077093E2
:1006B0007B0780937C0790937D0720EF33E244E72C
:1006C00059E46D817E818F8198850F943C04882345
:1006D000C1F02091E0023091E1024091E20250919C
:1006E000E3026D817E818F8198850F94E4060F94DB
:1006F000DC0460937E0770937F078093800790935C
:10070000810720EF33E244E759E4C601B5010F94B5
:100710003C048823B1F02091E4023091E50240913D
:10072000E6025091E702C601B5010F94E4060F946A
:10073000DC0460938207709383078093840790930F
:10074000850720EF33E244E759E46A8D7B8D8C8D79
:100750009D8D0F943C04882361F08A8D9B8DAC8D18
:10076000BD8D8093A4069093A506A093A606B09392
:10077000A70640E061E081E00E9464ED811106C0BF
:1007800081EA96E10E94FA9C80E003C080E073DA7F
:1007900081E028960FB6F894DEBF0FBECDBFDF9183
:1007A000CF911F910F91FF90EF90DF90CF90BF906E
:1007B000AF907F906F905F904F9008950E94611D61
:1007C00080E059DA8091920790919307A091940765
:1007D000B09195078093850690938606A09387062F
:1007E000B09388068091960790919707A0919807FB
:1007F000B09199078093810690938206A093830617
:10080000B093840680919A0790919B07A0919C07D2
:10081000B0919D0780937D0690937E06A0937F06FE
:10082000B09380066091AA077091AB078091AC07E6
:100830009091AD070F940F052091EE073091EF07CF
:100840004091F0075091F1070F94E4066093790608
:1008500070937A0680937B0690937C068091A40621
:100860009091A506A091A606B091A706809392024A
:1008700090939302A0939402B093950208958F925F
:100880009F92AF92BF92CF92DF92EF92FF920F931F
:100890001F93CF93DF93982EC62FD42FC22E20E024
:1008A00030E0A901609192027091930280919402CC
:1008B000909195020F943C0487FDA7C0911005C04C
:1008C000C11103C0E1E0ED2701C0E0E0CC2049F018
:1008D000A0907906B0907A06C0907B06D0907C06F6
:1008E00008C0F0EFAF2EF3E2BF2EF4E7CF2EF9E40D
:1008F000DF2EE11102C0DD23B9F050917D06409159
:100900007E0630917F0620918006852F942FA32F9D
:10091000B22F80938E0790938F07A0939007B09388
:100920009107E11107C004C050EF43E234E729E426
:10093000CC23B9F0D0918106C091820670918306D4
:10094000609184068D2F9C2FA72FB62F80938A0746
:1009500090938B07A0938C07B0938D07E11107C08C
:1009600004C0D0EFC3E274E769E49920B1F080904D
:10097000850690908606F0918706E0918806C4016E
:10098000AF2FBE2F8093860790938707A093880789
:10099000B0938907B82DA92D04C0B0EFA3E2F4E706
:1009A000E9E41F930F93FF92EF92E52EF42E032FAD
:1009B000122F2D2F3C2F472F562F6B2F7A2F8F2F33
:1009C0009E2F0E947E7B8091920290919302A09133
:1009D0009402B09195028093A4069093A506A093EB
:1009E000A606B093A7060F900F900F900F9080E08F
:1009F000DF91CF911F910F91FF90EF90DF90CF90FB
:100A0000BF90AF909F908F9036C9DF91CF911F918B
:100A10000F91FF90EF90DF90CF90BF90AF909F909D
:100A20008F9008959091690795FB222720F98217EE
:100A300091F0882311F0906201C09F7D9093690727
:100A4000882319F08FED9EE102C089EC9EE10E949F
:100A5000049D80E010C90895AF92BF92CF92DF92BB
:100A6000EF92FF920F931F93CF93E82E062FF42E51
:100A7000C0916907C5FBCC27C0F980E0D3DF909116
:100A80006807916090936807EE2021F0002339F009
:100A90001F2D06C0011103C011E01F2501C010E089
:100AA00040E06CE576E187E19AE00E94CBA887E11F
:100AB0009AE00E941FAC111102C0FF2019F00E94A1
:100AC000FC771FC0EE2041F0109276071092770756
:100AD0001092780710927907002341F010927A075C
:100AE00010927B0710927C0710927D0740E060E037
:100AF00081E00E9464ED811104C084E396E10E94CC
:100B0000FA9CE090AC06F090AD060091AE06109114
:100B1000AF068091C7028F938091C6028F93809118
:100B2000C5028F938091C4028F93A0EFAA2EA3E2F7
:100B3000BA2EA4E7CA2EA9E4DA2E20E030E0A901FB
:100B4000CA01B9010E947E7B81E095D81092800A8B
:100B50008AE296E10E946F1D0F900F900F900F9008
:100B60008C2FCF911F910F91FF90EF90DF90CF903E
:100B7000BF90AF9057CF2F923F924F925F926F925C
:100B80007F928F929F92AF92BF92CF92DF92EF921D
:100B9000FF920F931F93CF93DF93CDB7DEB72B97C1
:100BA0000FB6F894DEBF0FBECDBF6A874D8340916C
:100BB00098065091990660919A0670919B06498318
:100BC0005A836B837C834090940650909506609086
:100BD000960670909706882309F4AEC0222321F070
:100BE0008CE09FE10E947793C0909A07D0909B077A
:100BF000E0909C07F0909D0781EA93E00E94701CB2
:100C00009B01AC01C701B6010F94700618161CF5C4
:100C1000E090C4021091C5020091C602F090C70294
:100C200081EA93E00E94701CFF920F931F93EF9252
:100C300010EFA12E13E2B12E14E7C12E19E4D12E2C
:100C40007B018C01A6019501C601B501C2DC0F90A4
:100C50000F900F900F9080E293E00E94701CDC01D7
:100C6000CB01B0588093980690939906A0939A066A
:100C7000B0939B0684E293E00E94701CDC01CB01E0
:100C8000B0588093940690939506A0939606B093DF
:100C9000970688E493E00E94701CE62E172F082F19
:100CA000F92EA301920160919406709195068091AE
:100CB0009606909197060F94D7032091DC0230910D
:100CC000DD024091DE025091DF020F94E4060F94A2
:100CD000DC042B013C0129813A814B815C816091CC
:100CE00098067091990680919A0690919B060F94B0
:100CF000D7032091D8023091D9024091DA02509165
:100D0000DB020F94E4060F94DC0421E02F932F9371
:100D1000FF920F931F93EF92A12CB12C6501E12C50
:100D2000F12C8701A30192010E9494F20F900F9081
:100D30000F900F900F900F900E94611D20E030E007
:100D400040E251E46091E0027091E1028091E202A0
:100D50009091E3020F94E4060F94DC046E837F838A
:100D6000888799876091A6077091A7078091A80747
:100D70009091A90769837A838B839C838091BA07BA
:100D80009091BB07A091BC07B091BD078093F80676
:100D90009093F906A093FA06B093FB061B86412CAC
:100DA000512C32017D81272E312C7B85872E992471
:100DB00087FC9094821493040CF01FC1C090CC0661
:100DC000D090CD06E090CE06F090CF068091C00680
:100DD0009091C106A091C206B091C306C81AD90A63
:100DE000EA0AFB0ACC0CDD1CEE1CFF1C8FEF9FEF08
:100DF000DC018093E8069093E906A093EA06B0939D
:100E0000EB0680E293E00E94701C84E293E00E9473
:100E1000701C809169078064809369070E94FE229C
:100E20000E94FE220AE010E08091000181FF38C09C
:100E30008CE293E00E94701CA7019601EE24FF242F
:100E40008701E21AF30A040B150B31E03F933F933D
:100E50009F938F937F936F93A12CB12C650120E01A
:100E600030E0A90160E070E0CB010E9494F20F90A5
:100E70000F900F900F900F900F908091E806909137
:100E8000E906A091EA06B091EB06B7FF18C083EA25
:100E90009EE10E940E9D812C912C30E82FEBFAC12F
:100EA0008DE196E10E94ED9C64E670E080E090E0C8
:100EB0000E94A2FE0150110909F0B6CFB9CF80916E
:100EC00069078F7B809369070091F8061091F906F6
:100ED0002091FA063091FB068091BA079091BB07EA
:100EE000A091BC07B091BD07B901A801481B590BDF
:100EF0006A0B7B0BDB01CA014093E8065093E906BD
:100F00006093EA067093EB064091B2075091B307E5
:100F10006091B4077091B507480F591F6A1F7B1F76
:100F20004093B2075093B3076093B4077093B5072B
:100F30004091B6075091B7076091B8077091B90713
:100F4000480F591F6A1F7B1F4093B6075093B7077E
:100F50006093B8077093B9070093BA071093BB0763
:100F60002093BC073093BD074091A6075091A70777
:100F70006091A8077091A907480F591F6A1F7B1F2E
:100F80004093A6075093A7076093A8077093A907FB
:100F900089819A81AB81BC81841B950BA60BB70B11
:100FA000480E591E6A1E7B1EC401019682159305C8
:100FB00004F58CE293E00E94701C1F9251E05F9355
:100FC0009F938F937F936F93A12CB12C6501EE803B
:100FD000FF800885198520E030E0A90160E070E01D
:100FE000CB010E9494F20F900F900F900F900F90F2
:100FF0000F906B856F5F6B87D8CEC301B2010F94E2
:101000000F052091EA073091EB074091EC075091D2
:10101000ED070F94E4066B017C01AD816A2F70E04F
:1010200080E090E00F940D059B01AC01C701B60173
:101030000F9443046B017C0188E293E00E94701CD2
:101040009B01AC01C701B6010F94D8034B018E83FD
:101050009D8322E0AB01BC018BE79FE10E94299FA9
:1010600020E030E040EA52E4B4018E819D810F948B
:10107000E40620E030E048EC54E40F94D703AB01E1
:10108000BC0122E08FE49FE10E94299F40919207DA
:1010900050919307609194077091950722E084EF37
:1010A00092E20E94299F4091960750919707609184
:1010B00098077091990722E080EF92E20E94EC9EDF
:1010C00080E00E943B7E87E196E10E946F1D8CE2EA
:1010D00093E00E94701C9B014091A6075091A707C6
:1010E0006091A8077091A907E980FA800B811C81A3
:1010F000E41AF50A060B170B1F9241E04F939F93DA
:101100008F933F932F93A12CB12C650120E030E009
:10111000A90160E070E0CB010E9494F20F900F9063
:101120000F900F900F900F90BA85BB2309F4B0C0B9
:10113000C0909806D0909906E0909A06F0909B0691
:101140002090940630909506409096065090970611
:101150008BE09FE10E947793609036037090370395
:101160006114710409F444C0F30181819281A38167
:10117000B4819C01AD0166277727CB01621B730BFD
:10118000840B950B0F940F052091E2073091E30734
:101190004091E4075091E5070F94E40660939806A8
:1011A0007093990680939A0690939B06F30185812C
:1011B0009681A781B0859C01AD0166277727CB0179
:1011C000621B730B840B950B0F940F052091E607A0
:1011D0003091E7074091E8075091E9070F94E40642
:1011E0006093940670939506809396069093970665
:1011F00088E493E00E94701C5B01182F092FA20164
:101200009101609194067091950680919606909157
:1012100097060F94D7032091DC023091DD024091B4
:10122000DE025091DF020F94E4060F94DC042B01E0
:101230003C01A701960160919806709199068091F2
:101240009A0690919B060F94D7032091D802309173
:10125000D9024091DA025091DB020F94E4060F9418
:10126000DC0421E02F932F930F931F93BF92AF9233
:10127000A12CB12C6501E12CF12C8701A301920175
:101280000E9494F20F900F900F900F900F900F907C
:101290003E812D81B401832F922F2B960FB6F894A7
:1012A000DEBF0FBECDBFDF91CF911F910F91FF9099
:1012B000EF90DF90CF90BF90AF909F908F907F90F6
:1012C0006F905F904F903F902F90089540E050E0D6
:1012D00060E87FE340935E0750935F076093600789
:1012E0007093610740934E0750934F0760935007E8
:1012F0007093510740933E0750933F076093400718
:101300007093410710925A0710925B0710925C0786
:1013100010925D07109256071092570710925807C7
:1013200010925907109252071092530710925407C7
:101330001092550710924A0710924B0710924C07D3
:1013400010924D07109246071092470710924807D7
:1013500010924907109242071092430710924407D7
:1013600010924507811104C084EF9EE10C94049D06
:10137000089588E10FB6F8948093600010926000A1
:101380000FBE9B9AA398809168078064809368073A
:10139000809104018E7F809304018091050181601A
:1013A00080930501389A399A3A9A80910A018260AD
:1013B00080930A0180910A01816080930A018091E3
:1013C0000A01846080930A010F9A179A0E9A169A5E
:1013D0000D9A159A3F98479A0A98129A0998119A65
:1013E000809101018D7F80930101809102018260D3
:1013F00080930201809101018062809301018091BC
:1014000002018F7D809302016D9A75980E94B92028
:101410000E94DA2181E05ADF80E090E0A8E4B2E4A3
:101420008093A4069093A506A093A606B093A70662
:1014300084E690E09093A3068093A2069093A10681
:101440008093A00610928E0710928F07109290073B
:101450001092910710928A0710928B0710928C07B6
:1014600010928D07109286071092870710928807B6
:101470001092890710923107109230071092221DA6
:101480001092231D1092241D1092251D80E090E0E3
:10149000A0E0B2E480939C0690939D06A0939E06E4
:1014A000B0939F061092940610929506109296069D
:1014B00010929706109298061092990610929A062A
:1014C00010929B0688E893E1A0E0B0E080933A0791
:1014D00090933B07A0933C07B0933D0781E0809336
:1014E0009A0210928E0610928F0610929006109219
:1014F000910610928A0610928B0610928C0610921A
:101500008D068093690780E090E0AAE7B3E48093BA
:10151000BC069093BD06A093BE06B093BF06809311
:10152000B4069093B506A093B606B093B70680E0D4
:1015300090E8A3E9B3E48093AC069093AD06A09342
:10154000AE06B093AF061092B8061092B90610928C
:10155000BA061092BB061092B0061092B106109215
:10156000B2061092B3061092A8061092A906109225
:10157000AA061092AB068CE59FE8A4ECB2E4809337
:10158000180790931907A0931A07B0931B0710929E
:1015900089061092F4071092F3070E9446CA409100
:1015A000EB025091EC026091ED027091EE028AED37
:1015B0009AE00E9415D88BE593E20E94ED9C87E1AA
:1015C0009AE00E94F6A80E9452D50E943A4D0E94CD
:1015D00010D110929E0710929F071092A0071092B0
:1015E000A1071092920710929307109294071092FD
:1015F00095071092A2071092A3071092A4071092C9
:10160000A5071092960710929707109298071092CC
:1016100099071092A6071092A7071092A807109298
:10162000A90710929A0710929B0710929C0710929C
:101630009D071092AA071092AB071092AC07109268
:10164000AD0710929E0710929F071092A00710926C
:10165000A1070E9432720E9418220E9426220E9434
:1016600032D562EB77E08EE997E00E9480E78AEF5F
:1016700093E00F94AE0C90916707882311F092606D
:1016800001C09D7F90936707682F70E081E293E02F
:101690000E94D29D87E696E10E946F1D80E00E9425
:1016A000044E83EC98E00E94F9972EE088E190E0E8
:1016B0000FB6F894A895809360000FBE2093600049
:1016C00008954F925F926F927F928F929F92AF9206
:1016D000BF92CF92DF92EF92FF920F931F93CF931F
:1016E000DF93CDB7DEB764970FB6F894DEBF0FBEB9
:1016F000CDBF4B015C0129013A01E982FA820B83DB
:101700001C8388E393E00E94701C6B017C0180E3E2
:1017100093E00E94701C9B01AC01C701B6010F94BD
:10172000D7036D837E838F8398878CE393E00E9439
:10173000701C6B017C0184E393E00E94701C9B0190
:10174000AC01C701B6010F94D70369877A878B87ED
:101750009C87A3019201C501B4010F94D7032B010B
:101760003C0180E493E00E94701C6B017C0180E3EB
:1017700093E00E94701C9B01AC01C701B6010F945D
:10178000D7036D877E878F87988B84E493E00E94D0
:10179000701C6B017C0184E393E00E94701C9B0130
:1017A000AC01C701B6010F94D703698B7A8B8B8B81
:1017B0009C8B29813A814B815C81C501B4010F94D6
:1017C000D7034B015C019B01AC0169857A858B8550
:1017D0009C850F94E4066B017C0129893A894B8929
:1017E0005C89C301B2010F94E4069B01AC01C701FF
:1017F000B6010F94D70369837A838B839C832D85ED
:101800003E854F855889C301B2010F94E4066B01F0
:101810007C01A50194016D817E818F8198850F9453
:10182000E4069B01AC01C701B6010F94D7032B015D
:101830003C0129893A894B895C896D817E818F8140
:1018400098850F94E4066B017C012D853E854F85BC
:10185000588969857A858B859C850F94E4069B0160
:10186000AC01C701B6010F94D7034B015C0129817C
:101870003A814B815C81CA01B9010F94E4066B0186
:101880007C01A3019201C301B2010F94E4069B0104
:10189000AC01C701B6010F94D8036B017C01A5010F
:1018A0009401C501B4010F94E4069B01AC01C7018A
:1018B000B6010F94D8030F9451076B017C0120E00F
:1018C00030E0A901C501B4010F943C0487FF04C0B6
:1018D000F7FAF094F7F8F094A701960169817A81FC
:1018E0008B819C810F9443046D837E838F839887C3
:1018F0006093560770935707809358079093590742
:10190000A7019601C301B2010F9443042B013C01CE
:1019100060935A0770935B0780935C0790935D0711
:10192000A7019601C501B4010F9443046B017C012A
:1019300060935E0770935F078093600790936107E1
:1019400010924A0710924B0710924C0710924D07C5
:10195000D301C201B05889839A83AB83BC83A701AA
:101960009601C701B6010F94E4066D877E878F87C5
:10197000988BA301920169817A818B819C810F945C
:10198000E4069B01AC016D857E858F8598890F9457
:10199000D70369877A878B879C872D813E814F810A
:1019A000588569817A818B819C810F94E4064B0173
:1019B0005C0120E030E0A901C701B6010F94E40604
:1019C0009B01AC01C501B4010F94D703609342079A
:1019D00070934307809344079093450720E030E0DD
:1019E000A901C301B2010F94E4064B015C012D81F2
:1019F0003E814F815885C701B6010F94E4069B01D3
:101A0000AC01C501B4010F94D7034B015C012985DA
:101A10003A854B855C85CA01B9010F94E4062B0118
:101A20003C01A5019401C501B4010F94E4069B019A
:101A3000AC01C301B2010F94D8030F9451072B01DD
:101A40003C019B01AC0169857A858B859C850F944F
:101A5000430460933E0770933F0780934007909341
:101A60004107A3019201C501B4010F94430460939F
:101A70004607709347078093480790934907298149
:101A80003A814B815C81CA01B9010F94E4069B0144
:101A9000AC016D857E858F8598890F94D8030F944E
:101AA00051074B015C019B01AC01C701B6010F94CA
:101AB000430460934E0770934F07809350079093B1
:101AC0005107A501940169817A818B819C810F94D2
:101AD0004304609352077093530780935407909385
:101AE000550726E049E06EE377E082EB9EE16496DD
:101AF0000FB6F894DEBF0FBECDBFDF91CF911F911F
:101B00000F91FF90EF90DF90CF90BF90AF909F909C
:101B10008F907F906F905F904F900C94429F0895AC
:101B200088E096E10C94049DE9E5F6E011821082CC
:101B3000349686E0E937F807C9F708954091EB023B
:101B40005091EC026091ED027091EE028EEF95E102
:101B50000E942A9E6FE770E081EF95E10E94E09D70
:101B600061E070E084EE95E10E94E09D60E070E04D
:101B700084ED95E10E94E09D60E070E089EC95E1E4
:101B80000E94E09D61E070E081EC95E10E94E09DA3
:101B900061E070E08CEB95E10E94E09D61E070E017
:101BA00087EB95E10E94E09D61E070E082EA95E1BB
:101BB0000E94E09D61E070E088E995E10E94E09D6F
:101BC00061E070E08EE895E10E94E09D61E070E0E8
:101BD00084E895E10E94E09D60E070E085E795E192
:101BE0000E94E09D60E070E089E595E10E94E09D43
:101BF00060E070E08DE495E10E94E09D61E070E0BE
:101C000085E495E10E94E09D61E070E08AE395E162
